:020000040000FA
:1000000000040020990900002D0600007909000075
:1000100037060000410600004B060000000000000B
:10002000000000000000000000000000BD0900000A
:1000300055060000000000005F0600006906000091
:10004000730600007D060000870600009106000090
:100050009B060000A5060000AF060000B9060000E0
:10006000C3060000CD060000D7060000E106000030
:10007000EB060000F5060000FF060000090700007F
:10008000130700001D0700002707000031070000CC
:100090003B070000450700004F070000590700001C
:1000A000630700006D07000077070000810700006C
:1000B0008B070000950700009F070000A9070000BC
:1000C000B3070000BD070000C7070000D10700000C
:1000D000DB070000E5070000EF070000F90700005C
:1000E000030800000D0800001708000021080000A8
:1000F0002B080000350800003F08000049080000F8
:10010000530800001FB500F003F88DE80F001FBD75
:1001100000F038BC70B50B46010B184400F6FF70B8
:10012000040B4FF080500022090303692403406947
:1001300043431D1B104600F0E9F929462046BDE85F
:10014000704000F0E3B9F0B54FF6FF734FF4B475AB
:100150001A466E1E12E0A94201D3344600E00C4656
:10016000B1EB040130F8027B641E3B441A44F9D120
:100170009CB204EB134394B204EB12420029EAD17F
:1001800098B200EB134002EB124140EA0140F0BD8F
:10019000C34992B00446D1E90001CDE91001FF2224
:1001A0004021684600F094FB94E80F008DE80F00B2
:1001B000684610A902E004C841F8042D8842FAD12B
:1001C00010216846FFF7BFFF1090AA208DF8440069
:1001D00000F0FAF800F0DDF84FF01024A0691022CA
:1001E0006946803000F0DEF8A069082210A900F00E
:1001F000D9F800F0C2F870B504460068A94D072888
:1002000069D2DFE800F033041929561E2500D4E92D
:10021000026564682946304600F0FDF82A4621460A
:10022000304600F0BFF8AA002146304600F024FB1B
:10023000002800D0032070BD00F0D6FB4FF48050A2
:1002400007E0201D00F0C6F80028F4D100F0CCFB38
:1002500060682860002070BD241D94E807009200AB
:1002600000F00AFB0028F6D00E2070BD00F0BEF8AA
:100270000028FAD1D4E9010100EB81034FF080504E
:10028000026945696A43934209D84FF010225369C5
:1002900003EB81030169406941438B4201D9092085
:1002A00070BD5069401C01D10F2070BD2046FFF782
:1002B0006FFF00F09BF80028F7D1201D00F08AF8AE
:1002C0000028F2D160680028F0D100F07DF800F03D
:1002D00060F800F052F8072070BD10B50C461828E1
:1002E00002D00120086010BD2068FFF784FF206065
:1002F00010BD4FF01024A069401C05D0A569A66967
:1003000080353079AA2808D06069401C2DD06069FA
:100310000068401C29D060692CE010212846FFF7B6
:1003200012FF316881421CD1A16901F18002C03104
:1003300005E030B108CA51F8040D984201D10120FE
:1003400000E000208A42F4D158B1286810B1042896
:1003500003D0FEE7284600F070F85249686808604C
:1003600008E000F016F800F008F84FF4805001683B
:10037000491C01D000F012FBFEE7BFF34F8F4A4843
:1003800001684A4A01F4E06111430160BFF34F8FF5
:10039000FEE74FF010208169491C02D0806900F00F
:1003A0008CB870472DE9F04117460D4606460024EB
:1003B00006E03046296800F093F8641C2D1D361DB8
:1003C000BC42F6D3BDE8F0814FF0102080694FF4B5
:1003D00080519FE64FF080510A69496900684A439D
:1003E000824201D810207047002070474FF08050A3
:1003F0000169406941434FF01020826902F5805243
:10040000914201D2092070478069401C01D0002030
:1004100070470420704770B50C4605464FF480665F
:1004200008E0284600F049F8B44205D3A4F58064FA
:1004300005F58055002CF4D170BD4168044609B122
:10044000012600E000264FF010256869A26892009E
:1004500000F012FAF8B1A06881006869FFF75AFE4F
:10046000BEB16E694FF08050A56864680169426949
:100470005143A1420DD9016940694143A94208D9BC
:1004800029463046FFF7C7FF2A4621463046FFF788
:1004900089FFFFF772FFFFF797FFFFF77AFFF8E793
:1004A0000C0A0000000000200CED00E00400FA053A
:1004B000144801680029FCD07047134A02211160DA
:1004C00010490B68002BFCD00F4B1B1D18600868EF
:1004D0000028FCD00020106008680028FCD070477D
:1004E000094B10B501221A60064A1468002CFCD092
:1004F000016010680028FCD00020186010680028F7
:10050000FCD010BD00E4014004E5014070B50C468C
:10051000054600F073F810B900F07EF828B12146C6
:100520002846BDE8704000F007B821462846BDE8DF
:10053000704000F037B800007FB5002200920192B1
:10054000029203920A0B000B6946012302440AE05F
:10055000440900F01F0651F8245003FA06F635430B
:1005600041F82450401C8242F2D80D490868009A94
:1005700010430860081D0168019A1143016000F0F2
:100580003DF800280AD0064910310868029A104345
:100590000860091D0868039A104308607FBD0000C9
:1005A0000006004030B50F4C002200BF04EB0213E0
:1005B000D3F800582DB9D3F8045815B9D3F8085812
:1005C0001DB1521C082AF1D330BD082AFCD204EB1D
:1005D0000212C2F80008C3F804180220C3F8080881
:1005E00030BD000000E001404FF08050D0F83001F5
:1005F000082801D000207047012070474FF080503C
:10060000D0F83011062905D0D0F83001401C01D0B7
:1006100000207047012070474FF08050D0F8300123
:100620000A2801D0002070470120704708208F4918
:1006300009680958084710208C4909680958084773
:1006400014208A4909680958084718208749096809
:100650000958084730208549096809580847382053
:1006600082490968095808473C20804909680958A7
:10067000084740207D4909680958084744207B49BC
:1006800009680958084748207849096809580847FF
:100690004C20764909680958084750207349096871
:1006A00009580847542071490968095808475820D3
:1006B0006E490968095808475C206C49096809585F
:1006C0000847602069490968095808476420674954
:1006D00009680958084768206449096809580847A3
:1006E0006C20624909680958084770205F49096809
:1006F0000958084774205D49096809580847782057
:100700005A490968095808477C2058490968095816
:1007100008478020554909680958084784205349EB
:100720000968095808478820504909680958084746
:100730008C204E4909680958084790204B490968A0
:1007400009580847942049490968095808479820DA
:1007500046490968095808479C20444909680958CE
:100760000847A0204149096809580847A4203F4983
:10077000096809580847A8203C49096809580847EA
:10078000AC203A49096809580847B0203749096838
:1007900009580847B4203549096809580847B8205E
:1007A0003249096809580847BC2030490968095886
:1007B0000847C0202D49096809580847C4202B491B
:1007C000096809580847C82028490968095808478E
:1007D000CC202649096809580847D02023490968D0
:1007E00009580847D4202149096809580847D820E2
:1007F0001E49096809580847DC201C49096809583E
:100800000847E0201949096809580847E4201749B2
:10081000096809580847E820144909680958084731
:10082000EC201249096809580847F0200F49096867
:1008300009580847F4200D49096809580847F82065
:100840000A49096809580847FC20084909680958F5
:1008500008475FF480700549096809580847000097
:1008600003480449024A034B70470000000000207F
:10087000180A0000180A000040EA010310B59B079F
:100880000FD1042A0DD310C808C9121F9C42F8D0FA
:1008900020BA19BA884201D9012010BD4FF0FF30AB
:1008A00010BD1AB1D30703D0521C07E0002010BDC1
:1008B00010F8013B11F8014B1B1B07D110F8013B4D
:1008C00011F8014B1B1B01D1921EF1D1184610BD2E
:1008D00002F0FF0343EA032242EA024200F005B8B5
:1008E0007047704770474FF000020429C0F0128033
:1008F00010F0030C00F01B80CCF1040CBCF1020FD3
:1009000018BF00F8012BA8BF20F8022BA1EB0C01A7
:1009100000F00DB85FEAC17C24BF00F8012B00F89D
:10092000012B48BF00F8012B70474FF0000200B5C3
:10093000134694469646203922BFA0E80C50A0E802
:100940000C50B1F12001BFF4F7AF090728BFA0E8B0
:100950000C5048BF0CC05DF804EB890028BF40F87C
:10096000042B08BF704748BF20F8022B11F0804FBE
:1009700018BF00F8012B7047014B1B68DB68184754
:100980000000002009480A497047FFF7FBFFFFF706
:10099000B9FB00BD20BFFDE7064B1847064A1060B3
:1009A000016881F30888406800470000180A0000C9
:1009B000180A0000F3020000000000201EF0040FDF
:1009C0000CBFEFF30881EFF30981886902380078E2
:1009D000182803D100E00000074A1047074A1268B0
:1009E0002C3212681047000000B5054B1B68054A01
:1009F0009B58984700BD0000DB020000000000206B
:100A0000080A0000040000000010000000000000C0
:080A100000FFFFFF0090D0037E
:10100000801300204958020045C00000AF5702007D
:1010100045C0000045C0000045C0000000000000C1
:10102000000000000000000000000000A5580200C1
:1010300045C000000000000045C0000045C00000A1
:101040000D5902001359020045C0000045C00000C0
:1010500045C0000045C0000045C0000045C000007C
:101060001959020045C0000045C000001F59020088
:1010700045C00000255902002B59020031590200D9
:1010800045C0000045C0000045C0000045C000004C
:1010900045C0000045C0000045C0000045C000003C
:1010A00045C000003759020045C0000045C000009F
:1010B00045C0000045C0000045C0000045C000001C
:1010C0003D59020045C0000045C0000045C0000079
:1010D00045C0000045C0000045C0000045C00000FC
:1010E00045C0000045C0000045C0000045C00000EC
:1010F00045C0000045C0000045C0000045C00000DC
:1011000045C0000045C0000000F002F824F08BFB51
:101110000AA090E8000C82448344AAF10107DA4552
:1011200001D124F080FBAFF2090EBAE80F0013F0F2
:10113000010F18BFFB1A43F001031847EC4C0200E3
:101140000C4D02000A444FF0000C10F8013B13F064
:10115000070408BF10F8014B1D1108BF10F8015B10
:10116000641E05D010F8016B641E01F8016BF9D103
:1011700013F0080F1EBF10F8014BAD1C0C1B09D15A
:101180006D1E58BF01F801CBFAD505E014F8016BCC
:1011900001F8016B6D1EF9D59142D6D3704700005E
:1011A0000023002400250026103A28BF78C1FBD870
:1011B000520728BF30C148BF0B6070471FB500F011
:1011C0003DF88DE80F001FBD1EF0040F0CBFEFF3BC
:1011D0000880EFF30980014A1047000087BF000034
:1011E000F0B44046494652465B460FB402A0013077
:1011F00001B50648004700BF01BC86460FBC8046CB
:10120000894692469B46F0BC7047000009110000D9
:101210008269034981614FF001001044704700006A
:101220002512000001B41EB400B514F08DFE01B407
:101230000198864601BC01B01EBD000024F0F0BA42
:1012400070B51A4C054609202070A01C00F0D1F89A
:101250005920A08029462046BDE8704008F0BAB861
:1012600008F0C3B870B50C461149097829B1A0F14E
:1012700060015E2908D3012013E0602804D06928AA
:1012800002D043F201000CE020CC0A4E94E80E009C
:1012900006EB8000A0F58050241FD0F8806E284611
:1012A000B047206070BD012070470000080000209A
:1012B00018000020885902003249884201D20120DA
:1012C00070470020704770B50446A0F500002E4E10
:1012D000B0F1786F02D23444A4F500042948844266
:1012E00001D2012500E0002500F043F848B125B9FE
:1012F000B44204D32548006808E0012070BD0020F6
:1013000070BD002DF9D1B442F9D321488442F6D200
:10131000F3E710B50446A0F50000B0F1786F03D2F2
:1013200019480444A4F5000400F023F84FF080416C
:1013300030B11648006804E08C4204D2012003E07A
:1013400013488442F8D2002080F0010010BD10B58F
:1013500020B1FFF7DEFF08B1012010BD002010BD55
:1013600010B520B1FFF7AFFF08B1012010BD00207C
:1013700010BD084808490068884201D10120704723
:101380000020704700600200000000201C000020C8
:101390000800002054000020BEBAFECA10B5044662
:1013A0000021012000F03DF800210B2000F039F869
:1013B0000421192000F035F804210D2000F031F847
:1013C00004210E2000F02DF804210F2000F029F850
:1013D0000421C84300F025F80621162000F021F86A
:1013E0000621152000F01DF82046FFF729FF0020F8
:1013F00010BDAE2101807047FFF732BF1148704722
:1014000010487047104A10B514680F4B0F4A083344
:101410001A60FFF727FF0C48001D046010BD7047DD
:1014200070474907090E002804DB00F1E02080F82E
:101430000014704700F00F0000F1E02080F8141D48
:101440007047000003F9004210050240010000014E
:10145000FE48002101604160018170472DE9F7439A
:10146000044692B091464068FFF771FF40B1606852
:10147000FFF776FF20B9607800F00300022801D062
:10148000012000E00020F14E30724846FFF71BFFBC
:1014900018B1102015B0BDE8F0834946012001F0D5
:1014A0008EFE0028F6D101258DF842504FF4C05031
:1014B000ADF84000002210A9284606F001FC0028E3
:1014C000E8D18DF842504FF428504FF00008ADF8A5
:1014D000400047461C216846CDF81C8024F03BF9AB
:1014E0009DF81C0008AA20F00F00401C20F0F0001E
:1014F00010308DF81C0020788DF81D0061789DF863
:101500001E0061F3420040F001008DF81E009DF8BE
:1015100000000AA940F002008DF800002089ADF813
:101520003000ADF83270608907AFADF834000B972A
:10153000606810AC0E900A94684606F0B4F9002872
:10154000A8D1BDF8200030808DF8425042F601202D
:10155000ADF840009DF81E0008AA20F00600801C8F
:1015600020F001008DF81E000220ADF83000ADF82B
:10157000340013A80E900AA9684606F094F90028D2
:1015800088D1BDF820007080311D484600F033F945
:10159000002887D18DF8425042F6A620ADF84000D1
:1015A0001C216846CDF81C8024F0D5F89DF81C005D
:1015B000ADF8345020F00F00401C20F0F000103047
:1015C0008DF81C009DF81D0008AA20F0FF008DF882
:1015D0001D009DF81E000AA920F0060040F0010041
:1015E000801C8DF81E009DF800008DF8445040F0DE
:1015F00002008DF80000CDE90A4711A80E90ADF861
:101600003050684606F04FF9002899D1BDF8200007
:10161000F08000203EE73EB504460820ADF800000B
:101620002046FFF750FE08B110203EBD21460120A4
:1016300001F0C5FD0028F8D12088ADF804006088CD
:10164000ADF80600A088ADF80800E088ADF80A0003
:101650007E4801AB6A468088002106F02DFDBDF86A
:1016600000100829E1D003203EBD1FB5044600202C
:1016700002900820ADF80800CDF80CD02046FFF706
:1016800022FE10B1102004B010BD704802AA81885B
:101690004FF6FF7006F052FF0028F4D1BDF8081095
:1016A000082901D00320EEE7BDF800102180BDF825
:1016B00002106180BDF80410A180BDF80610E18021
:1016C000E1E701B582B00220ADF800005F4802AB4F
:1016D0006A464088002106F0EFFCBDF800100229A0
:1016E00000D003200EBD1CB5002100910221ADF8F1
:1016F00000100190FFF70DFE08B110201CBD5348EB
:101700006A4641884FF6FF7006F018FFBDF80010DA
:101710000229F3D003201CBDFEB54C4C06461546ED
:10172000207A0F46C00705D00846FFF7CCFD18B158
:101730001020FEBD0F20FEBDF82D01D90C20FEBDEE
:101740003046FFF7C0FD18BB208801A905F0B0FDA9
:101750000028F4D130788DF80500208801A906F022
:1017600089FC0028EBD100909DF800009DF8051041
:1017700040F002008DF80000090703D040F0080097
:101780008DF800002088694606F011FC0028D6D1AB
:10179000ADF8085020883B4602AA002106F08CFCD8
:1017A000BDF80810A942CAD00320FEBD7CB505468D
:1017B0000020009001900888ADF800000C462846F3
:1017C0000195FFF7C4FD18B92046FFF7A2FD08B147
:1017D00010207CBD15B1BDF8000050B11B486A4611
:1017E00001884FF6FF7006F0A9FEBDF800102180B9
:1017F0007CBD0C207CBD30B593B0044600200D4666
:101800000090142101A823F0A6FF1C2108A823F0B2
:10181000A2FF9DF80000CDF808D020F00F00401C7A
:1018200020F0F00010308DF800009DF8010020F04D
:10183000FF008DF801009DF8200040F002008DF8B7
:10184000200001208DF8460002E000001C0200206C
:1018500042F60420ADF8440011A801902088ADF8AC
:101860003C006088ADF83E00A088ADF84000E088FC
:10187000ADF842009DF8020006AA20F00600801C88
:1018800020F001008DF802000820ADF80C00ADF842
:1018900010000FA8059001A908A806F004F8002878
:1018A00003D1BDF818002880002013B030BD00001F
:1018B000F0B5007B059F1E4614460D46012800D05A
:1018C000FFDF0C2030803A203880002C08D0287AA6
:1018D000032806D0287B012800D0FFDF1720608175
:1018E000F0BDA889FBE72DE9F04786B0144691F8D2
:1018F0000C900E9A0D46B9F1010F0BD01021007B10
:101900002E8A8846052807D0062833D0FFDF06B088
:10191000BDE8F0870221F2E7E8890C2100EB4000E6
:1019200001EB4000188033201080002CEFD0E889B4
:10193000608100271AE00096688808F1020301AA76
:10194000696900F084FF06EB0800801C07EB470183
:1019500086B204EB4102BDF8040090810DF106014E
:1019600040460E3212F09DFD7F1CBFB26089B84226
:10197000E1D8CCE734201080E889B9F1010F11D00B
:10198000122148430E301880002CC0D0E8896081B5
:101990004846B9F1010F00D00220207300270DF155
:1019A000040A1FE00621ECE70096688808F10203AC
:1019B00001AA696900F04BFF06EB0800801C86B2A3
:1019C000B9F1010F12D007EBC70004EB4000BDF8DE
:1019D0000410C18110220AF10201103023F01AFE16
:1019E0007F1CBFB26089B842DED890E707EB4701A1
:1019F00004EB4102BDF80400D0810AF10201404627
:101A0000103212F04EFDEBE72DE9F0470E4688B09C
:101A100090F80CC096F80C80378AF5890C20109944
:101A200002F10C044FF0000ABCF1030F08D0BCF126
:101A3000040F3ED0BCF1070F7DD0FFDF08B067E791
:101A400005EB850C00EB4C00188031200880002A43
:101A5000F4D0A8F1060000F0FF09558125E0182117
:101A600001A823F078FE00977088434601AA7169A7
:101A700000F0EDFEBDF804002080BDF80600E08017
:101A8000BDF808002081A21C0DF10A01484612F0A1
:101A900008FDB9F1000F00D018B184F804A0A4F833
:101AA00002A007EB080087B20A346D1EADB2D6D291
:101AB000C4E705EB850C00EB4C0018803220088051
:101AC000002ABBD0A8F1050000F0FF09558137E0DE
:101AD00000977088434601AA716900F0B8FE9DF82E
:101AE0000600BDF80410E1802179420860F300018E
:101AF00062F34101820862F38201C20862F3C3010A
:101B0000020962F30411420962F34511820962F38A
:101B100086112171C0096071BDF80700208122463D
:101B20000DF10901484612F0BCFC18B184F802A07E
:101B3000A4F800A000E007E007EB080087B20A3431
:101B40006D1EADB2C4D279E7A8F1020084B205FBE4
:101B500008F000F10E0CA3F800C035230B80002A1A
:101B6000A6D055819481009783B270880E32716936
:101B700000F06DFE62E72DE9F84F1E460A9D0C4607
:101B800081462AB1607A00F58070D080E0891081AA
:101B900099F80C000C274FF000084FF00E0A0D28A2
:101BA00073D2DFE800F09E070E1C28303846556AD5
:101BB00073737300214648460095FFF779FEBDE830
:101BC000F88F207B9146082802D0032800D0FFDF41
:101BD000378030200AE000BFA9F80A80EFE7207BB9
:101BE0009146042800D0FFDF378031202880B9F1EA
:101BF000000FF1D1E3E7207B9146042800D0FFDFFE
:101C000037803220F2E7207B9146022800D0FFDFA8
:101C100037803320EAE7207B1746022800D0FFDF19
:101C20003420A6F800A02880002FC8D0A7F80A808A
:101C3000C5E7207B1746042800D0FFDF3520A6F833
:101C400000A02880002FBAD04046A7F80A8012E0F2
:101C5000207B1746052802D0062800D0FFDF102081
:101C6000308036202880002FA9D0E0897881A7F81D
:101C70000E80B9F80E00B881A1E7207B91460728B5
:101C800000D0FFDF37803720B0E72AE04FF01200A6
:101C900018804FF038001700288090D0E0897881B4
:101CA000A7F80E80A7F8108099F80C000A2805D034
:101CB0000B2809D00C280DD0FFDF80E7207B0A28F5
:101CC00000D0FFDF01200AE0207B0B2800D0FFDFDF
:101CD000042004E0207B0C2800D0FFDF05203873AF
:101CE0006DE7FFDF6BE770B50C46054601F0ABFB17
:101CF00020B10078222804D2082070BD43F20200EF
:101D000070BD0521284610F03FFE206008B100207C
:101D100070BD032070BD30B44880087820F00F00FB
:101D2000C01C20F0F000903001F8080B1DCA81E8BB
:101D30001D0030BC07F0CFBB2DE9FF4784B0002762
:101D40008246029707989046894612300AF0CAF9EF
:101D5000401D20F00306079828B907A95046FFF751
:101D6000C2FF002854D1B9F1000F05D00798017BBC
:101D700019BB052504681BE098F80000092803D06A
:101D80000D2812D0FFDF46E0079903254868B0B35D
:101D9000497B42887143914239D98AB2B3B2011D5D
:101DA00010F065FC0446078002E0079C0425083417
:101DB0000CB1208810B1032D29D02CE00798012107
:101DC00012300AF0C1F9ADF80C00024602AB294608
:101DD000504608F0EEF9070001D1A01C02900798C8
:101DE0003A461230C8F80400A8F802A003A94046F9
:101DF000029B0AF0B6F9D8B10A2817D200E006E033
:101E0000DFE800F007091414100B0D14141213204E
:101E100014E6002012E6112010E608200EE643F238
:101E200003000BE6072009E60D2007E6032005E680
:101E3000BDF80C002346CDE900702A4650460799AC
:101E400000F015FD57B9032D08D10798B3B2417BB7
:101E5000406871438AB2011D10F01DFCB9F1000FFA
:101E6000D7D0079981F80C90D3E72DE9FE4F914622
:101E70001A881C468A468046FAB102AB494608F0E9
:101E800098F9050019D04046A61C278810F0C0FE1E
:101E90003246072629463B46009610F0CEFA2088A7
:101EA0002346CDE900504A465146404600F0DFFC4B
:101EB000002020800120BDE8FE8F0020FBE710B548
:101EC00086B01C46AAB104238DF800301388ADF803
:101ED00008305288ADF80A208A788DF80E200988DB
:101EE000ADF80C1000236A462146FFF725FF06B027
:101EF00010BD1020FBE770B50D46052110F044FD24
:101F0000040000D1FFDF294604F11200BDE8704053
:101F10000AF003B92DE9F8430D468046002607F084
:101F2000D7FA04462878102878D2DFE800F0773B0B
:101F30003453313112313131083131313131287975
:101F4000001FC0B2022801D0102810D114BBFFDF3F
:101F500035E004B9FFDF0521404610F015FD007B98
:101F6000032806D004280BD0072828D0FFDF072637
:101F700055E02879801FC0B2022820D050B1F6E782
:101F80002879401FC0B2022819D0102817D0EEE7D8
:101F900004B9FFDF13E004B9FFDF287901280ED16F
:101FA000172137E00521404610F0EEFC070000D174
:101FB000FFDF07F1120140460AF08CF82CB12A46E7
:101FC00021464046FFF7A7FE29E01321404602F0D4
:101FD000F7FC24E004B9FFDF0521404610F0D4FCF3
:101FE000060000D1FFDF694606F112000AF07CF816
:101FF000060000D0FFDFA988172901D2172200E0D0
:102000000A46BDF80000824202D9014602E005E01E
:102010001729C5D3404600F03AFCD0E7FFDF304631
:10202000BDE8F883401D20F0030219B102FB01F066
:10203000001D00E000201044704713B5009848B11F
:102040000024684610F0BDFA002C02D1F74A00992E
:1020500011601CBD01240020F4E72DE9F0470C4677
:1020600015462421204623F076FB05B9FFDFA8782A
:1020700060732888DFF8B4A3401D20F00301AF7817
:102080008946DAF8000010F0BAFA060000D1FFDF46
:102090004FF000082660A6F8008077B109FB07F131
:1020A000091D0AD0DAF8000010F0A9FA060000D1E4
:1020B000FFDF6660C6F8008001E0C4F8048029886C
:1020C00004F11200BDE8F04709F0F6BF2DE9F04732
:1020D000804601F112000D4681460AF003F8401DCA
:1020E000D24F20F003026E7B14462968386810F046
:1020F000B1FA3EB104FB06F2121D03D069683868DC
:1021000010F0A8FA052010F0E7FB0446052010F0B7
:10211000EBFB201A012802D1386810F065FA494615
:102120004046BDE8F04709F0DCBF70B50546052123
:1021300010F02AFC040000D1FFDF04F11201284650
:10214000BDE8704009F0C6BF2DE9F04F91B04FF0E7
:10215000000BADF834B0ADF804B047880C46054626
:1021600092460521384610F00FFC060000D1FFDF33
:1021700024B1A780A4F806B0A4F808B029780922F1
:102180000B20B2EB111F7DD12A7A04F11001382700
:102190004FF00C084FF001090391102A73D2DFE8C9
:1021A00002F072F2F1F07F08D2888D9F3DDBF3EEF2
:1021B000B6B6307B022800D0FFDFA88908EBC0014B
:1021C000ADF804103021ADF83410002C25D060811A
:1021D000B5F80E9000271DE004EBC708317C88F8A5
:1021E0000E10F189A8F80C10CDF80090688804232F
:1021F00004AA296900F02BFBBDF81010A8F81010F4
:1022000009F10400BDF812107F1C1FFA80F9A8F82C
:102210001210BFB26089B842DED80DE1307B0228CF
:1022200000D0FFDFE98908EBC100ADF804003020E1
:10223000ADF83400287B0A90001FC0B20F90002C2C
:10224000EBD06181B5F81090002725E0CDF8009023
:102250006888696903AA0A9B00F0F9FA0A9804EBF6
:10226000C70848441FFA80F908F10C0204A90F9826
:1022700012F017F918B188F80EB0A8F80CB0BDF834
:102280000C1001E0D4E0CFE0A8F81010BDF80E105B
:102290007F1CA8F81210BFB26089B842D6D8CBE034
:1022A0000DA8009001AB224629463046FFF71BFBE4
:1022B000C2E0307B082805D0FFDF03E0307B082830
:1022C00000D0FFDFE8891030ADF804003620ADF80B
:1022D0003400002C3FD0A9896181F189A18127E0D8
:1022E000307B092800D0FFDFA88900F10C01ADF890
:1022F00004103721ADF83410002C2CD06081E8890F
:102300000090AB89688804F10C02296956E0E889DD
:102310003921103080B2ADF80400ADF83410002C33
:1023200074D0A9896181287A0E280AD002212173EC
:10233000E989E181288A0090EB8968886969039AB4
:102340003CE00121F3E70DA8009001AB22462946AD
:102350003046FFF759FB6FE0307B0A2800D0FFDFE3
:102360001220ADF80400ADF834704CB3A989618136
:10237000A4F810B0A4F80EB084F80C905CE020E053
:1023800002E031E039E042E0307B0B2800D0FFDF93
:10239000288AADF834701230ADF8040084B10421FD
:1023A0002173A9896181E989E181298A2182688A69
:1023B00000902B8A688804F11202696900F047FADC
:1023C0003AE0307B0C2800D0FFDF1220ADF804008B
:1023D000ADF834703CB305212173A4F80AB0A4F819
:1023E0000EB0A4F810B027E00DA8009001AB224673
:1023F00029463046FFF75CFA1EE00DA8009001ABBD
:10240000224629463046FFF7B6FB15E034E03B2173
:10241000ADF80400ADF8341074B3A4F80690A4F835
:1024200008B084F80AB007E0FFDF05E010000020E4
:10243000297A012917D0FFDFBDF80400AAF80000AF
:102440006CB1BDF834002080BDF804006080BDF898
:102450003400392803D03C2801D086F80CB011B0E4
:102460000020BDE8F08F3C21ADF80400ADF8341039
:1024700014B1697AA172DFE7AAF80000EFE72DE94D
:10248000F84356880F46804615460521304610F021
:102490007BFA040000D1FFDF123400943B46414632
:1024A00030466A6809F091FFBAE570B50D4605211E
:1024B00010F06AFA040000D1FFDF294604F112008F
:1024C000BDE8704009F01BBE70B50D46052110F047
:1024D0005BFA040000D1FFDF294604F11200BDE8D9
:1024E000704009F039BE70B50546052110F04CFA70
:1024F000040000D1FFDF04F1080321462846BDE8AF
:1025000070400422B1E470B50546052110F03CFA94
:10251000040000D1FFDF214628462368BDE8704053
:102520000522A2E470B50646052110F02DFA04003C
:1025300000D1FFDF04F1120009F0D4FD401D20F0AE
:10254000030511E0011D008803224318214630468F
:10255000FFF78BFC00280BD0607BABB2684382B2E4
:102560006068011D10F0CDF8606841880029E9D14C
:1025700070BD70B50E46054606F0AAFF040000D1F6
:10258000FFDF0120207266726580207820F00F0046
:10259000C01C20F0F00030302070BDE8704006F024
:1025A0009ABF2DE9F0438BB00D461446814606A92B
:1025B000FFF799FB002814D14FF6FF7601274FF45F
:1025C00020588CB103208DF800001020ADF81000C9
:1025D00007A8059007AA204604A911F081FF78B149
:1025E00007200BB0BDE8F0830820ADF808508DF847
:1025F0000E708DF80000ADF80A60ADF80C800CE0AC
:102600000698A17801742188C1818DF80E70ADF80B
:102610000850ADF80C80ADF80A606A4602214846C1
:10262000069BFFF789FBDCE708B501228DF8022045
:1026300042F60202ADF800200A4603236946FFF77E
:102640003EFC08BD08B501228DF8022042F60302C7
:10265000ADF800200A4604236946FFF730FC08BDA8
:1026600000B587B079B102228DF800200A88ADF854
:1026700008204988ADF80A1000236A460521FFF7B3
:102680005BFB07B000BD1020FBE709B1072316E490
:102690000720704770B588B00D461446064606A957
:1026A000FFF721FB00280ED17CB10620ADF80850C1
:1026B0008DF80000ADF80A40069B6A460821DC81CF
:1026C0003046FFF739FB08B070BD05208DF80000DB
:1026D000ADF80850F0E700B587B059B107238DF881
:1026E0000030ADF80820039100236A460921FFF766
:1026F00023FBC6E71020C4E770B588B00C46064639
:10270000002506A9FFF7EFFA0028DCD10698012181
:10271000123009F019FD9CB12178062921D2DFE899
:1027200001F0200505160318801E80B2C01EE28845
:1027300080B20AB1A3681BB1824203D90C20C2E760
:102740001020C0E7042904D0A08850B901E0062079
:10275000B9E7012913D0022905D004291CD0052985
:102760002AD00720AFE709208DF800006088ADF877
:102770000800E088ADF80A00A068039023E00A2072
:102780008DF800006088ADF80800E088ADF80A0018
:10279000A0680A25039016E00B208DF800006088E1
:1027A000ADF80800A088ADF80A00E088ADF80C008C
:1027B000A0680B25049006E00C208DF800006078DE
:1027C0008DF808000C256A4629463046069BFFF71F
:1027D000B3FA78E700B587B00D228DF80020ADF888
:1027E000081000236A461946FFF7A6FA49E700B524
:1027F00087B071B102228DF800200A88ADF8082058
:102800004988ADF80A1000236A460621FFF794FABA
:1028100037E7102035E770B586B0064601200D4633
:10282000ADF808108DF80000014600236A463046D6
:10283000FFF782FA040008D12946304605F056FC1D
:102840000021304605F070FC204606B070BDF8B59A
:102850001C4615460E46069F10F0C8F92346FF1D7C
:10286000BCB231462A4600940FF0B3FDF8BD30B437
:102870001146DDE902423CB1032903D0002330BCFC
:1028800008F022BB0123FAE71A8030BC704770B50C
:102890000C460546FFF72FFB2146284605F035FC80
:1028A0002846BDE87040012105F03EBC4FF0E02213
:1028B0004FF400400021C2F88001BFF34F8FBFF3F7
:1028C0006F8F1748016001601649900208607047D9
:1028D000134900B500220A600A60124B4FF0607283
:1028E0001A60002808BF00BD0F4A104BDFF840C037
:1028F00001280CD002281CBFFFDF00BD03200860A8
:102900001A604FF4000000BFCCF8000000BD0220A8
:1029100008601A604FF04070F6E700B5FFDF00BDB9
:1029200000F5004008F501409C02002014F500402D
:1029300004F5014070B50B2000F0BDF9082000F04F
:10294000BAF900210B2000F0D4F90021082000F092
:10295000D0F9F44C01256560A5600020C4F8400161
:10296000C4F84401C4F848010B2000F0B5F9082070
:1029700000F0B2F90B2000F091F9256070BD10B5A0
:102980000B2000F098F9082000F095F9E5480121A6
:1029900041608160E4490A68002AFCD10021C0F846
:1029A0004011C0F84411C0F848110B2000F094F910
:1029B000BDE81040082000F08FB910B50B2000F0E2
:1029C0008BF9BDE81040082000F086B900B530B1A1
:1029D000012806D0022806D0FFDF002000BDD34822
:1029E00000BDD34800BDD248001D00BD70B5D1491F
:1029F0004FF000400860D04DC00BC5F80803CF4829
:102A000000240460C5F840410820C43500F053F9A3
:102A1000C5F83C41CA48047070BD08B5C14A0021E0
:102A200028B1012811D002281CD0FFDF08BD4FF4C7
:102A30008030C2F80803C2F84803BB483C3001604C
:102A4000C2F84011BDE80840D0E74FF40030C2F8AA
:102A50000803C2F84803B44840300160C2F844118A
:102A6000B3480CE04FF48020C2F80803C2F84803D2
:102A7000AD4844300160C2F84811AD48001D0068FF
:102A8000009008BD70B516460D460446022800D9D0
:102A9000FFDF0022A348012304F110018B4000EB6B
:102AA0008401C1F8405526B1C1F84021C0F8043373
:102AB00003E0C0F80833C1F84021C0F8443370BDCA
:102AC0002DE9F0411D46144630B1012833D00228CB
:102AD00038D0FFDFBDE8F081891E002221F07F4160
:102AE0001046FFF7CFFF012D23D00020944D924FC9
:102AF000012668703E61914900203C39086002203F
:102B0000091D08608D490420303908608B483D3428
:102B1000046008206C6000F0DFF83004C7F804039C
:102B2000082000F0BBF88349F007091F08602E70E9
:102B3000D0E70120DAE7012B02D00022012005E0D6
:102B40000122FBE7012B04D000220220BDE8F04166
:102B500098E70122F9E774480068704770B500F003
:102B6000D8F8704C0546D4F840010026012809D158
:102B7000D4F80803C00305D54FF48030C4F8080327
:102B8000C4F84061D4F8440101280CD1D4F80803FA
:102B9000800308D54FF40030C4F80803C4F844613A
:102BA000012012F06AFCD4F8480101280CD1D4F8B5
:102BB0000803400308D54FF48020C4F80803C4F884
:102BC0004861022012F059FC5E48056070BD70B586
:102BD00000F09FF85A4D0446287850B1FFF706FFE1
:102BE000687818B10020687012F047FC55480460FE
:102BF00070BD0320F8E74FF0E0214FF40010C1F85A
:102C000000027047152000F067B84B4901200861A9
:102C1000082000F061B848494FF47C10C1F808035F
:102C20000020024601EB8003C3F84025C3F8402191
:102C3000401CC0B20628F5D37047410A43F609523A
:102C40005143C0F3080010FB02F000F5807001EB67
:102C50005020704710B5430B48F2376463431B0C98
:102C60005C020C60384C03FB0400384B4CF2F72438
:102C700043435B0D13FB04F404EB402000F580702C
:102C80004012107008681844086010BD2C48406855
:102C9000704729490120C1F800027047002809DB6C
:102CA00000F01F02012191404009800000F1E02066
:102CB000C0F80011704700280DDB00F01F02012151
:102CC00091404009800000F1E020C0F88011BFF37E
:102CD0004F8FBFF36F8F7047002809DB00F01F0292
:102CE000012191404009800000F1E020C0F88012ED
:102CF00070474907090E002804DB00F1E02080F846
:102D00000014704700F00F0000F1E02080F8141D5F
:102D100070470C48001F00680A4A0D49121D1160D7
:102D20007047000000B0004004B500404081004002
:102D300044B1004008F5014000800040408500405B
:102D40003400002014050240F7C2FFFF6F0C0100A1
:102D5000010000010A4810B5046809490948083112
:102D6000086012F01EFC0648001D046010BD0649F4
:102D7000002008604FF0E0210220C1F88002704777
:102D80001005024001000001FC1F004010B50D209D
:102D900000F077F8C4B26FF0040000F072F8C0B22F
:102DA000844200D0FFDF3E490120086010BD70B5AD
:102DB0000D2000F048F83B4C0020C4F8000101252C
:102DC000C4F804530D2000F04FF825604FF0E021C7
:102DD0006014C1F8000170BD10B50D2000F033F88B
:102DE0003048012141600021C0F80011BDE81040C9
:102DF0000D2000F039B82C4810B504682A492B483A
:102E0000083108602749D1F80001012804D0FFDF0C
:102E10002548001D046010BD2148001D00680022E7
:102E2000C0B2C1F8002113F009F8F1E710B51D4850
:102E3000D0F800110029FBD0FFF7DDFFBDE81040FE
:102E40000D2000F011B800280DDB00F01F02012159
:102E500091404009800000F1E020C0F88011BFF3EC
:102E60004F8FBFF36F8F7047002809DB00F01F0200
:102E7000012191404009800000F1E020C0F880125B
:102E80007047002804DB00F1E02090F8000405E022
:102E900000F00F0000F1E02090F8140D4009704799
:102EA00004D5004000D000401005024001000001A0
:102EB0004FF0E0214FF00070C1F8800101F5C071C2
:102EC000BFF34F8FBFF36F8FC1F80001384B8022E3
:102ED00083F8002441F8800C704700B502460420B6
:102EE000344903E001EBC0031B792BB1401EC0B293
:102EF000F8D2FFDFFF2000BD41F8302001EBC00118
:102F000000224A718A7101220A7100BD294A0021FA
:102F100002EBC0000171704710B50446042800D3CD
:102F2000FFDF244800EBC4042079012800D0FFDF34
:102F30006079A179401CC0B2814200D060714FF02D
:102F4000E0214FF00070C1F8000210BD2DE9F04102
:102F500019480568184919480831086014480426BA
:102F600090F80004134F4009154C042818D0FFDFD7
:102F700016E0217807EBC1000279012A08D14279D5
:102F800083799A4204D04279827157F831008047A0
:102F90002078401CC0B22070042801D3002020708B
:102FA000761EF6B2E5D20448001D0560BDE8F0814A
:102FB00019E000E0D40500201005024001000001E6
:102FC000500000200548064A0168914201D10021C5
:102FD000016004490120086070470000540000208F
:102FE000BEBAFECA40E5014070B50C46054609F080
:102FF00089FB21462846BDE870400AF06EBC704748
:103000002CFFFFFFDBE5B15100600200AE00FFFFC7
:103010008C00000068915B008308DF2FACFED6397E
:1030200029D64B9DC15EF1868A16B47C30B5F84D29
:103030000446062CA9780ED2DFE804F0030E0E0E2B
:103040000509FFDF08E0022906D0FFDF04E00329BD
:1030500002D0FFDF00E0FFDFAC7030BD30B50446CA
:103060001038EB4D07280CD2DFE800F0040C060CFA
:103070000C0C0C00FFDF05E0287E112802D0FFDFDA
:1030800000E0FFDF2C7630BD2DE9F04111F092FB1E
:10309000044612F063FD201AC5B206200FF01CFC96
:1030A000044606200FF020FC211AD94C207E12285D
:1030B00018D000200F1807200FF00EFC064607203E
:1030C0000FF012FC301A3918207E13280CD0002083
:1030D0000144A078042809D000200844281AC0B26E
:1030E000BDE8F0810120E5E70120F1E70120F4E7E8
:1030F000C74810B590F825004108C54800F12600E2
:1031000005D00DF006FBBDE8104006F003B80DF049
:10311000E1FAF8E730B50446A1F120000D460A288F
:103120004AD2DFE800F005070C1C2328353A3F445B
:10313000FFDF42E0207820283FD1FFDF3DE0B448A8
:103140008178052939D0007E122836D020782428AD
:1031500033D0252831D023282FD0FFDF2DE0207851
:1031600022282AD0232828D8FFDF26E0207822280A
:1031700023D0FFDF21E0207822281ED024281CD075
:1031800026281AD0272818D0292816D0FFDF14E0C7
:103190002078252811D0FFDF0FE0207825280CD0DB
:1031A000FFDF0AE02078252807D0FFDF05E0207840
:1031B000282802D0FFDF00E0FFDF257030BD1FB5FB
:1031C00004466A46002001F035FEB4B1BDF8022085
:1031D0004FF6FF700621824201D1ADF80210BDF812
:1031E0000420824201D1ADF80410BDF808108142DC
:1031F00003D14FF44860ADF8080068460EF0EBF8D4
:1032000005F088FF04B010BD70B514460D460646A3
:10321000FEF759F858B90DB1A54201D90C2070BD7F
:10322000002408E056F82400FEF74DF808B11020FD
:1032300070BD641CE4B2AC42F4D3002070BD2DE933
:10324000F04105461F4690460E4600240068FEF7F2
:1032500087F830B9A98828680844401EFEF780F82E
:1032600008B110203CE728680028A88802D0B8429E
:1032700002D850E00028F5D0092031E72968085D20
:10328000B8B1671CCA5D152A2ED03CDC152A3AD28B
:10329000DFE802F03912222228282A2A313139396E
:1032A00039393939393939392200085D30BB641C64
:1032B000A4B2A242F9D833E00228DDD1A01C085CF8
:1032C00088F80000072801D2400701D40A2007E748
:1032D000307840F0010015E0C143C90707E001283C
:1032E00007D010E00620FBE60107A1F1805100297C
:1032F000F5D01846F4E63078810701D50B20EFE6CB
:1033000040F0020030702868005D384484B2A8881C
:10331000A04202D2B0E74FF4485382B2A242ADD8E5
:103320000020DDE610B5027843F2022354080122A2
:10333000022C12D003DC3CB1012C16D106E0032C88
:1033400010D07F2C11D112E0002011E080790324ED
:10335000B4EB901F09D10A700BE08079B2EB901F9B
:1033600003D1F8E780798009F5D0184610BDFF2019
:103370000870002010BD08B500208DF8000024481A
:1033800090F82E1049B190F82F0002280ED0032893
:103390000ED0FFDF9DF8000008BD1D4869462530AE
:1033A00001F097FD0028F5D0FFDFF3E7032000E0F0
:1033B00001208DF80000EDE738B50C46054669465A
:1033C00001F087FD00280DD19DF80010207861F3F1
:1033D0004700207055F8010FC4F80100A888A4F830
:1033E0000500002038BD38B51378A8B1022813D0E5
:1033F000FF281AD007A46D46246800944C7905EB89
:103400009414247864F347031370032809D00FE061
:10341000E80100200302FF0123F0FE0313700228DD
:10342000F3D1D8B240F0010005E043F0FE00107087
:10343000107820F0010010700868C2F80100888838
:10344000A2F8050038BD02210FF09EBA38B50C462F
:103450000978222901D2082038BDADF800008DF886
:10346000022068460DF097F905F054FE050003D1DF
:1034700021212046FFF74EFE284638BD1CB500200E
:103480008DF80000CDF80100ADF80500FB4890F87C
:103490002E00022801D0012000E000208DF8070056
:1034A00068460DF0DAFA002800D0FFDF1CBD0022CC
:1034B0000A80437892B263F3451222F040020A80F8
:1034C00000780C282BD2DFE800F02A06090E11162E
:1034D000191C1F220C2742F0110009E042F01D00C8
:1034E00008800020704742F0110012E042F0100006
:1034F00040F00200F4E742F01000F1E742F0010072
:10350000EEE742F0010004E042F00200E8E742F09A
:10351000020040F00400E3E742F00400E0E7072087
:1035200070472DE9FF478AB00025BDF82C60824620
:103530001C4691468DF81C50700703D56068FDF756
:10354000C2FE68B9CD4F4FF0010897F82E0058B170
:1035500097F82F00022807D16068FDF701FF18B126
:1035600010200EB0BDE8F087300702D5A089802872
:103570003ED8700705D4B9F1000F02D097F82400A7
:10358000A0B3E07DC0F300108DF81B00627D072022
:10359000032162B3012A2DD0022AE2D0042AE0D10D
:1035A0008DF81710F00628D4A27D07202AB3012A2F
:1035B00023D0022A24D0042AD3D18DF8191000BFB9
:1035C0008DF81590606810B307A9FFF7ABFE0028CF
:1035D000C7D19DF81C00FF2816D0606850F8011F65
:1035E000CDF80F108088ADF8130014E000E001E082
:1035F0000720B6E78DF81780D4E78DF81980DFE74C
:1036000002208DF81900DBE743F20220A9E7CDF88C
:103610000F50ADF81350E07B40B9207C30B9607C8E
:1036200020B9A07C10B9E07CC00601D0062098E744
:103630008DF800A0BDF82C00ADF80200A068019044
:10364000A068029004F10F0001F037FC8DF80C0027
:10365000FFF791FE8DF80D009DF81C008DF80E000F
:103660008DF816508DF81850E07D08A900F00F0075
:103670008DF81A0068460DF0E9FF05F04BFD70E784
:10368000F0B58FB000258DF830508DF814508DF8BE
:10369000345006468DF828500195029503950495FF
:1036A00019B10FC901AC84E80F00744CA07805284B
:1036B00001D004280CD101986168884200D120B95A
:1036C0000398E168884203D110B108200FB0F0BD23
:1036D000207DC00601D51F2700E0FF273B460DAA2D
:1036E00005A903A8FFF7ABFD0028EFD1A08AC10709
:1036F00002D0C00600D4EE273B460AAA0CA901A8B6
:10370000FFF79DFD0028E1D19DF81400C00701D00E
:103710000A20DBE7A08A410708D4A17D31B19DF8DA
:103720002810890702D043F20120CFE79DF8281026
:10373000C90709D0400707D4208818B144F2506166
:10374000884201D90720C1E78DF818508DF819601B
:10375000BDF80800ADF81A000198079006A80DF012
:103760008FFF05F0D7FC0028B0D18DF820508DF8E0
:103770002160BDF81000ADF822000398099008A858
:103780000DF09DFF05F0C6FC00289FD101AD241D62
:1037900095E80F0084E80F00002097E770B586B029
:1037A0000D46040005D0FDF7DBFD20B1102006B06A
:1037B00070BD0820FBE72078C107A98802D0FF2947
:1037C00002D303E01F2901D20920F0E7800763D468
:1037D000FFF75AFC38B12178C1F3C100012804D0A9
:1037E000032802D005E01320E1E7244890F82400E4
:1037F000C8B1C8074FF001064FF0000502D08DF8A0
:103800000F6001E08DF80F50FFF7B5FD8DF8000057
:1038100020786946C0F3C1008DF8010060788DF80A
:103820000250C20801D00720C1E730B3C20701D05F
:103830008DF80260820705D59DF8022042F0020251
:103840008DF80220400705D59DF8020040F00400E5
:103850008DF80200002022780B18C2F38002DA7083
:1038600001EB40026388D380401CA388C0B253811F
:103870000228F0D3207A78B905E001E0E8010020C1
:103880008DF80260E6E7607A30B9A07A20B9E07A74
:1038900010B9207BC00601D0062088E704F108009B
:1038A00001F00BFB8DF80E0068460DF09FFA05F055
:1038B00031FC002889D18DF810608DF81150E08816
:1038C000ADF81200ADF8145004A80DF0E2FA05F0BE
:1038D00021FC002888D12078C00701D0152000E005
:1038E0001320FFF7BBFB002061E72DE9FF47022013
:1038F000FB4E8DF804000027708EADF80600B84628
:1039000043F202094CE001A80EF0A5FF050006D025
:10391000708EA8B3A6F83280ADF806803EE0039C16
:10392000A07F01072DD504F124000090A28EBDF8E0
:103930000800214604F1360301F057FC050005D0CC
:103940004D452AD0112D3CD0FFDF3AE0A07F20F07A
:103950000801E07F420862F3C711A177810861F393
:103960000000E07794F8210000F01F0084F82000A8
:103970002078282826D129212046FFF7CBFB21E0FB
:1039800014E040070AD5BDF8080004F10E0101F06B
:10399000AAFA05000DD04D4510D100257F1CFFB2BD
:1039A00002200EF099FF401CB842ACD8052D11D072
:1039B00008E0A07F20F00400A07703E0112D00D0E4
:1039C000FFDF0025BDF806007086052D04D02846CF
:1039D00004B0C7E5A6F832800020F9E770B50646C6
:1039E000FFF731FD054605F073FD040000D1FFDF50
:1039F0006680207820F00F00801C20F0F00020303E
:103A000020700320207295F83E006072BDE870407F
:103A100005F061BD2DE9F04786B0040000D1FFDF5D
:103A20002078AF4D20F00F00801C20F0F0007030A7
:103A3000207060680178491F1B2933D2DFE801F04C
:103A4000FE32323255FD320EFDFD42FC323232780A
:103A5000FCFCFBFA3232FCFCF9F8FC00C68830466C
:103A6000FFF7F1FC0546304607F02CF9E0B160683D
:103A7000007A85F83E0021212846FFF74BFB3046AF
:103A8000FEF753FB304603F053FE3146012012F09F
:103A900095FCA87F20F01000A877FFF726FF0028EC
:103AA00000D0FFDF06B05DE5207820F0F000203088
:103AB00020700320207266806068007A607205F0D2
:103AC0000AFDD8E7C5882846FFF7BDFC00B9FFDF2F
:103AD00060680079012800D0FFDF6068017A06B0D5
:103AE0002846BDE8F04707F0CCBCC6883046FFF753
:103AF000AAFC050000D1FFDF05F0EDFC606831464F
:103B00000089288160684089688160688089A8810F
:103B1000012012F053FC0020A875A87F00F00300DC
:103B20000228BFD1FFF7E1FE0028BBD0FFDFB9E7D5
:103B300000790228B6D000B1FFDF05F0CCFC666842
:103B4000B6F806A0307A361D012806D0687E814678
:103B500005F04CFA070003D101E0E878F7E7FFDF52
:103B60000022022150460EF006FF040000D1FFDFC4
:103B700022212046FFF7CEFA3079012800D002201A
:103B8000A17F804668F30101A177308B2081708B83
:103B90006081B08BA08184F822908DF80880B8688D
:103BA0000090F86801906A46032150460EF0E3FE4B
:103BB00000B9FFDFB888ADF81000B8788DF81200B2
:103BC00004AA052150460EF0D6FE00B9FFDFB888E2
:103BD000ADF80C00F8788DF80E0003AA04215046C9
:103BE0000EF0C9FE00B9FFDF062106F1120001F058
:103BF00098F940B37079800700D5FFDF7179E07DD7
:103C000061F34700E075D6F80600A0617089A083D3
:103C1000062106F10C0001F084F9F0B195F82500B9
:103C20004108607861F347006070D5F8260006E02F
:103C30003EE036E06DE055E04AE02CE040E0C4F8BC
:103C40000200688D12E0E07D20F0FE00801CE0752F
:103C5000D6F81200A061F08AD9E7607820F0FE0063
:103C6000801C6070F068C4F80200308AE080B8F10F
:103C7000010F04D0B8F1020F05D0FFDF12E70320D7
:103C8000FFF7D4F90EE7287E122800D0FFDF1120BD
:103C9000FFF7E4F906E706B02046BDE8F04701F07B
:103CA0002DBD05F018FC15F8300F40F0020005E0BE
:103CB00005F011FC15F8300F40F004002870F1E613
:103CC000287E132809D01528D8D11620FFF7C6F969
:103CD00006B0BDE8F04705F0FEBB1420F6E7000093
:103CE000E8010020A978052909D00429C6D105F0EA
:103CF000F2FB022006B0BDE8F047FFF797B9007964
:103D00000028BBD0E87801F0BFF805F0E4FB032001
:103D1000F0E7287E122802D1687E01F0B5F8112064
:103D2000D4E72DE9F047054600784FF00008000978
:103D3000DFF8C0A891460C464646012875D00228F7
:103D400074D007280AD00A2871D0FFDFA9F80060D4
:103D500014B1A4F800806680002003E4696801279C
:103D600004F108000A784FF0020C4FF6FF73172A8F
:103D70007ED00EDC142A32D006DC052A68D0092A4F
:103D800010D0102A75D120E0152A73D0162AF9D147
:103D9000F8E0183A082A6CD2DFE802F0F36B6B0AFD
:103DA000CAF2DFF1C8884FF01208102621468DE1D3
:103DB0004FF01C080A26BCB38888A0806868807908
:103DC00020726868C0796072C0E74FF01B08142643
:103DD00054B30320207268688088A080B6E70A790F
:103DE0003C2AB3D00D1D4FF010082C26E4B1698891
:103DF000A180298B6182298B2182698BA182A98B69
:103E0000E1826B790246A91D1846FFF7ECFA297981
:103E1000002001290CD084F80FC0FF212176E06139
:103E200020626062A06291E70FE02EE151E18CE137
:103E3000E77320760AF1040090E80E00DAF810002B
:103E4000C4E90930C4E9071280E7A9F8006083E7F4
:103E50002C264FF01D08002CF7D00546A380887B48
:103E60002A880F1D60F300022A80887B400802E048
:103E70009DE007E1BEE060F341022A80887B800874
:103E800060F382022A80887BB91CC00860F3C302F9
:103E90002A80B87A0011401C60F3041202F07F00FF
:103EA00028807878AA1CFFF79EFA387D05F1090270
:103EB00007F11501FFF797FA387B01F041F82874F4
:103EC000787B01F03DF86874F87EA874787AE8741D
:103ED000387F2875B87B6875388AE882DAF81C0064
:103EE000A861B87A524697F808A0C0F34111012999
:103EF00004D0108C504503D2824609E0FFDF10E069
:103F0000022903D0288820F0600009E0504504D140
:103F1000288820F06000403002E0288840F06000EF
:103F20002880A4F824A0524607F11D01A86996E054
:103F300011264FF02008002C87D0A380686804F178
:103F40000A02007920726868007B607269688B1DC4
:103F500048791946FFF747FAF8E60A264FF0210894
:103F6000002CE9D08888A080686880792072686811
:103F7000C07960729AF8301021F004019FE065E08A
:103F80004CE06FE00B264FF02208002CD4D0C888FC
:103F9000A0806868007920726868007A00F0D0FF1D
:103FA00060726868407A00F0CBFFA072CEE61C26F3
:103FB0004FF02608002CBFD0A3806868407960725B
:103FC0006868007AA0720AF1040090E80E00DAF83E
:103FD0001000C4E90530C4E90312686800793C2880
:103FE00003D0432803D0FFDFB0E62772AEE684F8A3
:103FF00008C0ABE610264FF02408002C9CD088881F
:10400000A0806868807920816868807A60816868AB
:104010000089A08168688089E08197E610264FF0CA
:104020002308002C88D08888A0806868C0882081F8
:1040300068680089608168684089A08168688089B3
:10404000E0819AF8301021F0020138E030264FF07C
:104050002508002C85D0A38069682822496821F0B2
:10406000D9FA73E614264FF01B08002C8ED0A380DB
:10407000686800790128BAD02772DAE90710C4E924
:10408000031063E64A46214660E0287A012803D0FF
:10409000022817D0FFDF59E610264FF01F08002C2A
:1040A00089D06888A080A8892081E8896081288AD1
:1040B000A081688AE0819AF8301021F001018AF825
:1040C000301043E64FF012081026688800F016FF03
:1040D0003CE6287AC8B3012838D0022836D0032815
:1040E00001D0FFDF32E609264FF01108002C85D001
:1040F0006F883846FFF7A7F990F822A0A780687A62
:104100002072042138460EF051FC052138460EF08D
:104110004DFC002138460EF049FC012138460EF0D6
:1041200045FC032138460EF041FC022138460EF0D2
:104130003DFC062138460EF039FC072138460EF0CA
:1041400035FC504600F0A0FE00E6FFE72846BDE83B
:10415000F04701F05DBC70B5012803D0052800D000
:10416000FFDF70BD8DB22846FFF76DF9040000D166
:10417000FFDF20782128F4D005F0AAF980B101787A
:1041800021F00F01891C21F0F00110310170022192
:10419000017245800020A075BDE8704005F09BB914
:1041A00021462846BDE870401322FFF74FB92DE99C
:1041B000F04116460C00804600D1FFDF307820F039
:1041C0000F00801C20F0F0001030307020780128A3
:1041D00004D0022818D0FFDFBDE8F0814046FFF789
:1041E00032F9050000D1FFDF0320A87505F073F94F
:1041F00094E80F00083686E80F00FE4810F8301FDC
:1042000041F001010170E7E74046FFF71CF90500A6
:1042100000D1FFDFA1884FF6FF700027814202D155
:10422000E288824203D0814201D1E08840B105F0AA
:1042300052F994E80F00083686E80F00AF75CBE717
:10424000A87D0128C8D178230022414612F00CF83D
:104250000220A875C0E738B505460C460846FDF7AC
:1042600032F818BB203D062D4AD2DFE805F0031BCB
:10427000373C42300021052012F076F808B11120B9
:1042800038BDA01C0DF0FAF804F044FF050038D149
:10429000002208231146052011F0E6FF052830D042
:1042A000FFDF2EE06068FDF752F808B1102038BD3E
:1042B000618820886A460DF099FB04F02BFF050009
:1042C0001FD16068E8B1BDF80010018019E0A07846
:1042D00000F0010120880DF0BAFB0EE0206801F02B
:1042E00043FE05460DE0207800F001000CF0DBF9FC
:1042F00003E0618820880DF0F4FA04F00BFFF0E78A
:104300000725284638BD70B505460C460846FDF71A
:1043100000F808B1102070BD202D07D0212D0DD040
:10432000222D0BD0252D09D0072070BD2088A11C7F
:104330000CF08EFABDE8704004F0ECBE062070BDB3
:10434000AC482530704708B53421AA4821F003FA5B
:104350000120FEF76BFE1120FEF780FEA54968469E
:10436000263105F04BF8A3489DF8002010F8251FD2
:1043700062F3470121F001010170002141724FF405
:104380006171A0F8071002218172FEF7B1FE00B141
:10439000FFDFFDF75DF801F07CF908BD10B50C46B4
:1043A0004021204621F0B5F9A07F20F00300A0773E
:1043B000202020700020A07584F8230010BD7047D5
:1043C0002DE9FC410746FCF77EFF10B11020BDE847
:1043D000FC81884E06F12501D6F825000090B6F83C
:1043E0002950ADF8045096F82B408DF80640384619
:1043F000FEF7E2FF0028EAD1FEF77AFE0028E6D0B9
:10440000009946F8251FB580B471E0E710B5044661
:10441000FCF77FFF08B1102010BD76487549224691
:1044200090F8250026314008FEF7DDFF002010BD82
:104430003EB504460D460846FCF76BFF08B1102058
:104440003EBD14B143F204003EBD6A4880780528A1
:1044500003D0042801D008203EBD694602A80AF016
:104460009CFA2A4669469DF80800FEF7BCFF00202A
:104470003EBDFEB50D4604004FF0000711D00822E6
:10448000FEF7C2FE002811D1002608E054F82600ED
:104490006946FEF747FF002808D1761CF6B2AE4207
:1044A000F4D30CF047F810B143F20320FEBD514E97
:1044B00086F824700CB300271BE000BF54F82700D7
:1044C00002A9FEF72FFF00B1FFDF9DF808008DF86D
:1044D000000054F8270050F8011FCDF80110808823
:1044E000ADF8050068460CF04AF800B1FFDF7F1C0C
:1044F000FFB2AF42E2D386F824500020FEBD2DE982
:10450000F0478AB01546894604001ED00F4608229F
:104510002946FEF779FE002811D1002613E000BFDE
:1045200054F826006946103000F0D3FC002806D16C
:104530003FB157F82600FCF7C6FE10B110200AB0B4
:104540000BE4761CF6B2AE42EAD30026A5F10108D0
:104550001CE000BF06F1010A0AF0FF0712E000BFED
:1045600054F82600017C4A0854F827100B7CB2EB63
:10457000530F05D106221130113121F01FF858B127
:104580007F1CFFB2AF42EBD30AF0FF064645E1DBEA
:104590004E4624B1012003E043F20520CFE700207E
:1045A0000CF012F810B90CF01BF810B143F2042013
:1045B000C5E774B300270DF1170828E054F8270069
:1045C0006946103000F085FC00B1FFDF54F8270089
:1045D000102250F8111FCDF801108088ADF80500A9
:1045E00054F827100DF1070021F014F8AEB156F879
:1045F000271001E0E80100201022404621F00AF8CF
:1046000068460BF0A1FF00B1FFDF7F1CFFB2AF4295
:10461000D4D3FEF733FF002091E7404601F098FC29
:10462000EEE730B585B00446FCF74DFE18B960687A
:10463000FCF796FE10B1102005B030BD60884AF23C
:10464000B811884206D82078F84D28B1012806D044
:10465000022804D00720EFE7FEF74AFD18E0607853
:10466000022804D0032802D043F20220E4E785F8B0
:104670002F00C1B200200090ADF8040002292CD018
:10468000032927D0FFDF68460CF043F804F042FD11
:104690000028D1D1606801F04EFC207858B101208B
:1046A0008DF800000DF1010001F052FC68460DF09C
:1046B00032FA00B1FFDF207885F82E00FEF7DEFE2B
:1046C000608860B1A88580B20BF076FF00B1FFDF93
:1046D0000020B1E78DF80500D5E74020FAE74FF458
:1046E0006170EFE710B50446FCF713FE20B960686F
:1046F00038B1FCF72CFE08B1102010BD606801F045
:1047000027FCCA4830F82C1F6180C178617080781E
:104710002070002010BD2DE9F84314468946064656
:10472000FCF7F7FDA0B94846FCF71AFE80B9204611
:10473000FCF716FE60B9BD4DA878012800D13CB148
:104740003178FF2906D049B143F20400BDE8F8836F
:104750001020FBE7012801D00420F7E7CCB305289F
:1047600011D004280FD069462046FEF7A0FE00288D
:10477000ECD1217D49B1012909D0022909D00329B1
:1047800009D00720E2E70820E0E7024604E0012222
:1047900002E0022200E00322804623461746002062
:1047A0000099FEF7BEFE0028D0D1A0892880A07B0A
:1047B000E875BDF80000A882AF75BDF800100907C4
:1047C00001D5A18931B1A1892980C00704D0032076
:1047D00003E006E08021F7E70220FEF727FC86F8D9
:1047E00000804946BDE8F8430020FEF749BF7CB58C
:1047F0008E4C05460E46A078022803D0032801D02F
:1048000008207CBD15B143F204007CBD07200EF0EA
:104810006BF810B9A078032806D0FEF735FC28B154
:10482000A078032804D009E012207CBD13207CBDB1
:10483000304600F00CFB0028F9D1E670FEF79BFD36
:1048400009F0E8FF01208DF800008DF801008DF8D7
:1048500002502088ADF80400E07D8DF8060068461F
:104860000DF002F804F056FC0028E0D1A0780328EF
:1048700004D00420FEF7DAFB00207CBDE07800F0D5
:10488000F6FA0520F6E71CB510B143F204001CBD92
:10489000664CA078042803D0052801D008201CBD50
:1048A00000208DF8000001218DF801108DF8020024
:1048B00068460CF0D9FF04F02DFC0028EFD1A07859
:1048C000052805D05FF00200FEF7B0FB00201CBDFC
:1048D000E07800F0D9FA0320F6E72DE9FC418046A4
:1048E0000E4603250846FCF73BFD002866D14046EE
:1048F000FEF7A9FD040004D02078222804D2082065
:1049000065E543F2020062E5A07F00F003073EB1D7
:10491000012F0CD000203146FEF751FC0500EFD1ED
:10492000012F06D0022F1AD0FFDF28464FE50120C5
:10493000F1E7A07D3146022801D011B107E0112036
:1049400045E56846FCF791FE0028D9D16946404606
:1049500006F05AFD0500E8D10120A075E5E7A07D2D
:10496000032804D1314890F83000C00701D02EB39D
:104970000EE026B1A07F40071ED4002100E00121F7
:10498000404606F061FD0500CFD1A075002ECCD0C9
:104990003146404600F0A7FA05461128C5D1A07F50
:1049A0004107C2D4316844F80E1F7168616040F05D
:1049B000040020740025B8E71125B6E7102006E5AD
:1049C00070B50C460546FEF73EFD010005D02246B7
:1049D0002846BDE87040FEF739BD43F2020070BDC5
:1049E00010B5012807D1114B9B78012B00D011B1D4
:1049F00043F2040010BD0BF011FEBDE8104004F0BE
:104A000089BB012300F04ABA00231A46194600F078
:104A100045BA70B506460C460846FCF754FC18B972
:104A20002068FCF776FC18B1102070BDE80100206A
:104A3000F94D2A7E112A04D0132A00D33EB1082052
:104A4000F3E721463046FEF7A9FE60B1EDE7092005
:104A5000132A0DD0142A0BD0A188FF29E5D31520E5
:104A6000FEF7FCFA0020D4E90012C5E90712DCE7E2
:104A7000A1881F29D9D31320F2E71CB5E648007E90
:104A8000132801D208201CBD00208DF800006846C4
:104A90000CF0FFF904F03EFB0028F4D11120FEF7E2
:104AA000DDFA00201CBD2DE9F04FDFF86CA3814634
:104AB00091B09AF818009B4615460C46132803D36C
:104AC000FFF7DBFF00281FD12046FCF7FCFBE8BB0B
:104AD0002846FCF7F8FBC8BB20784FF00107C00759
:104AE0004FF0000102D08DF83A7001E08DF83A10D5
:104AF00020788846C0F3C1008DF8000060788DF8FA
:104B00000910C10803D0072011B0BDE8F08F70B3C1
:104B1000C10701D08DF80970810705D59DF80910EE
:104B200041F002018DF80910400705D59DF80900F4
:104B300040F004008DF8090000206E4606EB4001AD
:104B400062884A81A2880A82401C00E00DE0C0B25F
:104B50000328F3D32078C0F3C100012825D003280F
:104B600023D04846FCF7AFFB28B11020CCE7FFE785
:104B70008DF80970E0E799F80000400808D0012896
:104B800009D0022807D0032805D043F20220BBE752
:104B90008DF8028001E08DF80270484650F8011F40
:104BA000CDF803108088ADF80700FEF7E4FB8DF820
:104BB00001000020424606EB40012B88CB826B8827
:104BC0008B83AB884B84EB880B85401CCA85C0B2B5
:104BD0008A860328EFD3E088ADF83C0068460CF0E5
:104BE00094FA00288FD19AF818005546112801D060
:104BF000082089E706200DF077FE38B12078C0F351
:104C0000C100012804D0032802D006E012207BE76F
:104C100095F8240000283FF476AFFEF735FA022815
:104C200001D2132070E7584600F011F900289DD1F9
:104C300085F819B068460CF0A8FB04F06BFA040084
:104C400094D1687E00F013F91220FEF707FA20468F
:104C50005AE770B5704D287E122801D00820E4E68E
:104C60000CF096FB04F056FA040005D1687E00F0C3
:104C70000BF91120FEF7F2F92046D6E670B506468C
:104C800015460C460846FCF744FB18B92846FCF7C5
:104C900040FB08B11020C8E62A46214630460CF0F9
:104CA00085FE04F037FA0028F5D121787F29F2D16A
:104CB0000520BAE67CB505460C460846FCF703FB22
:104CC00008B110207CBD2846FEF7BDFB20B100785E
:104CD000222804D208207CBD43F202007CBD4E484D
:104CE00090F83000400701D511207CBD2078C00825
:104CF00002D16078C00801D007207CBDADF800501B
:104D000020788DF8020060788DF803000220ADF85D
:104D1000040068460BF09EFF04F0FCF97CBD70B502
:104D200086B014460D460646FEF78DFB28B1007886
:104D3000222805D2082006B077E643F20200FAE7FF
:104D40002846FCF70DFB20B944B12046FCF7FFFADA
:104D500008B11020EFE700202060A0802E4890F8D6
:104D60003000800701D51120E5E703A930460BF09C
:104D7000C2FD10B104F0CEF9DDE7ADF80060BDF87A
:104D80001400ADF80200BDF81600ADF80400BDF83F
:104D90001000BDF81210ADF80600ADF808107DB196
:104DA000298809B1ADF80610698809B1ADF802107B
:104DB000A98809B1ADF80810E98809B1ADF8041067
:104DC000DCB1BDF80610814201D9081A2080BDF877
:104DD0000210BDF81400814201D9081A6080BDF8A4
:104DE0000800BDF80410BDF816200144BDF81200FB
:104DF0001044814201D9081AA08068460BF02CFEAD
:104E0000B8E71CB505490968CDE9001068460CF003
:104E10007EF904F07FF91CBDE8010020FC5A020075
:104E20001CB500200090019068460CF070F904F069
:104E300071F9F0E710800888508048889080C88811
:104E400010818888D080002050819081704710B5F3
:104E5000044604F0CBF830B1407830B1204604F07D
:104E6000DEFB002010BD052010BD122010BD10B5C6
:104E700004F0BCF8040000D1FFDF607800B9FFDF68
:104E80006078401E607010BD10B504F0AFF80400EB
:104E900000D1FFDF6078401C607010BD1CB5ADF81C
:104EA00000008DF802308DF803108DF8042068465C
:104EB0000CF03FFD04F02EF9ADE70CB528A2D2E9C5
:104EC0000012CDE900120079694601EB501000781C
:104ED0000CBD0278520804D0012A02D043F202200D
:104EE0007047FEF71FBA1FB56A46FFF7A3FF684673
:104EF0000CF081FA04F00EF904B010BD70B50C008E
:104F000006460DD0FEF79FFA050000D1FFDFA68010
:104F100028892081288960816889A081A889E08109
:104F200083E510B500231A4603E0845C2343521C3A
:104F3000D2B28A42F9D30BB1002010BD012010BDBE
:104F400000B540B1012805D0022803D0032804D0C1
:104F5000FFDF002000BDFF2000BD042000BD0000D9
:104F6000070605040302010010B50446FCF7ABF97F
:104F700008B1102010BD2078C0F30210042807D813
:104F80006078072804D3A178102901D8814201D282
:104F9000072010BDE078410706D421794A0703D4E1
:104FA000000701D4080701D5062010BD002010BD60
:104FB00010B513785C08837F64F3C7138377137885
:104FC0009C08C37F64F30003C3771078C309487853
:104FD00063F34100487013781C090B7864F347139E
:104FE0000B701378DB0863F3000048705078487149
:104FF00010BD10B5C4780B7864F300030B70C4784F
:10500000640864F341030B70C478A40864F382035A
:105010000B70C478E40864F3C3030B700379117850
:1050200063F30001117003795B0863F341011170B0
:1050300003799B0863F3820111700079C00860F363
:10504000C301117010BD70B514460D46064604F03C
:105050003FFA80B10178182221F00F01891C21F05C
:10506000F001A03100F8081B214620F018FBBDE834
:10507000704004F030BA29463046BDE87040132233
:10508000FEF7E4B92DE9F047064608A8894690E8FE
:1050900030041F4690461421284620F05CFB002176
:1050A000CAF80010B8F1000F03D0B9F1000F03D116
:1050B00014E03878C00711D02068FCF72AF9C0BB8B
:1050C000B8F1000F07D12068123028602068143032
:1050D00068602068A8602168CAF8001038788007E6
:1050E00024D56068FCF733F918BBB9F1000F21D063
:1050F000FFF726F90168C6F868118188A6F86C11D7
:10510000807986F86E0101F0F8FCF94FEF60626873
:1051100062B196F8680106F2691140081032FEF794
:1051200062F910223946606820F074FA0020BDE868
:10513000F08706E0606820B1E8606068C6F8640146
:10514000F4E71020F3E730B5054608780C4620F068
:105150000F00401C20F0F001103121700020607021
:1051600095F8230030B104280FD0052811D0062867
:1051700014D0FFDF20780121B1EB101F04D295F885
:10518000200000F01F00607030BD21F0F0002030E2
:1051900002E021F0F00030302070EBE721F0F00069
:1051A0004030F9E7F0B591B0022715460C460646A7
:1051B0003A46ADF80870092103AB04F0FAFF0490F9
:1051C000002810D004208DF804008DF80170E03420
:1051D000099605948DF818500AA968460FF0C4F88E
:1051E00000B1FFDF012011B0F0BD10B588B00C4652
:1051F0000A99ADF80000C3B11868CDF802005868EC
:10520000CDF80600ADF80A20102203A820F002FA1B
:1052100068460CF060F903F07DFF002803D1A17F00
:1052200041F01001A17708B010BD0020CDF80200B8
:10523000E6E72DE9F84F0646808A0D4680B28246A1
:10524000FEF701F904463078DFF8A48200274FF01A
:105250000209A8F120080F2870D2DFE800F06FF2F1
:105260003708387D8CC8F1F0EFF35FF3F300A07FCF
:1052700000F00300022809D05FF0000080F0010177
:1052800050460DF081FB050003D101E00120F5E758
:10529000FFDF98F85C10C90702D0D8F860000BE077
:1052A000032105F11D0010F0AAFDD5F81D0091495C
:1052B000B0FBF1F201FB1200C5F81D0070686867D1
:1052C000B068A8672078252800D0FFDFCAE0A07F5B
:1052D00000F00300022809D05FF0000080F0010117
:1052E00050460DF051FB060003D101E00120F5E727
:1052F000FFDF3078810702D52178252904D040F0DE
:1053000001003070BDE8F88F85F80090307F28717B
:1053100006F11D002D36C5E90206F3E7A07F00F077
:105320000300022808D0002080F0010150460DF053
:105330002BFB040004D102E00120F5E7A7E1FFDF29
:105340002078C10604D5072028703D346C60D9E769
:1053500040F008002070D5E7E07F000700D5FFDFB0
:10536000307CB28800F0010301B05046BDE8F04F38
:10537000092105F0A9BD04B9FFDF716821B1102230
:1053800004F1240020F046F928212046FDF7C2FE52
:10539000A07F00F0030002280ED104F124000023B6
:1053A00000901A4621465046FFF71FFF112807D0EC
:1053B00029212046FDF7AEFE307A84F82000A1E7CF
:1053C000A07F000700D5FFDF14F81E0F40F0080093
:1053D0002070E782A761E761C109607861F341004D
:1053E000014660F382016170307AE0708AE7A07F45
:1053F00000F00300022809D05FF0000080F00101F6
:1054000050460DF0C1FA040003D101E00120F5E798
:10541000FFDF022104F1850010F0F1FC0420287068
:1054200004F5B4706860B4F88500288230481038FC
:105430007C346C61C5E9028064E703E024E15BE051
:105440002DE015E0A07F00F00300022807D0002027
:1054500080F0010150460DF097FA18B901E00120E3
:10546000F6E7FFDF324621465046BDE8F84FEAE551
:1054700004B9FFDF20782128A1D93079012803D190
:10548000E07F40F00800E077324621465046FFF7C3
:10549000DAFD2046BDE8F84F2321FDF73BBE327907
:1054A000AA8005F108030921504604F082FEE86055
:1054B00010B10520287025E7A07F00F00300022826
:1054C00008D0002080F0010150460DF05DFA040084
:1054D00003D101E00120F5E7FFDF04F162010223BF
:1054E0001022081F0DF0D7F807703179417009E7D5
:1054F0004802002040420F00A07F00F00300022875
:1055000008D0002080F0010150460DF03DFA050062
:1055100003D101E00120F5E7FFDF95F8840000F0FA
:10552000030001287AD1A07F00F00307E07F10F08C
:10553000010602D0022F04D133E095F8A000C00785
:105540002BD0D5F8601121B395F88320087C62F345
:1055500087000874A17FCA09D5F8601162F3410081
:105560000874D5F8601166F300000874AEB1D5F880
:105570006001102204F12401883520F04BF8287EC8
:1055800040F001002876287820F0010005F888090D
:1055900000E016B1022F04D02DE095F88800C00776
:1055A00027D0D5F85C1121B395F88320087C62F3ED
:1055B00087000874A17FCA09D5F85C1162F3410025
:1055C0000874D5F85C1166F3000008748EB1D5F844
:1055D0005C01102204F12401883520F01BF82878A2
:1055E00040F0010005F8180B287820F0010005F8BC
:1055F000A009022F44D0002000EB400005EBC000C2
:1056000090F88800800709D595F87C00D5F86421CA
:10561000400805F17D011032FDF7E5FE8DF80090A0
:1056200095F884006A4600F003008DF8010095F8B3
:1056300088108DF8021095F8A0008DF8030021461F
:10564000504601F043FA2078252805D0212807D0BC
:10565000FFDF2078222803D922212046FDF75AFDBA
:10566000A07F00F0030002280CD0002080F0010190
:1056700050460DF09BF900283FF44FAEFFDF41E6A6
:105680000120B9E70120F1E7706847703AE6FFDFD3
:1056900038E670B5FE4C002584F85C5025660EF0A7
:1056A00030FE04F11001204603F0CEFE84F83050A5
:1056B00070BD70B50D46FDF7C6FE040000D1FFDFDA
:1056C0004FF4B871284620F046F804F12400286110
:1056D000A07F00F00300022808D0012105F1E000BE
:1056E0000EF010FE002800D0FFDF70BD0221F5E7AC
:1056F0000A46014602F1E0000EF024BE70B50546F0
:10570000406886B001780A2906D00D2933D00E29C9
:105710002FD0FFDF06B070BD86883046FDF793FEC0
:10572000040000D1FFDF20782128F3D028281BD1E6
:10573000686802210E3001F0BEF9A8B1686808213E
:10574000801D01F0B8F978B104F1240130460CF065
:105750008DF803F0DFFC00B1FFDF06B02046BDE8A6
:1057600070402921FDF7D6BC06B0BDE8704003F0BB
:10577000B2BE012101726868C6883046FDF763FE3B
:10578000040000D1FFDFA07F00F00301022902D155
:1057900020F01000A077207821280AD06868017ACC
:1057A00009B1007980B1A07F00F00300022862D027
:1057B000FFDFA07F00F003000228ABD1FEF795F8D1
:1057C0000028A7D0FFDFA5E703F085FEA17F08062C
:1057D0002BD5E07FC00705D094F8200000F01F0013
:1057E000102820D05FF0050084F8230020782928B5
:1057F0001DD02428DDD13146042010F0DFFD222108
:105800002046FDF787FCA07F00F00300022830D07F
:105810005FF0000080F0010130460DF0C7F800286D
:10582000C7D0FFDFC5E70620DEE70420DCE701F094
:105830000300022808D0002080F0010130460DF05E
:10584000A3F8050003D101E00120F5E7FFDF2521E2
:105850002046FDF75FFC03208DF80000694605F146
:10586000E0000EF066FD0228A3D00028A1D0FFDFE3
:105870009FE70120CEE703F02EFE9AE72DE9F043E3
:1058800087B09946164688460746FDF7DCFD0400BA
:105890004BD02078222848D3232846D0E07F000729
:1058A00043D4A07F00F00300022809D05FF000007D
:1058B00080F0010138460DF067F8050002D00CE0D9
:1058C0000120F5E7A07F00F00300022805D00121A8
:1058D000002238460DF04FF805466946284601F08B
:1058E0001CF9009800B9FFDF45B10098E03505616B
:1058F0002078222806D0242804D007E00099002030
:10590000086103E025212046FDF704FC00980121F1
:1059100041704762868001A9C0E902890EF024FD2A
:10592000022802D0002800D0FFDF07B0BDE8F083D6
:1059300070B586B00546FDF786FD017822291ED98F
:10594000807F00F00300022808D0002080F00101D1
:1059500028460DF019F804002FD101E00120F5E7E9
:10596000FFDF2AE0B4F85E0004F1620630440178FB
:10597000427829B121462846FFF714FCB0B9C9E6A0
:10598000ADF804200921284602AB04F012FC039074
:105990000028F4D005208DF80000694604F1E000ED
:1059A0000EF0C7FC022801D000B1FFDF0223102255
:1059B000314604F15E000CF0A4FEB4F8600000284B
:1059C000D0D1A7E610B586B00446FDF73CFD0178BE
:1059D00022291BD9807F00F00300022808D0002074
:1059E00080F0010120460CF0CFFF040003D101E05C
:1059F0000120F5E7FFDF06208DF80000694604F17D
:105A0000E0000EF096FC002800D0FFDF06B010BDCD
:105A10002DE9F05F05460C46002700789046010905
:105A20003E4604F1080BBA4602297DD0072902D070
:105A30000A2909D146E0686801780A2905D00D29AC
:105A400030D00E292ED0FFDFBBE114271C26002CFE
:105A50006BD08088A080FDF7F6FC5FEA000900D1DA
:105A6000FFDF99F817005A46400809F11801FDF7C1
:105A7000BAFC6868C0892082696851F8060FC4F8CA
:105A800012004868C4F81600A07E20F0060001E06D
:105A90002802002040F00100A07699F81E0040F096
:105AA00020014DE01A270A26002CD1D0C088A08002
:105AB000FDF7C9FC050000D1FFDF59462846FFF776
:105AC00042FB7EE10CB1A88BA080287A0B287DD008
:105AD00006DC01287BD0022808D0032804D135E059
:105AE0000D2875D00E2874D0FFDF6AE11E27092625
:105AF000002CADD0A088FDF7A6FC5FEA000900D11C
:105B0000FFDF287B00F003000128207A1BD020F063
:105B100001002072297B890861F341002072297BF2
:105B2000C90861F3820001E041E1F2E02072297BC3
:105B3000090961F3C300207299F81E0040F040018A
:105B400089F81E103DE140F00100E2E713270D2621
:105B5000002CAAD0A088FDF776FC8146807F00F05B
:105B60000300022808D0002080F00101A0880CF07A
:105B70000BFF050003D101E00120F5E7FFDF99F8F5
:105B80001E0000F00302022A50D0686F817801F0F5
:105B900003010129217A4BD021F001012172837880
:105BA0009B0863F3410121728378DB0863F3820170
:105BB000217283781B0963F3C3012172037863F3B5
:105BC00006112172437863F3C71103E061E0A9E095
:105BD00090E0A1E0217284F809A0C178A172022AA4
:105BE00029D00279E17A62F30001E1720279520868
:105BF00062F34101E1720279920862F38201E1727B
:105C00000279D20862F3C301E1724279217B62F327
:105C1000000121734279520862F3410121734279F4
:105C2000920862F382012173407928E0A86FADE702
:105C300041F00101B2E74279E17A62F30001E172D9
:105C40004279520862F34101E1724279920862F3AB
:105C50008201E1724279D20862F3C301E1720279F2
:105C6000217B62F3000121730279520862F3410142
:105C700021730279920862F3820121730079C008CE
:105C800060F3C301217399F80000232831D926213C
:105C900040E018271026E4B3A088FDF7D4FB834624
:105CA000807F00F00300022809D0002080F001016D
:105CB000A0880CF069FE5FEA000903D101E0012031
:105CC000F4E7FFDFE868A06099F8000040F0040105
:105CD00089F8001099F80100800708D50120207389
:105CE0009BF8000023286CD92721584651E084F8FE
:105CF0000CA066E015270F265CB1A088FDF7A3FB7A
:105D0000814606225946E86808F0C1FA0120A073CE
:105D1000A0E041E048463CE016270926E4B3287B92
:105D200020724EE0287B19270E26ACB3C4F808A0D9
:105D3000A4F80CA0012807D0022805D0032805D01C
:105D4000042803D0FFDF0DE0207207E0697B042800
:105D500001F00F0141F0800121721ED0607A20F025
:105D600003006072A088FDF76EFB054600782128CD
:105D700027D0232800D0FFDFA87F00F003000228EF
:105D800013D0002080F00101A0880CF00FFE22212A
:105D90002846FDF7BFF914E004E0607A20F0030024
:105DA000401CDEE7A8F8006010E00120EAE70CB133
:105DB0006888A080287A68B301280AD002284FD0CA
:105DC000FFDFA8F800600CB1278066800020BDE8E6
:105DD000F09F15270F26002CE4D0A088FDF733FB99
:105DE000807F00F00300022808D0002080F001012D
:105DF000A0880CF0C9FD050003D101E00120F5E702
:105E0000FFDFD5F81D000622594608F040FA84F855
:105E10000EA0D6E717270926002CC3D0A088FDF7CF
:105E200012FB8146807F00F00300022808D000208A
:105E300080F00101A0880CF0A7FD050003D101E06E
:105E40000120F5E7FFDF6878800701D5022000E038
:105E50000120207299F800002328B2D9272159E7A0
:105E600019270E26002C9DD0A088FDF7ECFA5FEADA
:105E7000000900D1FFDFC4F808A0A4F80CA084F842
:105E800008A0A07A40F00300A07299F81E10C9097A
:105E900061F38200A07299F81F2099F81E1012EA8F
:105EA000D11F05D099F8201001F01F0110292BD027
:105EB00020F00800A07299F81F10607A61F3C30007
:105EC0006072697A01F003010129A2D140F0040057
:105ED000607299F81E0000F003000228E87A16D0DC
:105EE000217B60F300012173AA7A607B62F30000DA
:105EF0006073EA7A520862F341012173A97A490872
:105F000061F3410060735CE740F00800D2E7617B19
:105F100060F300016173AA7A207B62F300002073B2
:105F2000EA7A520862F341016173A97A490861F380
:105F30004100207345E710B5FE4C30B101461022F8
:105F400004F120001FF066FB012084F8300010BD32
:105F500010B5044600F0D1FDF64920461022BDE8F8
:105F6000104020311FF056BB70B5F24D06004FF0C7
:105F7000000413D0FBF7A7F908B110240CE00621A8
:105F8000304608F06BF9411C05D028665FF001002F
:105F900085F85C0000E00724204670BD0020F7E78C
:105FA000007810F00F0204D0012A05D0022A0CD18B
:105FB00010E0000909D10AE00009012807D00228F1
:105FC00005D0032803D0042801D0072070470870AB
:105FD000002070470620704705282AD2DFE800F02D
:105FE00003070F171F00087820F0FF001EE0087855
:105FF00020F00F00401C20F0F000103016E0087870
:1060000020F00F00401C20F0F00020300EE0087857
:1060100020F00F00401C20F0F000303006E008783F
:1060200020F00F00401C20F0F000403008700020ED
:106030007047072070472DE9F041804688B00D4633
:1060400000270846FBF78CF9A8B94046FDF7FBF995
:10605000040003D02078222815D104E043F2020086
:1060600008B0BDE8F08145B9A07F410603D500F036
:106070000300022801D01020F2E7A07FC10601D45E
:10608000010702D50DB10820EAE7E17F090701D534
:106090000D20E5E700F00300022805D125B12846D0
:1060A000FEF762FF0700DBD1A07F00F003000228AB
:1060B00008D0002080F0010140460CF065FC06008D
:1060C00002D00FE00120F5E7A07F00F003000228D6
:1060D0000ED0002080F00101002240460CF04BFC65
:1060E000060007D0A07F00F00300022804D009E0DA
:1060F0000120EFE70420B3E725B12A4631462046C8
:10610000FEF756FF6946304600F007FD009800B9DB
:10611000FFDF0099022006F1E0024870C1F82480F8
:106120004A6100220A81A27F02F00302022A1CD0E7
:1061300001200871287800F00102087E62F3010056
:1061400008762A78520862F3820008762A78920844
:1061500062F3C30008762A78D20862F30410087646
:1061600024212046FCF7D6FF33E035B30871301DFB
:1061700088613078400908777078C0F3400048772C
:10618000287800F00102887F62F301008877A27FFF
:10619000D20962F382008877E27F62F3C3008877D6
:1061A000727862F304108877A878C87701F1210229
:1061B00028462031FEF71DFF03E00320087105206B
:1061C000087625212046FCF7A5FFA07F20F040009F
:1061D000A07701A900980EF0C7F8022801D000B1FD
:1061E000FFDF38463CE72DE9FF4F534A0D4699B093
:1061F0009A4607CA0AAB002783E807001998FDF7FB
:1062000022F9060006D03078262806D008201DB0D6
:10621000BDE8F08F43F20200F9E7B07F00F0030918
:10622000B9F1020F0AD05DB91B98FEF79DFE002858
:10623000EDD1B07F00F00300022801D11B9890BB84
:10624000B07F00F00300022808D0002080F0010198
:1062500019980CF099FB040003D101E00120F5E747
:10626000FFDF852D28D007DCF5B1812D1ED0822DD2
:106270001ED0832D08D11DE0862D1FD0882D1FD064
:10628000892D1FD08A2D1FD00F2020710F281DD0DF
:1062900003F01EF9E0B101208DF83C00201D1090A4
:1062A0002079B8B15BE111E00020EEE70120ECE7D6
:1062B0000220EAE70320E8E70520E6E70620E4E716
:1062C0000820E2E70920E0E70A20DEE707209EE752
:1062D00011209CE7B9F1020F03D0A56F03D1A06F85
:1062E00002E0656FFAE7606F804632D04FF0010040
:1062F00001904FF002000090214630461B9AFEF7B5
:1063000057FE1B98007800F00101A87861F30100A6
:10631000A870B17FC90961F38200A870F17F61F3B1
:10632000C300A870617861F30410A8702078400958
:10633000287003E028020020045B02006078C0F3AC
:10634000400068701B988078E870002068712871A0
:1063500003E00220019001200090A87898F8021034
:10636000C0F3C000C1F3C00108405FEA000B2DD0AC
:106370005046FAF7A8FF78BBDAF80C00FAF7A3FF4B
:1063800050BBDAF81C00FAF79EFF28BBDAF80C00C5
:10639000A060DAF81C00E060607898F8012042EA1A
:1063A000500100BF61F34100607098F80210C0B264
:1063B00000EA111161F3000060700020207700995D
:1063C00006F11700022908D0012107E0607898F84B
:1063D000012002EA5001E5E732E0002104EB8101EF
:1063E00048610199701C022901D0012100E00021BF
:1063F00004EB81014861A87800F00300012857D11F
:1064000098F8020000F00300012851D1B9F1020F01
:1064100004D02A1D691D1B98FEF7EBFD287998F81A
:10642000041008408DF83400697998F8052011406F
:106430008DF8381008433BD05046FAF744FF08B1B6
:106440001020E4E60AF110010491B9F1020F17D00F
:106450000846002104F18C03CDE9000304F5AE7277
:1064600002920DAB5A462046FEF70CFE0028E8D1FA
:10647000B9F1020F08D0504608D14FF0010107E0F2
:1064800050464FF00101E5E70498F5E74FF00001B1
:1064900004F1A403CDE9000304F5B072029281F087
:1064A00001010EAB5A462046FEF7ECFD0028C8D18C
:1064B0006078800734D4A87898F80210C0F3800080
:1064C000C1F3800108432BD0297898F800000AAA6C
:1064D000B9F1020F06D032F811204300DA4002F081
:1064E00003070AE032F810204B00DA4012F00307ED
:1064F00005D0012F0BD0022F0BD0032F07D0BBF1FB
:10650000000F0DD0012906D0042904D008E002278D
:10651000F5E70127F3E7012801D0042800D104277B
:10652000B07F40F08000B077F17F6BF30001F1772E
:106530006078800706D50320A071BBF1000F0ED153
:10654000002028E00220022F18D0012F18D0042F9D
:1065500029D00020A071B07F20F08000B0772521E5
:106560003046FCF7D7FD0FA904F1E0000DF0E1FE85
:1065700010B1022800D0FFDF002048E6A071DFE75D
:10658000A0710D2104F120001FF0E5F8207840F003
:106590000200207001208DF85C0017AA314619987E
:1065A00000F094FADBE70120A071D8E72DE9F04371
:1065B00087B09046894604460025FCF744FF060054
:1065C00006D03078272806D0082007B0BDE8F08331
:1065D00043F20200F9E7B07F00F00300022809D07F
:1065E0005FF0000080F0010120460CF0CDF90400BE
:1065F00003D101E00120F5E7FFDFA7795FEA090099
:1066000005D0012821D0B9F1020F26D110E0B8F150
:10661000000F22D1012F05D0022F05D0032F05D066
:10662000FFDF2DE00C252BE0012529E0022527E0E6
:106630004046FAF748FEB0B9032F0ED1102241466A
:1066400004F11D001EF0E6FF1AE0012F02D0022F18
:1066500003D104E0B8F1000F12D00720B5E740469F
:10666000FAF731FE08B11020AFE7102104F11D0048
:106670001FF04FF80621404607F0F0FDC4F81D005A
:106680002078252140F0020020703046FCF742FDC2
:106690002078C10713D020F00100207002208DF86F
:1066A000000004F11D0002908DF804506946C330CB
:1066B0000DF03FFE022803D010B1FFDF00E0257788
:1066C000002082E730B587B00D460446FCF7BBFEDC
:1066D000A0B1807F00F00300022812D05FF000001C
:1066E00080F0010120460CF04FF904000ED028463E
:1066F000FAF7E9FD38B1102007B030BD43F20200CF
:10670000FAE70120ECE72078400701D40820F3E7FE
:10671000294604F13D00202205461EF07BFF20782B
:1067200040F01000207001070FD520F00800207005
:1067300007208DF80000694604F1E00001950DF096
:10674000F8FD022801D000B1FFDF0020D4E770B5CA
:106750000D460646FCF777FE18B10178272921D1AE
:1067600002E043F2020070BD807F00F003000228C7
:1067700008D0002080F0010130460CF005F904003B
:1067800003D101E00120F5E7FFDFA079022809D15C
:106790006078C00706D02A4621463046FEF702FD43
:1067A00010B10FE0082070BDB4F860000E280BD2C5
:1067B00004F1620102231022081F0BF06CFF01217B
:1067C00001704570002070BD112070BD70B5064687
:1067D00014460D460846FAF776FD18B92046FAF732
:1067E00098FD08B1102070BDA6F57F40FF380ED08F
:1067F0003046FCF728FE38B1417822464B08811C10
:106800001846FCF7F0FD07E043F2020070BD204699
:10681000FDF7FCFD0028F9D11021E01D0FF0EFFA83
:10682000E21D294604F1170000F087F9002070BD31
:106830002DE9F04104468AB01546884600270846EF
:10684000FAF78EFD18B92846FAF78AFD10B1102024
:106850000AB006E42046FCF7F6FD060003D03078C7
:1068600027281AD102E043F20200F1E7B07F00F0DE
:106870000300022808D0002080F0010120460CF01F
:1068800083F8040003D101E00120F5E7FFDF207861
:10689000400702D56078800701D40820D8E7B07F90
:1068A00000F00300022803D0A06F03D1A16F02E023
:1068B000606FFAE7616F407800B19DB1487810B120
:1068C000B8F1000F0ED0ADB1EA1D06A8E16800F0E6
:1068D00034F9102206A905F117001EF06FFE18B159
:1068E000042707E00720B3E71022E91D04F12D007B
:1068F0001EF090FEB8F1000F06D0102208F107013B
:1069000004F11D001EF086FE2078252140F00200D3
:1069100020703046FCF7FEFB2078C10715D020F030
:106920000100207002208DF8000004F11D0002908B
:10693000103003908DF804706946B3300DF0F9FC07
:10694000022803D010B1FFDF00E0277700207FE7A7
:10695000F8B515460E460746FCF775FD040004D051
:106960002078222804D00820F8BD43F20200F8BDA8
:10697000A07F00F00300022802D043F20500F8BD1A
:106980003046FAF7A0FC18B92846FAF79CFC08B183
:106990001020F8BD00953288B31C21463846FEF71A
:1069A00024FC112815D00028F3D1297C4A08A17FA6
:1069B00062F3C711A177297CE27F61F30002E277DD
:1069C000297C890884F82010A17F21F04001A1775B
:1069D000F8BDA17F0907FBD4D6F80200C4F8360041
:1069E000D6F80600C4F83A003088A086102229465E
:1069F00004F124001EF00EFE287C4108E07F61F3C4
:106A00004100E077297C61F38200E077287C8008F0
:106A100084F82100A07F40F00800A0770020D3E791
:106A200070B50D4606460BB1072070BDFCF70BFD97
:106A3000040007D02078222802D3A07F800604D447
:106A4000082070BD43F2020070BDADB1294630464A
:106A50000AF00CFF02F05EFB297C4A08A17F62F37A
:106A6000C711A177297CE27F61F30002E277297CDC
:106A7000890884F8201004E030460AF01AFF02F07A
:106A800049FBA17F21F02001A17770BD70B50D46B3
:106A9000FCF7D9FC040005D02846FAF73AFC20B1EF
:106AA000102070BD43F2020070BD29462046FEF75B
:106AB0004AFB002070BD04E010F8012B0AB1002051
:106AC0007047491E89B2F7D20120704770B515464C
:106AD000064602F0FDFC040000D1FFDF207820F024
:106AE0000F00801C20F0F0002030207066802868A5
:106AF000A060BDE8704002F0EEBC10B5134C94F8F5
:106B00003000002808D104F12001A1F110000DF09F
:106B100052FC012084F8300010BD10B190F8B9206B
:106B20002AB10A4890F8350018B1002003E0B830C7
:106B300001E0064834300860704708B50023009330
:106B400013460A460CF01BF908BD0000280200207D
:106B500018B18178012938D101E0102070470188EF
:106B600042F60112881A914231D018DC42F6010235
:106B7000A1EB020091422AD00CDC41B3B1F5C05F19
:106B800025D06FF4C050081821D0A0F57060FF38F0
:106B90001BD11CE001281AD002280AD117E0B0F559
:106BA000807F14D008DC012811D002280FD00328E0
:106BB0000DD0FF2809D10AE0B0F5817F07D0A0F5FC
:106BC0008070033803D0012801D0002070470F20C7
:106BD00070470A281FD008DC0A2818D2DFE800F026
:106BE000191B1F1F171F231D1F21102815D008DC7C
:106BF0000B2812D00C2810D00D2816D00F2806D143
:106C00000DE011280BD084280BD087280FD003204B
:106C100070470020704705207047072070470F20FD
:106C2000704704207047062070470C20704743F2DD
:106C30000200704738B50C46050041D06946FFF7A1
:106C4000AFF9002819D19DF80010607861F30200B7
:106C500060706946681CFFF7A3F900280DD19DF804
:106C60000010607861F3C5006070A978C1F341013C
:106C7000012903D0022905D0072038BD217821F051
:106C8000200102E0217841F020012170410704D069
:106C9000A978C90861F386106070607810F0380F29
:106CA00007D0A978090961F3C710607010F0380F98
:106CB00002D16078400603D5207840F04000207073
:106CC000002038BD70B50446002008801546606875
:106CD000FFF7B0FF002816D12089A189884211D87A
:106CE00060688078C0070AD0B1F5007F0AD840F20A
:106CF0000120B1FBF0F200FB1210288007E0B1F593
:106D0000FF7F01D90C2070BD01F2012129800020F4
:106D100070BD10B50478137864F300031370047821
:106D2000640864F3410313700478A40864F38203D5
:106D300013700478E40864F3C3031370047824091F
:106D400064F3041313700478640964F34513137037
:106D50000078800960F38613137031B10878C10799
:106D600001D1800701D5012000E0002060F3C713A6
:106D7000137010BD4278530702D002F0070306E0FB
:106D800012F0380F02D0C2F3C20300E001234A78A8
:106D900063F302024A70407810F0380F02D0C0F35B
:106DA000C20005E0430702D000F0070000E0012028
:106DB00060F3C5024A7070472DE9F04F95B00D00A1
:106DC000824612D0122128461EF0A3FC4FF6FF7B0C
:106DD00005AA0121584607F05CF8002426463746EC
:106DE0004FF420586FF4205973E0102015B0BDE81F
:106DF000F08F00BF9DF81E0001280AD1BDF81C10BD
:106E000041450BD011EB09000AD001280CD0022813
:106E10000CD0042C0ED0052C0FD10DE0012400E085
:106E20000224BDF81A6008E0032406E00424BDF83B
:106E30001A7002E0052400E00624BDF81A1051453E
:106E400047D12C74BEB34FF0000810AA4FF0070AC8
:106E5000CDE90282CDE900A80DF13C091023CDF85F
:106E6000109042463146584607F0C6F808BBBDF8B8
:106E70003C002A46C0B210A90DF013FBC8B9AE8180
:106E8000CFB1CDE900A80DF1080C0AAE40468CE860
:106E90004102132300223946584607F0ADF840B9A5
:106EA000BDF83C00F11CC01EC0B22A1D0DF0F9FA5D
:106EB00010B103209AE70AE0BDF82900E881062C0A
:106EC00005D19DF81E00A872BDF81C002881002085
:106ED0008CE705A806F0E9FF00288BD0FFF779FEC4
:106EE00084E72DE9F0471C46DDE90978DDF82090BC
:106EF00015460E00824600D1FFDF0CB1208818B184
:106F0000D5B11120BDE8F087022D01D0012100E0AC
:106F1000002106F1140005F0ABFEA8F800000246BF
:106F20003B462946504603F044F9C9F8000008B929
:106F3000A41C3C600020E5E71320E3E7F0B414460E
:106F4000DDE904528DB1002314B1022C09D101E016
:106F5000012306E00D7CEE0703D025F00105012397
:106F60000D742146F0BC03F0AFBF1A80F0BC70472F
:106F70002DE9FE4F91461A881C468A468046FAB192
:106F800002AB494603F015F9050019D04046A61C8E
:106F900027880BF03DFE3246072629463B460096E1
:106FA0000BF04BFA20882346CDE900504A46514663
:106FB0004046FFF7C3FF002020800120BDE8FE8F80
:106FC0000020FBE72DE9F04786B082460EA89046E8
:106FD00090E8B000894604AA05A903A88DE8070037
:106FE0001E462A4621465046FFF77BFF039901B112
:106FF00001213970002818D1F94904F1140204ABB9
:107000000860039805998DE80700424649465046B6
:1070100006F0E5F9A8B1092811D2DFE800F005086B
:107020000510100A0C0C0E00002006B06AE71120B3
:10703000FBE70720F9E70820F7E70D20F5E7032035
:10704000F3E7BDF810100398CDE9000133462A4656
:1070500021465046FFF772FFE6E72DE9F04389B07D
:107060000D46DDE9108781461C461646142103A80B
:107070001EF071FB012002218DF810108DF80C001C
:107080008DF81170ADF8146064B1A278D20709D000
:107090008DF81600E088ADF81A00A088ADF8180049
:1070A000A068079008A80095CDE90110424603A901
:1070B00048466B68FFF786FF09B0BDE8F083F0B57E
:1070C0008BB000240646069407940727089405A869
:1070D0000994019400970294CDE903400D461023D2
:1070E0002246304606F088FF78B90AA806A901941E
:1070F00000970294CDE90310BDF814300022294610
:10710000304606F04FFD002801D0FFF762FD0BB0BE
:10711000F0BD06F0EFBB2DE9FC410C468046002691
:1071200002F0D6F9054620780D287DD2DFE800F080
:10713000BC0713B325BD49496383AF959B00A8489D
:10714000006820B1417841F010014170ADE0404647
:1071500002F0EEF9A9E0042140460BF015FC07000F
:1071600000D1FFDF07F11401404605F015FDA5BB76
:1071700013214046FDF724FC97E0042140460BF024
:1071800003FC070000D1FFDFE088ADF8000000201D
:10719000B8819DF80000010704D5C00602D5A0887B
:1071A000B88105E09DF8010040067ED5A088F881F1
:1071B00005B9FFDF22462946404601F0BDFC022604
:1071C00073E0E188ADF800109DF8011009060FD5B5
:1071D000072803D006280AD00AE024E0042140460C
:1071E0000BF0D2FB060000D1FFDFA088F081022661
:1071F000CDB9FFDF17E0042140460BF0C5FB0700C7
:1072000000D1FFDF07F1140006F0ABFB90F0010F97
:1072100002D1E079000648D5387C022640F0020011
:10722000387405B9FFDF00E03EE0224629464046BB
:1072300001F082FC39E0042140460BF0A5FB017C03
:10724000002D01F00206C1F340016171017C21F0C3
:1072500002010174E7D1FFDFE5E702260121404684
:1072600002F098F921E0042140460BF08DFB054621
:10727000606800902089ADF804000122694640460C
:1072800002F0A9F9287C20F0020028740DE0002DFE
:10729000C9D1FFDFC7E7022600214046FBF714F9FA
:1072A000002DC0D1FFDFBEE7FFDF3046BDE8FC8127
:1072B0003EB50C0009D001466B4601AA002006F03D
:1072C0001DFF20B1FFF785FC3EBD10203EBD002014
:1072D0002080A0709DF8050002A900F00700FEF7CD
:1072E0007BFE50B99DF8080020709DF8050002A9AA
:1072F000C0F3C200FEF770FE08B103203EBD9DF84A
:10730000080060709DF80500C109A07861F30410C1
:10731000A0709DF80510890961F3C300A0709DF865
:107320000410890601D5022100E0012161F3420029
:107330009DF8001061F30000A07000203EBD70B504
:10734000144606460D4651EA040005D075B10846BC
:10735000F9F7FDFF78B901E0072070BD29463046F6
:1073600006F02DFF10B1BDE8704032E454B1204664
:10737000F9F7EDFF08B1102070BD21463046BDE899
:10738000704095E7002070BD2DE9FC5F0C469046EB
:107390000546002701780822007A3E46B2EB111F0D
:1073A0007ED104F10A0100910A31821E4FF0020AD7
:1073B00004F1080B0191092A73D2DFE802F0ECDF37
:1073C00005F427277AA9CD00688804210BF0DCFAA0
:1073D000060000D1FFDFB08920B152270726C2E0A6
:1073E0008C02002051271026002C7DD06888A080B8
:1073F0000120A071A88900220099FFF7A0FF0028B2
:1074000073D1A8892081288AE081D1E0B5F8129053
:10741000072824D1E87B000621D5512709F1140063
:1074200086B2002CE1D0A88900220099FFF787FFDF
:1074300000285AD16888A08084F806A0A8892081F5
:107440000120A073288A2082A4F81290A88A0090B4
:1074500068884B46A969019A01F04BFBA8E05027C8
:1074600009F1120086B2002C3ED0A88900225946AC
:10747000FFF765FF002838D16888A080A889E080E0
:10748000287A072813D002202073288AE081E87B1D
:10749000C0096073A4F81090A88A0090688801E081
:1074A00083E080E04B4604F11202A969D4E7012091
:1074B000EAE7B5F81290512709F1140086B2002CC2
:1074C00066D0688804210BF05FFA83466888A08044
:1074D000A88900220099FFF732FF00286ED184F8B6
:1074E00006A0A889208101E052E067E00420A07393
:1074F000288A2082A4F81290A88A009068884B46B7
:10750000A969019A01F0F5FAA989ABF80E104FE0CC
:107510006888FBF798FF0746688804210BF034FA67
:10752000064607B9FFDF06B9FFDF687BC00702D058
:107530005127142601E0502712264CB36888A080FA
:10754000502F06D084F806A0287B594601F0E1FAB6
:107550002EE0287BA11DF9E7FE49A88949898142CF
:1075600005D1542706269CB16888A08020E05327C7
:107570000BE06888A080A889E08019E06888042171
:107580000BF002FA00B9FFDF55270826002CF0D1D6
:10759000A8F8006011E056270726002CF8D068886C
:1075A000A080002013E0FFDF02E0012808D0FFDF09
:1075B000A8F800600CB1278066800020BDE8FC9F21
:1075C00057270726002CE3D06888A080687AA0712E
:1075D000EEE7401D20F0030009B14143091D01EB16
:1075E0004000704713B5DB4A00201071009848B185
:1075F000002468460AF0E5FF002C02D1D64A009923
:1076000011601CBD01240020F4E770B50D4606464C
:1076100086B014465C2128461EF09DF804B9FFDFB1
:10762000A0786874A2782188284601F09CFA00208E
:10763000A881E881228805F11401304605F091FA0D
:107640006A460121304606F024FC19E09DF803004B
:10765000000715D5BDF806103046FFF730FD9DF840
:107660000300BDF8061040F010008DF80300BDF8CF
:107670000300ADF81400FF233046059A06F06AFDBA
:10768000684606F012FC0028E0D006B070BD10B5C8
:107690000C4601F1140005F09BFA0146627C20467D
:1076A000BDE8104001F094BA30B50446A94891B045
:1076B0004FF6FF75C18905AA284606F0EAFB30E0BF
:1076C0009DF81E00A0422AD001282AD1BDF81C0036
:1076D000B0F5205F03D042F60101884221D100209D
:1076E00002AB0AAA0CA9019083E8070007200090CA
:1076F000BDF81A1010230022284606F07DFC38B988
:10770000BDF828000BAAC0B20CA90CF0CAFE10B13B
:10771000032011B030BD9DF82E00A04201D1002001
:10772000F7E705A806F0C1FB0028C9D00520F0E75F
:1077300070B5054604210BF027F9040000D1FFDFE6
:1077400004F114010C46284605F026FA2146284685
:10775000BDE8704005F027BA70B58AB00C46064601
:10776000FBF771FE050014D02878222827D30CB12E
:10777000A08890B101208DF80C0003208DF8100036
:1077800000208DF8110054B1A088ADF818002068D1
:1077900007E043F202000AB070BD0920FBE7ADF834
:1077A00018000590042130460BF0EEF8040000D1DB
:1077B000FFDF04F1140005F022FA000701D40820CD
:1077C000E9E701F085FE60B108A802210094CDE947
:1077D000011095F8232003A930466368FFF7F2FBF8
:1077E000D9E71120D7E72DE9F04FB2F802A0834680
:1077F00089B0154689465046FBF725FE0746042109
:1078000050460BF0C1F80026044605964FF00208DA
:107810000696ADF81C6007B9FFDF04B9FFDF4146EB
:10782000504603F0BCFE50B907AA06A905A88DE88A
:1078300007004246214650466368FFF752FB454821
:1078400007AB0660DDE9051204F11400CDF80090E5
:10785000CDE90320CDE9013197F823205946504660
:107860006B6805F015FA06000AD0022E04D0032E2C
:1078700014D0042E00D0FFDF09B03046BDE8F08FF1
:10788000BDF81C000028F7D00599CDE9001042464C
:10789000214650466368FFF751FBEDE7687840F0FA
:1078A00008006870E8E72DE9F04F99B004464FF002
:1078B00000082848ADF81C80ADF82080ADF8248081
:1078C000A0F80880ADF81480ADF81880ADF82C80D1
:1078D000ADF82880007916460D464746012808D0A5
:1078E000022806D0032804D0042802D0082019B0AA
:1078F000C4E72046F9F7E7FC80BB2846F9F7E3FC2C
:1079000060BB6068F9F72CFD40BB606848B16089D6
:107910002189884202D8B1F5007F01D90C20E6E721
:1079200080460EAA06A92846FFF7CCF90028DED12A
:1079300068688078C0F34100022808D19DF81900DA
:1079400010F0380F03D02869F9F701FD30B905A907
:10795000206904E08C0200201400002020E0FFF7E2
:1079600069F90028C3D1206948B1607880079DF883
:10797000150000F0380001D5F0B300E0E0BB9DF841
:10798000140080060ED59DF8150010F0380F03D0B6
:107990006068F9F7DCFC18B96068F9F7E1FC08B138
:1079A0001020A4E70AA96069FFF744F900289ED1D6
:1079B000606940B19DF8290000F0070101293CD120
:1079C00010F0380F39D00BA9A069FFF733F9002860
:1079D0008DD19DF8280080062FD49DF82C008006BC
:1079E0002BD4A06950B19DF82D0000F007010129AA
:1079F00023D110F0380F00E01FE01ED0E06818B16E
:107A00000078D0B11C2818D20FAA611C2046FFF7BD
:107A100080F90121384661F30F2082468DF852101B
:107A2000B94642F603000F46ADF850000DF13F0293
:107A300018A928680CF054FD08B1072057E79DF8F5
:107A4000600015A9CDF80090C01CCDE9019100F0AF
:107A5000FF0B00230BF20122514614A806F05CF93B
:107A6000F0BBBDF854000C90FD492A8928690092AA
:107A7000CDE901016B89BDF838202868069906F028
:107A80004BF901007ED120784FF0020AC10601D4E3
:107A900080062BD5ADF80C90606950B90AA906A8EC
:107AA000FFF768F99DF8290020F00700401C8DF8C9
:107AB00029009DF8280008A940F0C8008DF828008A
:107AC0008DF8527042F60210ADF8500003AACDF8BE
:107AD00000A0CDE90121002340F2032214A800E018
:107AE0001EE00A9906F018F901004BD1DC484D461A
:107AF00008385B460089ADF83D000FA8CDE902903B
:107B0000CDF80490CDF810904FF007090022CDF881
:107B10000090BDF854104FF6FF7006F043F810B116
:107B2000FFF757F8E3E69DF83C00000625D5294607
:107B3000012060F30F218DF852704FF42450ADF8FE
:107B40005000ADF80C5062789DF80C00002362F3F1
:107B500000008DF80C006278CDF800A0520862F3A6
:107B600041008DF80C0003AACDE9012540F2032263
:107B700014A806F0D1F8010004D1606888B3206928
:107B8000A8B900E086E005A906A8FFF7F3F8607839
:107B9000800706D49DF8150020F038008DF81500F8
:107BA00005E09DF8140040F040008DF814008DF8B9
:107BB000527042F60110ADF85000208940F20121C8
:107BC000B0FBF1F201FB1202606809ABCDF8008056
:107BD000CDE90103002314A8059906F09DF80100E2
:107BE00058D12078C00729D0ADF80C50A06950B901
:107BF0000BA906A8FFF7BEF89DF82D0020F007009E
:107C0000401C8DF82D009DF82C008DF8527040F02E
:107C100040008DF82C0042F60310ADF8500007A983
:107C200003AACDF800A0CDE90121002340F20322F0
:107C300014A80B9906F070F801002BD1E06868B326
:107C40002946012060F30F218DF8527042F604108E
:107C5000ADF85000E068002302788DF85820407895
:107C60008DF85900E06816AA4088ADF85A00E0681F
:107C700000798DF85C00E068C088ADF85D00CDF853
:107C80000090CDE901254FF4027214A806F044F8E3
:107C9000010003D00C9800F0C7FF28E670480321CC
:107CA0000838017156B100893080BDF82400708019
:107CB000BDF82000B080BDF81C00F080002016E662
:107CC00070B501258AB016460B46012802D002285D
:107CD00016D104E08DF80E504FF4205003E08DF8DB
:107CE0000E5042F60100ADF80C005BB10024601CA0
:107CF00060F30F2404AA08A918460CF0F1FB18B190
:107D0000072048E5102046E504A99DF820205448A6
:107D1000CDE90021801E02900023214603A802F233
:107D2000012205F0F9FF10B1FEF753FF33E54C488F
:107D300008380EB1C1883180057100202BE5F0B5FF
:107D400093B0074601268DF83E6041F60100ADF87C
:107D50003C0012AA0FA93046FFF7B2FF002848D115
:107D60003F4C0025083CE7B31C2102A81DF0F3FCA2
:107D70009DF808008DF83E6040F020008DF8080066
:107D800042F60520ADF83C000E959DF83A0011959D
:107D900020F00600801C8DF83A009DF838006A46F5
:107DA00020F0FF008DF838009DF8390009A920F077
:107DB000FF008DF839000420ADF82C00ADF830003C
:107DC0000EA80A9011A80D900FA80990ADF82E509A
:107DD00002A8FFF768FD00280BD1BDF80000608104
:107DE00000E008E0BDF80400A081401CE08125719E
:107DF000002013B0F0BD6581A581BDF84800F4E70F
:107E00002DE9F74F1649A0B00024083917940A79D4
:107E1000A146012A04D0022A02D0082023B02DE571
:107E2000CA88824201D00620F8E721988A46824219
:107E300001D10720F2E701202146ADF848004FF6B6
:107E4000FF788DF86E0042F6020B60F30F21ADF85B
:107E50004A80ADF86CB006918DF8724002E00000E7
:107E6000940200201CA9ADF870401391ADF8508029
:107E700012A806F03EF800252E462F460DAB07222D
:107E800012A9404606F038F878B10A285DD195B3BA
:107E90008EB3ADF86450ADF866609DF85E008DF865
:107EA000144019AC012864D06BE09DF83A001FB370
:107EB000012859D1BDF8381059451FD118A809A972
:107EC00001940294CDE9031007200090BDF836100C
:107ED00010230022404606F08FF8B0BBBDF86000CA
:107EE000042801D006284AD1BDF8241021988142E7
:107EF0003AD10F2092E73AE0012835D1BDF8380099
:107F0000B0F5205F03D042F6010188422CD1BAF8C7
:107F10000600BDF83610884201D1012700E0002795
:107F200005B19EB1219881421ED118A809AA0194D9
:107F30000294CDE90320072000900D461023002273
:107F4000404606F059F800B902E02DE04E460BE03D
:107F5000BDF86000022801D0102810D1C0B217AAC5
:107F600009A90CF09EFA50B9BDF8369086E70520B5
:107F700054E705A917A8221D0CF0B2FA08B1032096
:107F80004CE79DF814000023001DC2B28DF81420A8
:107F900022980092CDE901401BA8069905F0BCFE8D
:107FA00010B902228AF80420FEF713FE36E710B556
:107FB0000B46401E88B084B205AA00211846FEF781
:107FC000A8FE00200DF1080C06AA05A901908CE876
:107FD0000700072000900123002221464FF6FF7082
:107FE00005F0E0FD0446BDF81800012800D0FFDFD1
:107FF0002046FEF7EEFD08B010BDF0B5F74F044681
:1080000087B038790E46032804D0042802D008200F
:1080100007B0F0BD04AA03A92046FEF753FE0500F1
:10802000F6D160688078C0F3410002280AD19DF83B
:108030000D0010F0380F05D02069F9F788F908B164
:108040001020E5E7208905AA21698DE807006389EA
:10805000BDF810202068039905F05EFE10B1FEF710
:10806000B8FDD5E716B1BDF8140030800420387192
:108070002846CDE7F8B50C0006460CD001464FF671
:10808000FF7500236A46284606F038F828B100BF7D
:10809000FEF79FFDF8BD1020F8BD69462046FEF7AB
:1080A000C9FD0028F8D1A078314600F00103284628
:1080B000009A06F04FF8EBE730B587B0144600227F
:1080C0000DF1080C05AD01928CE82C0007220092FE
:1080D0000A46014623884FF6FF7005F063FDBDF8A0
:1080E00014102180FEF775FD07B030BD70B50D4648
:1080F00004210AF049FC040000D1FFDF294604F105
:108100001400BDE8704004F073BD70B50D46042145
:108110000AF03AFC040000D1FFDF294604F1140004
:10812000BDE8704004F087BD70B50D4604210AF02B
:108130002BFC040000D1FFDF294604F11400BDE848
:10814000704004F09FBD70B5054604210AF01CFC88
:10815000040000D1FFDF214628462368BDE87040B7
:108160000122FEF705BF70B5064604210AF00CFC9B
:10817000040000D1FFDF04F1140004F029FD401DCC
:1081800020F0030511E0011D00880022431821465C
:108190003046FEF7EDFE00280BD0607CABB26843A2
:1081A00082B2A068011D0AF0ACFAA06841880029DB
:1081B000E9D170BD70B5054604210AF0E5FB040065
:1081C00000D1FFDF214628466368BDE870400222E7
:1081D000FEF7CEBE70B50E46054601F079F90400F3
:1081E00000D1FFDF0120207266726580207820F0C8
:1081F0000F00001D20F0F00040302070BDE87040FE
:1082000001F069B910B50446012900D0FFDF20460E
:10821000BDE810400121FAF757B92DE9F04F97B0AA
:108220004FF0000A0C008346ADF814A0D04619D0D8
:10823000E06830B1A068A8B10188ADF81410A0F8CA
:1082400000A05846FBF7FFF8070043F2020961D08F
:10825000387822285CD3042158460AF095FB0500A3
:1082600005D103E0102017B0BDE8F08FFFDF05F166
:10827000140004F0ADFC401D20F00306A078012896
:1082800003D0022801D00720EDE7218807AA58462D
:1082900005F0FFFD30BB07A805F007FE10BB07A8DF
:1082A00005F003FE48B99DF82600012805D1BDF868
:1082B0002400A0F52451023902D04FF45050D2E7E7
:1082C000E068B0B1CDE902A00720009005AACDF882
:1082D00004A00492A2882188BDF81430584605F005
:1082E00061FC10B1FEF775FCBDE7A168BDF8140094
:1082F00008809DF81F00C00602D543F20140B2E796
:108300000B9838B1A1780078012905D080071AD4DC
:108310000820A8E74846A6E7C007F9D002208DF854
:108320003C00A8684FF00009A0B1697C4288714305
:1083300091420FD98AB2B3B2011D0AF098F9804672
:10834000A0F800A006E003208DF83C00D5F80080DE
:108350004FF001099DF8200010F0380F00D1FFDF29
:108360009DF820001E49C0F3C200084497F823106E
:1083700010F8010C884201D90F2074E72088ADF86D
:10838000400014A90095CDE90191434607220FA9A9
:108390005846FEF717FE002891D19DF8500050B9BD
:1083A000A078012807D1687CB3B2704382B2A86874
:1083B000011D0AF070F9002055E770B50646154614
:1083C0000C460846FEF7C4FB002805D12A46214684
:1083D0003046BDE8704073E470BD11E58C020020AA
:1083E0000E5B020070B51E4614460D0009D044B164
:1083F000616831B138B1FC49C988814203D0072096
:1084000070BD102070BD2068FEF7A2FB0028F9D1D6
:10841000324621462846BDE87040FFF744BA70B5A1
:1084200015460C0006D038B1EF490989814203D0C6
:10843000072070BD102070BD2068FEF789FB002862
:10844000F9D129462046BDE87040D6E570B506460C
:1084500086B00D4614461046F8F75BFFD0BB606847
:10846000F8F77EFFB0BBA6F57F40FF3803D030465B
:10847000FAF7E9FF80B128466946FEF79DFC00281F
:108480000CD19DF810100F2008293DD2DFE801F033
:1084900008060606060A0A0843F2020006B070BD86
:1084A0000320FBE79DF80210012908D1BDF8001058
:1084B000B1F5C05FF2D06FF4C052D142EED09DF85A
:1084C000061001290DD1BDF80410A1F52851062987
:1084D00007D200E029E0DFE801F00303040303030F
:1084E000DCE79DF80A1001290FD1BDF80810B1F59D
:1084F000245FD3D0A1F60211B1F50051CED00129ED
:10850000CCD0022901D1C9E7FFDF606878B9002328
:1085100005AA2946304605F0F1FD10B1FEF759FBDA
:10852000BCE79DF81400800601D41020B6E76188EE
:10853000224628466368FFF7BFFDAFE72DE9F04309
:10854000814687B0884614461046F8F7E2FE18B117
:10855000102007B0BDE8F083002306AA4146484634
:1085600005F0CCFD18B100BFFEF733FBF1E79DF835
:108570001800C00602D543F20140EAE700250727AC
:1085800005A8019500970295CDE9035062884FF642
:10859000FF734146484605F02FFD060013D1606881
:1085A000F8F7B7FE60B960680195CDE90250009711
:1085B0000495238862884146484605F01DFD06461D
:1085C000BDF8140020803046CEE739B1864B0A88CA
:1085D0009B899A4202D843F2030070471DE610B50A
:1085E00086B0814C0423ADF81430638943B1A4896B
:1085F0008C4201D2914205D943F2030006B010BD6E
:108600000620FBE7ADF81010002100910191ADF8B4
:10861000003002218DF8021005A9029104A90391EE
:10862000ADF812206946FFF7F8FDE7E72DE9FC47B2
:1086300081460D460846F8F746FE88BB4846FAF7DD
:1086400002FF5FEA00080AD098F80000222829D328
:10865000042148460AF098F9070005D103E043F2E7
:108660000200BDE8FC87FFDF07F1140004F0C7FA41
:1086700006462878012803D0022804D00720F0E716
:10868000B0070FD502E016F01C0F0BD0A8792C1DF7
:10869000C00709D0E08838B1A068F8F714FE18B117
:1086A0001020DEE70820DCE721882A780720B1F5D2
:1086B000847F35D01EDC40F20315A1F20313A942DA
:1086C00026D00EDCB1F5807FCBD003DCF9B10129D7
:1086D00026D1C6E7A1F58073013BC2D0012B1FD183
:1086E00013E0012BBDD0022B1AD0032BB9D0042BE1
:1086F00016D112E0A1F20912082A11D2DFE802F025
:108700000B04041010101004ABE7022AA9D007E0F4
:10871000012AA6D004E0320700E0F206002AA0DA1F
:10872000CDB200F0D5FE50B198F82300CDE9000598
:10873000FA89234639464846FEF78FFC91E7112017
:108740008FE72DE9F04F8BB01F4615460C46834648
:108750000026FAF778FE28B10078222805D20820F2
:108760000BB081E543F20200FAE7B80801D0072018
:10877000F6E7032F00D100274FF6FF79CCB1022D89
:1087800073D32046F8F7ECFD30B904EB0508A8F1E7
:108790000100F8F7E5FD08B11020E1E7AD1EAAB22F
:1087A0002146484605F085FD38F8021C88425CD118
:1087B000ADB20D49B80702D58889401C00E0012000
:1087C0001FFA80F8F80701D08F8900E04F4605AA0C
:1087D0004146584605F05DFB4FF0070A4FF000098F
:1087E000DCB320460BE000008C02002040881028FB
:1087F0003BD8361D304486B2AE4236D2A01902882C
:108800004245F3D351E000BF9DF8170002074CD555
:1088100094B304EB0608361DB8F80230B6B2102B3C
:1088200023D89A19AA4220D8B8F8002091421CD126
:10883000C0061CD5CDE900A90DF1080C0AAAA119A2
:1088400048468CE80700B8F800100022584605F0AA
:10885000A9F920B1FEF7BDF982E726E005E0B8F8F6
:108860000200BDF82810884201D00B2078E7B8F844
:108870000200304486B207E0FFE7C00604D5584640
:10888000FEF71DFC002888D19DF81700BDF81A10CE
:1088900020F010008DF81700BDF81700ADF80000AB
:1088A000FF235846009A05F055FC05A805F0FDFA8F
:1088B00018B9BDF81A10B942A6D9042158460AF0D1
:1088C00063F8040000D1FFDFA2895AB1CDE900A905
:1088D0004D46002321465846FEF7BFFB0028BBD17A
:1088E000A5813DE700203BE72DE9FF4F8BB01E46F9
:1088F00017000D464FF0000412D0B00802D0072038
:108900000FB0B1E4032E00D100265DB10846F8F7A0
:108910001EFD28B93888691E0844F8F718FD08B10B
:108920001020EDE7C64AB00701D5D18900E001214A
:10893000F0074FF6FF7802D0D089401E00E0404695
:1089400086B206AA0B9805F0A4FA4FF000094FF082
:10895000070B0DF1140A38E09DF81B00000734D511
:10896000CDF80490CDF800B0CDF80890CDE9039A89
:10897000434600220B9805F03FFB60BB05B3BDF8F2
:1089800014103A8821442819091D8A4230D3BDF8B1
:108990001E2020F8022BBDF8142020F8022BCDE970
:1089A00000B9CDE90290CDF810A0BDF81E10BDF8B9
:1089B000143000220B9805F01FFB08B103209FE73D
:1089C000BDF814002044001D84B206A805F06DFA1D
:1089D00020B10A2806D0FEF7FCF891E7BDF81E107A
:1089E000B142B9D934B17DB13888A11C884203D2D3
:1089F0000C2085E7052083E722462946404605F0FE
:108A000058FC014628190180A41C3C80002077E70F
:108A100010B50446F8F77DFC08B1102010BD884859
:108A2000C0892080002010BDF0B58BB00D460646F1
:108A3000142103A81CF08FFE01208DF80C008DF886
:108A4000100000208DF81100ADF814503046FAF7F0
:108A5000FAFC48B10078222812D30421304609F0EC
:108A600093FF040005D103E043F202000BB0F0BD18
:108A7000FFDF04F11400074604F0C1F8800601D4BA
:108A80000820F3E7207C022140F00100207409A8AF
:108A90000094CDE90110072203A930466368FEF770
:108AA00091FA20B1217C21F001012174DEE72946F1
:108AB0003046F9F7FAFC08A9384604F08FF800B1FF
:108AC000FFDFBDF82040172C01D2172000E0204620
:108AD000A84201D92C4602E0172C00D217242146C7
:108AE0003046FFF712FB21463046F9F704FA002022
:108AF000BCE7F8B51C4615460E46069F0AF076F808
:108B00002346FF1DBCB231462A46009409F061FCA1
:108B1000F8BD70B50C4605460E2120461CF0F9FD47
:108B2000002020802DB1012D01D0FFDF70BD062077
:108B300000E00520A07170BD10B54880087813468C
:108B400020F00F00001D20F0F00080300C4608706F
:108B50001422194604F108001CF0A1FD00F0BBFC32
:108B60003748046010BD2DE9F047DFF8D890491D63
:108B7000064621F0030117460C46D9F8000009F01B
:108B80003EFD050000D1FFDF4FF000083560A5F87D
:108B900000802146D9F8000009F031FD050000D120
:108BA000FFDF7560A5F800807FB104FB07F1091DA8
:108BB0000BD0D9F8000009F022FD040000D1FFDF3E
:108BC000B460C4F80080BDE8F087C6F80880FAE712
:108BD0002DE9F0411746491D21F00302194D0646C3
:108BE00001681446286809F035FD22467168286836
:108BF00009F030FD3FB104FB07F2121D03D0B1684C
:108C0000286809F027FD042009F066FE04460420C8
:108C100009F06AFE201A012804D12868BDE8F04155
:108C200009F0E2BCBDE8F08110B50C4605F0FDF896
:108C300000B1FFDF2046BDE81040FDF7CABF0000CD
:108C40008C0200201400002038B50C468288817BFD
:108C500019B14189914200D90A462280C188121D6A
:108C600090B26A4608F02BFFBDF80000032800D33D
:108C70000320C1B2208800F0D7FF38BD38B50C46BC
:108C80008288817B19B10189914200D90A462280EC
:108C9000C188121D90B26A4608F011FFBDF80000AD
:108CA000022800D30220C1B2208800F0BDFF401C82
:108CB000C0B238BD2DE9FE4F82468B46F9481446B6
:108CC0000BF10302D0E90010CDE9011022F00302FC
:108CD00068464FF49071009209F073FCF24E002C3C
:108CE00002D1F24A00999160009901440091357FC8
:108CF00005F1010504D1E8B20BF06CFB00B1FFDF18
:108D0000009800EB0510C01C20F0030100915CB935
:108D1000707AB27A1044C2B200200870308C80B2EF
:108D200004F00BFF00B1FFDF0098316A08440090A7
:108D30002146684600F03BFF80460098C01C20F0AA
:108D400003000090B37AF27A717A04B1002009F03E
:108D50002EFD0099084400902146684600F06FFF00
:108D6000D14800273D4690F801900CE0284600F0DD
:108D700001FF064681788088F9F754F971786D1CF7
:108D800000FB0177EDB24D45F0D10098C01C20F0FA
:108D90000300009004B100203946F9F74EF900991C
:108DA000002708440090C0483D4690F801900CE030
:108DB000284600F0DFFE0646C1788088FEF709FCF1
:108DC00071786D1C00FB0177EDB24D45F0D1009834
:108DD000C01C20F00300009004B100203946FEF7CB
:108DE00001FC00994FF0000908440090AE484D4640
:108DF00047780EE0284600F0BDFE0646807B30B185
:108E000006F1080001F00FFF727800FB02996D1C5B
:108E1000EDB2BD42EED10098C01C20F003000090DE
:108E200004B10020494601F002FF00990844009077
:108E30002146684600F075FE0098C01D20F007002E
:108E40000090DAF80010814204D3A0EB0B01B1F5D9
:108E5000803F04DB4FF00408CAF8000004E0CAF8C1
:108E60000000B8F1000F02D04046BDE8FE8F34BBD1
:108E70008F490020009A03F079F8FBF764FA8A48DA
:108E800001AA00211030F8F7E9FA00B1FFDF8648A7
:108E9000407FFEF754FF00B1FFDF83484FF4F671C7
:108EA00040301CF058FC80480421403080F8E91123
:108EB00080F8EA11062180F8EB11032101710020EE
:108EC000D3E770B5784C06464034207804EB401563
:108ED000E078083590B9A01990F8E80100280ED084
:108EE000A0780F2800D3FFDF202128461CF033FC98
:108EF000687866F3020068700120E070284670BD53
:108F00002DE9F04105460C460027007805219046E2
:108F10003E46B1EB101F00D0FFDF287A50B1012888
:108F20000ED0FFDFA8F800600CB12780668000201B
:108F3000BDE8F0810127092674B16888A08008E0A7
:108F40000227142644B16888A0802869E060A88AB6
:108F50002082287B2072E5E7A8F80060E7E730B5BB
:108F6000514C012000212070617020726072032238
:108F7000A272E07221732174052121831F21618374
:108F800060744CA161610A2121776077474D4FF4ED
:108F9000B06020626868C11C21F00301814200D0EA
:108FA000FFDF6868606030BD30B5404C15686368AD
:108FB00010339D4202D20420136030BD3A4B5D78DD
:108FC0005A6802EB0512107051700320D0801720F0
:108FD00090800120D0709070002090735878401CD1
:108FE0005870606810306060002030BD70B5064673
:108FF0002D480024457807E0204600F0BBFD0178AD
:10900000B14204D0641CE4B2AC42F5D1002070BD82
:10901000F7B5074608780C4610B3FFF7E7FF05469B
:10902000A7F12006202F06D0052E19D2DFE806F082
:109030000F2B2B151A0000F0A8FD0DB1697800E088
:109040000021401AA17880B20844FF2808D8A078EF
:1090500030B1A088022831D202E0608817282DD2D2
:109060000720FEBD207AE0B161881729F8D3A188D6
:109070001729F5D3A1790029F2D0E1790029EFD0A1
:10908000402804D9ECE7242F18D1207A48B1618810
:109090004FF6FB70814202D8A18881420ED904208C
:1090A000FEBD0BE0145B0200A803002018000020A6
:1090B000000000206E5246357800000065B9207827
:1090C00002AA0121FFF770FF0028E9D12078FFF7FD
:1090D0008DFF050000D1FFDF052E18D2DFE806F076
:1090E000030B0E081100A0786870A088E8800FE0DC
:1090F0006088A8800CE0A078A87009E0A078E870EB
:1091000006E054F8020FA8606068E86000E0FFDF46
:109110000020C5E71A2835D00DDC132832D2DFE84D
:1091200000F01B31203131272723252D3131293102
:109130003131312F0F00302802D003DC1E2821D11D
:10914000072070473A3809281CD2DFE800F0151BC9
:109150000F1B1B1B1B1B07000020704743F2040062
:10916000704743F202007047042070470D2070479B
:109170000F20704708207047112070471320704758
:10918000062070470320704710B5007800F00100FA
:1091900008F087FCBDE81040BCE710B5007800F08F
:1091A000010008F087FCBDE81040B3E70EB5017878
:1091B00001F001018DF80010417801F001018DF8F6
:1091C00001100178C1F340018DF802104178C1F31C
:1091D00040018DF80310017889088DF8041041785A
:1091E00089088DF8051081788DF80610C1788DF802
:1091F000071000798DF80800684607F097FAFFF726
:1092000089FF0EBD2DE9F84FDFF8F883FE4C0026EC
:109210004FF490771FE0012000F054FD0120FFF78C
:1092200050FE05463946D8F8080009F0E8F96860AC
:1092300000B9FFDF686807F008F9B0B12846FAF70F
:10924000E9FB284600F044FD28B93A466968D8F899
:10925000080009F0FFF994F9E9010428DBDA02209B
:1092600009F03AFB07460025A5E03A466968D8F8B8
:10927000080009F0EFF9F2E7B8F802104046491C7F
:1092800089B2A8F80210B94201D30021418002211D
:10929000B8F8020009F078FB002864D0B8F80200A2
:1092A000694608F070FBFFF735FF00B1FFDF9DF85E
:1092B000000078B1B8F8020009F0AAFC5FEA0009E2
:1092C00000D1FFDF484608F018FF18B1B8F80200D7
:1092D00002F054F9B8F8020009F088FC5FEA0009CE
:1092E00000D1FFDF484608F000FFE0BB0321B8F8DB
:1092F000020009F049FB5FEA000B47D1FFDF45E0C0
:10930000DBF8100010B10078FF2849D0022000F0EF
:10931000D9FC0220FFF7D5FD8246484608F0F1FF50
:10932000CAF8040000B9FFDFDAF8040009F0B9F860
:10933000002100900170B8F802105046AAF80210FF
:1093400001F01EFE484609F0AEF800B9FFDF5046B6
:1093500000F0BEFC18B99AF80100000704D5009887
:10936000CBF8100012E024E0DBF8100038B10178EF
:10937000491C11F0FF01017008D1FFDF06E0002257
:109380001146484600F0CBFB00B9FFDF94F9EA0133
:10939000022805DBB8F8020001F0B7FD0028AFD1C4
:1093A00094F9E901042804DB484609F0E0F800B12B
:1093B00001266D1CEDB2BD4204D294F9EA010228E7
:1093C000BFF65AAF002E7FF422AFBDE8F84F03205E
:1093D00000F078BC10B58B4CE06008682061AFF2FB
:1093E000DB10F9F77AFD607010BD87480021403826
:1093F00001708448017085494160704770B5054629
:109400004FF080500C46D0F8A410491C05D1D0F87C
:10941000A810C9430904090C0BD050F8A01F01F093
:1094200001012970416821608068A080287830B9E6
:1094300070BD062120460CF0E2FC01202870607906
:1094400040F0C000607170BD70B54FF080540D46A3
:10945000D4F88010491C0BD1D4F88410491C07D1D2
:10946000D4F88810491C03D1D4F88C10491C0CD0B6
:10947000D4F880100160D4F884104160D4F88810CA
:109480008160D4F88C10C16002E010210CF0B7FCB0
:10949000D4F89000401C0BD1D4F89400401C07D1A4
:1094A000D4F89800401C03D1D4F89C00401C09D08B
:1094B00054F8900F286060686860A068A860E06851
:1094C000E86070BD2846BDE8704010210CF097BCE4
:1094D0004D480079F5E470B54B4CE07830B3207816
:1094E00004EB4010407A00F00700204490F9E801B6
:1094F000002800DCFFDF2078002504EB4010407AD4
:1095000000F00700011991F8E801401E81F8E80118
:109510002078401CC0B220700F2800D12570A078A0
:10952000401CA0700CF062FBE57070BDFFDF70BDE9
:109530003EB50546032109F027FA0446284609F0FE
:1095400055FB054604B9FFDF206918B10078FF28F4
:1095500000D1FFDF01AA6946284600F0E0FA60B9B1
:10956000FFDF0AE0002202A9284600F0D8FA00B97D
:10957000FFDF9DF8080000B1FFDF9DF80000411EED
:109580008DF80010EED220690199884201D10020A7
:1095900020613EBD70B50546A0F57F400C46FF3802
:1095A00000D1FFDF012C01D0FFDF70BDFFF790FF7E
:1095B000040000D1FFDF207820F00F00401D20F0D4
:1095C000F000503020706580002020720120207350
:1095D000BDE870407FE72DE9F04116460D4607468D
:1095E000FFF776FF040000D1FFDF207820F00F00A6
:1095F000401D20F0F0005030207067800120207264
:10960000286805E018000020E8030020F813002077
:109610002061A888A0822673BDE8F0415BE77FB592
:10962000FFF7E4FC040000D1FFDF02A92046FFF7AA
:109630000BFB054603A92046FFF720FB8DF80050E1
:109640008DF80100BDF80800001DADF80200BDF85E
:109650000C00001DADF80400E088ADF80600684677
:1096600008F007FA002800D0FFDF7FBD2DE9F041A8
:10967000FB4C0646207808B1082059E43046F7F73D
:1096800048FE08B1102053E4F64D287808B9FFF7DA
:1096900066FCA87A697A0844C7B200F076FAB84244
:1096A00007D2381AC1B232460020FFF77DFC0028ED
:1096B000E3D16068C01C20F00300606000F05DFB37
:1096C000616801220844804601463046FFF7F2FAFD
:1096D000070012D00020FFF789FC06000BD006F12E
:1096E0001300616820F00300884200D0FFDF687833
:1096F000401E6870666038461AE4002241463046D3
:10970000FFF7D8FA00B1FFDF306860604FF6FF70F6
:1097100060800120207000200AE42DE9F041044619
:10972000CF4817460E46007808B10820A5E708463E
:10973000F7F7C9FD08B110209FE7CA4D287808B98E
:10974000FFF70DFC601E1E2807D8012C22D13078AF
:10975000FE281FD8287700208FE7A4F120001F28BB
:1097600005D8E0B23A463146BDE8F04150E4A4F1F4
:1097700040001F2805D831462046BDE8F04100F0E2
:10978000CFBAA4F1A0001F2804D80020A02C03D039
:10979000A12C06D0072070E7317801F0010169772C
:1097A0006BE731680922F82901D38B0701D01046F5
:1097B00063E76B7C03F00303012B04D16B8BD7337E
:1097C0009CB28C42F3D8296257E72DE9F0478146D5
:1097D0000E460846F7F79DFD48B94846F7F7B7FD2E
:1097E00028B909F1030020F00301494502D01020F7
:1097F000BDE8F0879B484FF0000A4030817869B19E
:109800004178804600EB4114083437883246002105
:10981000204600F06BFA050004D027E0A6F800A06F
:109820000520E5E7B9F1000F24D03088B84201D90E
:109830000C251FE0607800F00705284600F042FA8A
:1098400008EB0507324697F8E8014946401C87F8BF
:10985000E801204607F5F47700F048FA0546387825
:10986000401E3870032000F02DFA2DB10C2D01D0D0
:10987000A6F800A02846BBE76078794E00F0070103
:10988000012923D002290CD0032934D0FFDF98F816
:1098900001104046491CC9B288F801100F2935D083
:1098A00036E0616821B1000702D46088FFF740FE0E
:1098B00098F8EA014746012802D17078F9F72CFBA5
:1098C00097F9EA010428E2DBFFDFE0E7616821B1F4
:1098D0004FF49072B06808F0BDFE98F8E901474671
:1098E000032802D17078F9F717FB97F9E9010428EA
:1098F000CDDBFFDFCBE7C00602D56088FFF718FE9F
:1099000098F9EB010628C2DBFFDFC0E780F801A071
:109910008178491E8170617801F0070101EB080030
:1099200090F8E811491C80F8E811A3E770B50D46DE
:109930000446F7F7C8FC18B92846F7F7EAFC08B15F
:10994000102070BD29462046BDE870400AF079BD60
:1099500070B505460AF098FDC4B22846F7F7F7FC43
:1099600008B1102070BD35B128782C7018B1A04214
:1099700001D0072070BD2046FDF796FE052805D1D1
:109980000AF086FD012801D0002070BD0F2070BDB7
:1099900070B5044615460E460846F7F794FC18B90C
:1099A0002846F7F7B6FC08B1102070BD022C03D092
:1099B000102C01D0092070BD2A46314620460AF0FD
:1099C00070FD0028F7D0052070BD70B514460D4617
:1099D0000646F7F778FC38B92846F7F79AFC18B925
:1099E0002046F7F7B4FC08B1102070BD2246294686
:1099F00030460AF075FD0028F7D0072070BD3EB54F
:109A00000446F7F786FC08B110203EBD684606F014
:109A1000F4FDFFF77FFB0028F7D19DF806002070CA
:109A2000BDF808006080BDF80A00A08000203EBD9F
:109A300070B505460C460846F7F789FC20B93CB1DD
:109A40002068F7F766FC08B1102070BDA08828B127
:109A500021462846BDE87040FDF77EBE092070BD56
:109A600018000020A803002070B504460D460846E3
:109A7000F7F729FC30B9601E1E2814D82846F7F7DE
:109A800022FC08B11020EAE7032C01D90720E6E701
:109A900004B9FFDFFC4800EB840050F8041C2846A2
:109AA000BDE870400847A4F120001F2805D82946CA
:109AB0002046BDE87040FAF7CEBBF02CE6D1A8688E
:109AC000F7F701FC0028DDD1284608F03AF8BDE898
:109AD0007040FFF71FBB70B504460D460846F7F708
:109AE00018FC30B9601E1E280FD82846F7F7EBFB8C
:109AF00008B11020B3E7012C03D0022C01D0032CB5
:109B000001D10620ABE70720A9E7A4F120001F2818
:109B1000F9D829462046BDE87040FAF7F4BB08F0B2
:109B2000B3BA38B50446D948007B00F00105D9B96D
:109B300004F064FB0DB1226800E00022D4484178B3
:109B4000C06806F048FCD2481030C0788DF800009C
:109B500010B1012802D004E0012000E000208DF8BF
:109B60000000684606F0C3FD002D02D020682830B2
:109B7000206038BD30B5C54D04466878A04200D895
:109B8000FFDF686800EB041030BD70B5BF480025EA
:109B90002C46467807E02046FFF7ECFF4078641C2F
:109BA0002844C5B2E4B2B442F5D1284657E72DE9BE
:109BB000F0410C4607464FF0000800F00CF906464D
:109BC000FF2801D94FF013083868C01C20F00302A9
:109BD0003A6054EA080421D1AC48F3B2072124309A
:109BE0000CF012FB09E0072C10D2DFE804F00604A9
:109BF00008080A040600A74804E0A74802E0A748AE
:109C000000E0A7480CF020FB054600E0FFDFA5427E
:109C100000D0FFDF641CE4B2072CE4D3386800EB0B
:109C200006103860404628E5021D5143452900D200
:109C300045210844C01CB0FBF2F0C0B270472DE9CA
:109C4000FC5F064691484FF000088B464746444665
:109C500090F8019022E02046FFF78CFF050000D12C
:109C6000FFDF687869463844C7B22846FEF7ECFF44
:109C7000824601A92846FFF701F80346BDF8040013
:109C80005246001D81B2BDF80000001D80B208F0F0
:109C9000F9FE6A78641C00FB0288E4B24C45DAD114
:109CA0003068C01C20F003003060BBF1000F00D012
:109CB00000204246394608F0F3FE3168084430601F
:109CC000BDE8FC9F7149403108710020C8707047A1
:109CD0006E494031CA782AB10A7801EB4211083145
:109CE000814201D001207047002070472DE9F041EA
:109CF00006460078154600F00F0400201080601E14
:109D00000F46052800D3FFDF5F482A46183800EBCE
:109D10008400394650F8043C3046BDE8F04118470D
:109D200070B50C46402802D0412806D120E0A0782A
:109D300061780D18E178814201D907208FE62078FB
:109D4000012801D913208AE6FF2D08D80AF032FD38
:109D500006460BF003FF301A801EA84201DA1220DB
:109D60007DE64A482168816021790173002076E60A
:109D7000BDE87040084600F059B82DE9F0470027CB
:109D8000DFF808A13E463D46B9463C469AF80180B8
:109D90000AE02046FFF7EEFE4178807B0E4410FB80
:109DA0000155641CE4B27F1C4445F2D109EB8700E5
:109DB000C6EBC60100EB81009AF8092000EB850193
:109DC00001EBC2019AF80A209AF80B0001EBC201DC
:109DD00001EB80000CE52DE9F047DFF8B09000269C
:109DE000344699F8090099F80A2099F8017002445C
:109DF000D5B299F80B20104400F0FF0808E0204687
:109E0000FFF7B8FE817B407811FB0066641CE4B26A
:109E1000BC42F4D199F8091099F80A002944294460
:109E2000414400B1012008443044E1E438B504461F
:109E3000407800F00300012803D002280BD007204F
:109E400038BD606858B1F7F78BFAD0B96068F7F79A
:109E50007EFA20B915E06068F7F735FA88B96946E7
:109E60002046FCF79DF80028EAD1607800F0030056
:109E7000022817D19DF80000A0B16068F7F767FAD3
:109E800080B1102038BD0000345B0200A803002020
:109E90001800002057410000FBAC0000E92F000033
:109EA000C74101006189F8290DD8208988420AD864
:109EB000607800F003020A48012A06D1D731026A0D
:109EC00089B28A4201D20920DCE794E80E0000F151
:109ED000100585E80E000AB9002101830020D1E7B2
:109EE000A80300202DE9F04107461446884608469D
:109EF00001F022FD064608EB88001C22796802EB7F
:109F0000C0000D18688C58B14146384601F01CFD60
:109F1000014678680078C200082305F120000CE0B3
:109F2000E88CA8B14146384601F015FD0146786835
:109F300008234078C20005F1240008F0E2FB38B1A4
:109F4000062121726681D0E90010C4E9031009E0FE
:109F5000287809280BD00520207266816868E060A7
:109F6000002028702046BDE8F04101F0DBBC07204E
:109F700020726681F4E72DE9F04116460D4607464A
:109F8000406801EB85011C2202EBC1014418204608
:109F900001F003FD40B10021708865F30F2160F3EB
:109FA0001F4106200CF00AFA09202070324629468B
:109FB0003846BDE8F04195E72DE9F0410E460746E9
:109FC00000241C21F07816E004EB8403726801EB96
:109FD000C303D25C6AB1FFF77BFA050000D1FFDF53
:109FE0006F802A4621463046FFF7C5FF0120BDE8B5
:109FF000F081641CE4B2A042E6D80020F7E770B517
:10A00000064600241C21C0780AE000BF04EB84034C
:10A01000726801EBC303D5182A782AB1641CE4B234
:10A02000A042F3D8402070BD282128461BF071FBC8
:10A03000706880892881204670BD70B50346002075
:10A040001C25DC780DE000BF00EB80065A6805EBAC
:10A05000C6063244167816B1128A8A4204D0401CD1
:10A06000C0B28442F0D8402070BDF0B50446002054
:10A070001C26E5780EE000BF00EB8007636806EB66
:10A08000C7073B441F788F4202D15B78934204D0CC
:10A09000401CC0B28542EFD84020F0BD00780328B4
:10A0A00001D000207047012070470078022801D0BD
:10A0B00000207047012070470078072801D0002059
:10A0C0007047012070472DE9F04106468846107818
:10A0D000F1781546884200D3FFDF2C781C27641CDA
:10A0E000F078E4B2A04201D8201AC4B204EB840193
:10A0F000706807EBC1010844017821B141468847E7
:10A1000008B12C7073E72878A042E8D1402028706D
:10A110006DE770B514460B880122A240134207D1A7
:10A1200013430B8001230A22011D08F0B4FA0470C6
:10A1300070BD2DE9FF4F81B00878DDE90E7B9A46AE
:10A1400091460E4640072CD4019808F061FD0400AA
:10A1500000D1FFDF07F1040820461FFA88F107F05D
:10A16000A0FE050000D1FFDF204629466A4608F020
:10A17000EAF80098A0F80370A0F805A0284608F0B7
:10A1800090F9017869F306016BF3C711017020465D
:10A190001FFA88F107F0C8FE00B9FFDF019806F04A
:10A1A0008CF806EB0900017F491C017705B0BDE87A
:10A1B000F08F2DE9F84F0E469A4691460746032147
:10A1C00008F0E2FB0446008DDFF8B885002518B1E1
:10A1D00098F80000B0421ED1384608F019FD07007B
:10A1E00000D1FFDF09F10401384689B207F059FEBA
:10A1F000050010D0384629466A4608F0A4F80098B1
:10A2000000210A460180817006F010F90098C01DF7
:10A21000CAF8000021E098F80000B04216D104F11D
:10A22000260734F8341F012000FA06F911EA090F55
:10A2300000D0FFDF2088012340EA090020800A22A5
:10A24000391D384608F042FA067006E0324604F13D
:10A25000340104F12600FFF75CFF0A2188F80010A2
:10A260002846BDE8F88FFEB515460C46064602ABFB
:10A270000C220621FFF79DFF002827D00299607865
:10A2800012220A70801C487008224A80A07002982E
:10A290002988052381806988C180A9880181E9888E
:10A2A000418100250C20CDE90005062221463046DB
:10A2B000FFF73FFF2946002266F31F41F0231046B7
:10A2C0000BF0D2FF6078801C60700120FEBDFEB5EF
:10A2D00014460D460622064602AB1146FFF769FFFB
:10A2E000002812D0029B132000211870A878587003
:10A2F000022058809C800620CDE9000102460523FB
:10A3000029463046FFF715FF0120FEBD2DE9FE432B
:10A310000C46804644E002AB0E2207214046FFF780
:10A3200048FF002841D060681C2267788678BF1CEF
:10A3300006EB860102EBC101451802981421017059
:10A3400047700A214180698A0181E98A4181A9888F
:10A350008180A9898181304601F0EEFA02990523B6
:10A360000722C8806F700420287000250E20CDE9D8
:10A37000000521464046FFF7DCFE294666F30F2123
:10A3800068F31F41F023002206200BF06DFF607878
:10A39000FD49801C607062682046921CFFF793FEA6
:10A3A000606880784028B6D10120BDE8FE83FEB504
:10A3B0000D46064638E002AB0E2207213046FFF775
:10A3C000F8FE002835D068681C23C17801EB8102B3
:10A3D00003EBC20284180298152202706278427060
:10A3E0000A224280A2894281A2888281084601F025
:10A3F000A3FA014602988180618AC180E18A0181C5
:10A40000A088B8B10020207000210E20CDE9000105
:10A410000523072229463046FFF78BFE6A68DB4991
:10A420002846D21CFFF74FFE6868C0784028C2D18A
:10A430000120FEBD0620E6E72DE9FE430C468146DD
:10A4400044E0204601F093FAD0B302AB0822072182
:10A450004846FFF7AEFE0028A7D060681C2265784A
:10A460000679AD1C06EB860102EBC1014718029884
:10A47000B7F81080062101704570042141803046F4
:10A4800001F05AFA0146029805230722C180A0F87C
:10A4900004807D70082038700025CDE90005214634
:10A4A0004846FFF746FE294666F30F2169F31F4130
:10A4B000F023002206200BF0D7FE6078801C60702D
:10A4C0006268B3492046121DFFF7FDFD60680179FF
:10A4D0004029B6D1012068E72DE9F34F83B00E463D
:10A4E00080E0304601F043FA002875D071681C20E6
:10A4F00091F8068008EB880200EBC2000C18414678
:10A50000304601F028FA0146A078C3007068407810
:10A51000C20004F1240008F010F907468088E18B9E
:10A52000401A80B2002581B3AA46218B814200D80F
:10A5300008468146024602AB07210398FFF739FE21
:10A54000010028D0BAF1000F03D0029AB888022582
:10A5500010808B46E28B3968A9EB05001FFA80FA60
:10A560000A440398009208F053FBED1D009A5946E7
:10A570005346009507F061FFE08B504480B2E083C2
:10A58000B988884209D1012508E0FFE7801C4FF017
:10A59000010A80B2C9E7002008E60025CDE9009550
:10A5A000238A072231460398FFF7C3FDE089401E46
:10A5B000E0818DB1A078401CA0707068F17842787D
:10A5C00011FB02F1CAB2816901230E3008F063F871
:10A5D00080F800800020E08372686E493046921D4A
:10A5E000FFF771FD7068817940297FF47AAF01200F
:10A5F000DCE570B5064648680D4614468179402969
:10A6000010D104EB84011C2202EBC101084401F0CB
:10A61000E5F9002806D06868294684713046BDE80F
:10A62000704059E770BDFEB50C460746002645E070
:10A63000204601F09CF9D8B360681C22417901EBF7
:10A64000810102EBC1014518688900B9FFDF02AB47
:10A65000082207213846FFF7ACFD002833D00299C5
:10A66000607816220A70801C487004204880606858
:10A67000407901F061F901460298052307228180A3
:10A680006989C1800820CDE9000621463846FFF7D8
:10A6900050FD6078801C6070A88969890844B0F515
:10A6A000803F00D3FFDFA88969890844A8816E81B3
:10A6B000626839492046521DFFF705FD60684179FF
:10A6C0004029B5D10120FEBD30B5438C458BC3F385
:10A6D000C704002345B1838B641EED1AC38A6D1E27
:10A6E0001D4495FBF3F3E4B22CB1008918B1A042EC
:10A6F00000D8204603444FF6FF70834200D3034640
:10A7000013800C7030BD2DE9FC41074616460D46FE
:10A71000486802EB86011C2202EBC10144186A461C
:10A7200001A92046FFF7D0FFA089618901448AB2C0
:10A73000BDF80010914212D0081A00D500206081A7
:10A740006868407940280AD1204601F03DF9002888
:10A7500005D06868294646713846FFF764FFBDE8B2
:10A76000FC812DE9FE4F894680461546508803211D
:10A7700008F00AF98346B8F8020040280ED24020BB
:10A780000DE000002C0000209DA00000ABA0000008
:10A79000B9A00000DDB90000C9B90000403880B29E
:10A7A00082460146584601F0E2F800287ED00AEBC6
:10A7B0008A001C22DBF8041002EBC0000C182046B3
:10A7C00001F0EBF8002877D1B8F80000E18A884260
:10A7D0003CD8A189D1B348456ED100265146584690
:10A7E00001F0B2F8218C0F18608B48B9B9F1020F53
:10A7F00062D3B8F804006083618A884226D80226B2
:10A80000A9EB06001FFA80F9B888A28B801A0028ED
:10A8100014DD4946814500DA084683B268886968D4
:10A82000029139680A44CDE9003208F0DFF9DDE928
:10A830000121F61D009B009607F0CBFDA18B01EBDB
:10A84000090080B2A083618B884207D9688803B071
:10A8500052465946BDE8F04F01F0DDB81FD14FF028
:10A8600009002872B8F802006881D7E90001C5E93B
:10A870000401608BA881284601F054F851465846DF
:10A8800001F062F80146DBF8040008230078C200FA
:10A8900004F1200007F035FF0020A0836083A08929
:10A8A0000AF0FF02401EA081688800E004E003B0C7
:10A8B0005946BDE8F04F26E7BDE8FE8F2DE9F0418F
:10A8C000064615460F461C461846F6F7FCFC18B916
:10A8D0002068F6F71EFD08B1102013E47168688C3B
:10A8E0000978B0EBC10F01D313200BE43946304691
:10A8F00001F02AF80146706808230078C20005F1CB
:10A90000200007F0C8FED4E90012C0E900120020C0
:10A91000E3E710B50446032108F036F80146007855
:10A9200000F00300022805D02046BDE8104001F1E8
:10A93000140298E48A8A2046BDE81040C7E470B546
:10A940000446032108F020F8054601462046FFF79B
:10A9500073FD002816D029462046FFF764FE002824
:10A9600010D029462046FFF722FD00280AD02946AC
:10A970002046FFF7CBFC002804D029462046BDE83E
:10A980007040A9E570BD2DE9F0410C4680461EE0FF
:10A99000E178427811FB02F1CAB2816901230E30DD
:10A9A00007F0AFFE077860681C22C179491EC171AB
:10A9B00007EB8701606802EBC10146183946204663
:10A9C00000F0D5FF18B1304600F0E0FF20B160681C
:10A9D000C1790029DCD180E7FEF77AFD050000D1BE
:10A9E000FFDF0A202872384600F0A6FF688139464A
:10A9F000204600F0B0FF0146606808234078C2009E
:10AA000006F1240007F07DFED0E90010C5E903102F
:10AA1000A5F80280284600F085FFB07800B9FFDF76
:10AA2000B078401EB07058E770B50C46054603215B
:10AA300007F0AAFF01464068C2792244C271284645
:10AA4000BDE870409FE72DE9FE4F824650781446DE
:10AA50000F464FF0000800284FD0012807D00228E9
:10AA600022D0FFDF2068B8606068F86024E702AB9E
:10AA70000E2208215046FFF79CFB0028F2D00298D6
:10AA8000152105230170217841700A214180C0F809
:10AA90000480C0F80880A0F80C80628882810E20B3
:10AAA000CDE90008082221E0A678304600F044FFF6
:10AAB000054606EB86012C22786802EBC1010822CC
:10AAC000465A02AB11465046FFF773FB0028C9D027
:10AAD00002980721017021784170042141800821EA
:10AAE0008580C680CDE9001805230A4639465046C0
:10AAF000FFF71FFB87F80880DEE6A678022516B16F
:10AB0000022E13D0FFDF2A1D914602AB08215046CA
:10AB1000FFF74FFB0028A5D002980121022E0170FB
:10AB2000217841704580868002D005E00625EAE75D
:10AB3000A188C180E1880181CDE900980523082220
:10AB400039465046D4E710B50446032107F01CFFF0
:10AB5000014600F108022046BDE8104073E72DE9E8
:10AB6000F05F0C4601281DD0957992F80480567943
:10AB700005EB85011F2202EBC10121F0030B08EB5D
:10AB8000060111FB05F14FF6FF7202EAC10909F156
:10AB9000030115FB0611F94F21F0031A40B10128FA
:10ABA0003DD124E06168E57891F800804E78DFE7D8
:10ABB0005946786807F023FD606000B9FFDF594609
:10ABC00060681AF0C8FDE5705146786807F017FD17
:10ABD0006168486100B9FFDF6068426902EB090102
:10ABE0008161606880F800806068467017E0606886
:10ABF00052464169786807F02DFD5A4661687868C9
:10AC000007F028FD032007F067FE0446032007F045
:10AC10006BFE201A012802D1786807F0E5FC0BEBE7
:10AC20000A00BDE8F09F02460021022097E773B5B5
:10AC3000D24D0A202870009848B100244FEA0D0038
:10AC400007F0BFFC002C01D1009969607CBD012494
:10AC50000020F5E770B50C461546382120461AF05D
:10AC60007AFD012666700A2104F11C001AF073FDBA
:10AC700005B9FFDF297A207861F301002070A879F7
:10AC8000002817D02A4621460020FFF768FF616898
:10AC9000402088706168C870616808716168487197
:10ACA000616888716168288808816168688848815E
:10ACB0006068868170BDC878002802D0002201201B
:10ACC0004DE7704770B50546002165F31F41002030
:10ACD0000BF074FB0321284607F056FE040000D158
:10ACE000FFDF21462846FFF767F9002804D02078C7
:10ACF00040F010002070012070BD2DE9FF4180461A
:10AD00000E460F0CFEF7E4FB050007D06F80032111
:10AD1000384607F039FE040008D106E004B0384692
:10AD2000BDE8F0411321F9F74BBEFFDF5FEA0800F1
:10AD300005D0B8F1060F18D0FFDFBDE8FF812078FD
:10AD40002A4620F0080020700020ADF80200022002
:10AD50008DF800004FF6FF70ADF80400ADF8060066
:10AD600069463846F9F723FAE7E7C6F3072101EB0E
:10AD700081021C23606803EBC202805C042803D0BC
:10AD800008280AD0FFDFD8E7012000904FF44043A5
:10AD90002A46204600F008FECFE704B02A462046A7
:10ADA000BDE8F041FFF7E7B82DE9F05F0027B0F804
:10ADB0000A9090460C4605463E46B9F1400F01D236
:10ADC000402001E0A9F140001FFA80FA287AC01E55
:10ADD00008286BD2DFE800F00D04192058363C47F4
:10ADE00072271026002C6CD0D5E90301C4E90201BA
:10ADF0005CE070271226002C63D00A2205F10C01BA
:10AE000004F108001AF04BFC50E071270C26002CCE
:10AE100057D0E868A06049E0742710269CB3D5E9B4
:10AE20000301C4E902016888032107F0ADFD8346F0
:10AE3000FEF74EFB02466888508051465846FFF7A1
:10AE400051F833E075270A26ECB1A88920812DE05E
:10AE500076271426BCB105F10C0004F1080307C8DD
:10AE600083E8070022E07727102664B1D5E90301C3
:10AE7000C4E902016888032107F086FD014668885D
:10AE8000FFF781FD12E01CE073270826CCB168882B
:10AE9000032107F079FD01460078C00606D56888D1
:10AEA000FFF78AF810B96888F8F798FDA8F80060ED
:10AEB0002CB12780A4F8069066806888A0800020C6
:10AEC000AFE6A8F80060FAE72DE9FC410C461E4603
:10AED00017468046032107F057FD05460A2C0AD283
:10AEE000DFE804F005050505050509090907042340
:10AEF00003E0062301E0FFDF0023CDE900762246D0
:10AF000029464046FFF715F929E438B50546A0F56E
:10AF10007F40FF3830D0284607F068FE040000D19B
:10AF2000FFDF204607F0EDF9002815D001466A46FC
:10AF3000204607F008FA00980321B0F8054028469B
:10AF400007F022FD0546052C03D0402C05D24024F5
:10AF500004E0007A80B1002038BD403CA4B2214614
:10AF600000F005FD40B1686804EB84013E2202EB6D
:10AF7000C101405A0028EFD0012038BD2C0000202C
:10AF80002DE9F04F054689B0408807F02FFE0400F8
:10AF900000D1FFDF06AA2046696800F0C1FC069CCC
:10AFA000001F34F8031F218063886380228881B2E8
:10AFB0008A4205D1042B0AD0052B1DD0062B15D0B3
:10AFC0002A462046FFF7CDFB09B0BDE8F08F1646B4
:10AFD000241D2A4621463046F7F751FA0828F3D1B6
:10AFE0002A4621463046FCF7FEFBEDE76888211D26
:10AFF0006B68FAF743FCE7E717466888032107F018
:10B00000C3FC4FF000088DF804800646ADF80680BA
:10B01000042FD9D36279002AD6D020794FF6FF7950
:10B020004FF01C0A13282CD008DC012878D0062801
:10B0300047D0072875D0122874D106E0142872D0A2
:10B04000152871D016286DD1ACE10C2F6AD130785B
:10B0500000F00301022965D140F0080030706079EA
:10B06000B07001208DF804002089ADF808006089D7
:10B07000ADF80A00A089ADF80C00E089ADF80E002B
:10B0800019E0B07890429FD1307801079CD5062F07
:10B090009AD120F0080030706888414660F31F4163
:10B0A00000200BF08BF902208DF80400ADF8089019
:10B0B0002089ADF80A0068882A4601A9F9F777F8CF
:10B0C00082E7082F80D12789B4F80A90402F01D257
:10B0D000402001E0A7F1400080B2804601463046A2
:10B0E00000F045FC08B3716808EB88002C2202EBE5
:10B0F000C000095A4945E3D1FE4807AAD0E9021029
:10B10000CDE9071060798DF81C0008F0FF048DF878
:10B110001E4068883146FFF796FC2A46214639E0F2
:10B12000B6E014E03CE039E0E6E0F248D0E9001097
:10B13000CDE907106079ADF820708DF81C00ADF8EE
:10B140002290688807AA3146FFF77DFC3CE7082F6C
:10B15000B6D16089B4F80880402801D2402000E0D0
:10B16000403887B23946304600F001FC0028A7D0AD
:10B1700007EB870271680AEBC2000844028A424565
:10B180009ED1017808299BD140786179884297D176
:10B19000F9B22A463046FEF7EEFE15E70E2F07D02D
:10B1A000CDF81C80CDF8208060798DF81C00C8E7B0
:10B1B0006189E7898B46B4F80C903046FEF73DFF75
:10B1C000ABF14001402901D309204AE0B9F1170F42
:10B1D00001D3172F01D20B2043E040280ED000EB03
:10B1E000800271680AEBC20008440178012903D18A
:10B1F000407861798842A9D00A2032E03046FEF7D3
:10B20000FEFE014640282BD001EB810372680AEB59
:10B21000C30002EB0008012288F80020627988F858
:10B220000120706822894089B84200D93846248AB2
:10B2300003232B72AA82EF812882A5F80C906C82DE
:10B24000084600F079FB6881A8F81490A8F81870F7
:10B25000A8F80E40A8F810B0284600F063FBB3E64B
:10B26000042005212972A5F80A80E88101212973AB
:10B27000A049D1E90421CDE9072161798DF81C109D
:10B28000ADF81E00688807AA3146FFF7DCFBE3E74C
:10B29000062FE4D3B078904215D13078010712D54B
:10B2A00020F0080030706888414660F31F4100209C
:10B2B0000BF084F802208DF804002089ADF8080016
:10B2C000ADF80A90F7E604213046FEF7CEFE0446BC
:10B2D0004028C4D00220830300902A4621463046ED
:10B2E00000F062FB4146688864F30F2160F31F4160
:10B2F00006200BF063F867E60E2FB0D1042130462C
:10B30000FEF7B3FE81464028A9D04146688869F31C
:10B310000F2160F31F4106200BF050F8208A0790A0
:10B32000E08900907068A7894089B84200D9384602
:10B330008346B4F80A8020890590484600F0FCFA5C
:10B340006881079840B10220079B00902A46494631
:10B35000304600F029FB37E6B8F1170F1ED3172F40
:10B360001CD30420287200986882EF81A5F810B0E1
:10B37000A5F80C8009EB89020AEBC2007168009AFB
:10B380000C180598A4F81480A4F818B0E281208263
:10B39000284600F0C7FA0620207015E601200B238E
:10B3A0000090D3E7082FA6D121893046FEF745FE4D
:10B3B000074640289FD007EB870271680AEBC2005E
:10B3C0000844804600F0E9FA002894D16489B8F86E
:10B3D0000E002044B0F5803F05D368883A463146D8
:10B3E00000F019FBF0E5002C85D0A8F80E00688865
:10B3F0003A463146FFF7FDF808202872384600F03B
:10B400009BFA6881AC8127E770B50D46064603219B
:10B4100007F0BAFA040004D02078000704D5112000
:10B4200070BD43F2020070BD2A4621463046FEF749
:10B430001AFF18B9286860616868A061207840F038
:10B4400008002070002070BD70B50D46064603212F
:10B4500007F09AFA040004D02078000704D40820EA
:10B4600070BD43F2020070BD2A4621463046FEF709
:10B470002EFF00B9A582207820F00800207000205F
:10B4800070BD2DE9F04F0E4691B08046032107F0C4
:10B490007BFA0446404607F0BBFB074600200790B6
:10B4A00008900990ADF830000A9002900390049043
:10B4B00004B9FFDF0DF108091FBBFFDF21E03846AB
:10B4C0000BA9002206F0E0FD9DF82C0000F07F059E
:10B4D0000A2D00D3FFDF6019017F491E01779DF817
:10B4E0002C0000060DD52A460CA907A8FEF711FE70
:10B4F00002E00000405B020019F80510491C09F841
:10B500000510761EF6B2DAD204F13400FA4D04F1D9
:10B51000260BDFF8E8A304F12A07069010E058464E
:10B52000069900F06AFA064628700A2800D3FFDF61
:10B530005AF8261040468847E08CC05DB04202D0E1
:10B54000208D0028EBD10A202870EC4D4E4628357E
:10B550000EE00CA907A800F050FA0446375D55F834
:10B56000240000B9FFDF55F82420394640469047B3
:10B57000BDF81E000028ECD111B026E510B503215E
:10B5800007F002FA040000D1FFDF0A2104F11C00D9
:10B590001AF0E1F8207840F00400207010BD10B5DA
:10B5A0000C46032107F0F0F92044007F002800D06A
:10B5B000012010BD2DE9F84F89461546824603212A
:10B5C00007F0E2F9070004D02846F5F77CFE40B901
:10B5D00003E043F20200BDE8F88F4846F5F799FE14
:10B5E00008B11020F7E7786828B16988008981429E
:10B5F00001D90920EFE7B9F800001C2418B1402850
:10B6000009D2402008E03846FEF7F9FC8046402881
:10B6100019D11320DFE7403880B280460146384612
:10B6200000F0A5F948B108EB8800796804EBC00088
:10B63000085C012803D00820CDE70520CBE7FDF703
:10B6400047FF06000BD008EB8800796804EBC000C8
:10B650000C18B9F8000020B1E88910B113E01120EE
:10B66000B9E72888172802D36888172801D207204D
:10B67000B1E7686838B12B1D224641463846FFF7CE
:10B680001DF90028A7D104F10C0269462046FFF7F6
:10B690001BF8288860826888E082B9F8000030B121
:10B6A00002202070E889A080E889A0B12BE0032067
:10B6B0002070A889A08078688178402905D180F819
:10B6C000028039465046FEF721FE404600F034F92C
:10B6D000A9F8000021E07868218B4089884200D9D0
:10B6E00008462083A6F802A004203072B9F80000B2
:10B6F0007081E0897082F181208B3082A08AB081D4
:10B70000304600F00FF97868C178402905D180F8FB
:10B71000038039465046FEF74AFE00205BE770B5CD
:10B720000D460646032107F02FF9040003D0402DF3
:10B7300004D2402503E043F2020070BD403DADB2AB
:10B74000294600F014F958B105EB85011C22606808
:10B7500002EBC101084400F020F918B1082070BDC7
:10B76000052070BD2A462146304600F054F90020DD
:10B7700070BD2DE9F0410D4616468046032107F0C5
:10B7800003F90446402D01D2402500E0403DADB212
:10B790008CB1294600F0EBF880B105EB85011C2245
:10B7A000606802EBC1014718384600F0F6F838B17E
:10B7B0000820BDE8F08143F20200FAE70520F8E72F
:10B7C00033463A4629462046FFF778F80028F0D15C
:10B7D000EAB221464046FEF796FF0020E9E72DE950
:10B7E000F0410D4616468046032107F0CDF8044689
:10B7F000402D01D2402500E0403DAFB224B130469B
:10B80000F5F761FD38B902E043F20200D1E7306894
:10B81000F5F759FD08B11020CBE73946204600F076
:10B82000A6F860B107EB87011C22606802EBC1013A
:10B830004518284600F0B1F818B10820B9E70520EE
:10B84000B7E7B088A98A884201D90C20B1E76168BE
:10B85000E88C4978B0EBC10F01D31320A9E7394632
:10B86000204600F078F80146606808234078C2005E
:10B8700005F1240006F00FFFD6E90012C0E900121E
:10B88000FAB221464046FEF7B4FE002091E72DE9CA
:10B89000F0470D461F4690468146032107F074F895
:10B8A0000446402D01D2402001E0A5F1400086B2BF
:10B8B0003CB14DB13846F5F74AFD50B11020BDE816
:10B8C000F08743F20200FAE76068C8B1A0F80C8084
:10B8D00024E03146204600F04AF888B106EB8601A4
:10B8E0001C22606802EBC1014518284600F055F89B
:10B8F00040B10820E3E700002C000020585B020064
:10B900000520DCE7A5F80880F2B221464846FEF79C
:10B91000FAFE1FB1A8896989084438800020CEE763
:10B9200006F011BD017821F00F01491C21F0F00152
:10B9300010310170FDF7CFBD10B50446402800D985
:10B94000FFDF4034A0B210BD406842690078484330
:10B9500002EBC0007047C2784068037812FB03F224
:10B960004378406901FB032100EBC1007047C278B6
:10B970008A4209D9406801EB81011C2202EBC10116
:10B98000405C08B10120704700207047007806280D
:10B9900001D901207047002070470078062801D0A7
:10B9A0000120704700207047F0B401EB81061C278E
:10B9B000446807EBC6063444049D05262670E380E0
:10B9C0002571F0BCFEF78EBA10B5418911B1FFF7B1
:10B9D000DDFF08B1002010BD012010BD10B5C18CE5
:10B9E0008278B1EBC20F04D9C18911B1FFF7CEFF44
:10B9F00008B1002010BD012010BD10B50C46012378
:10BA00000A22011D06F07DFE007821880122824075
:10BA10009143218010BDF0B402EB82051C264C68D6
:10BA200006EBC505072363554B681C79402C03D1F1
:10BA30001A71F0BCFEF700BDF0BC704710B5EFF313
:10BA4000108000F0010472B6F9484178491C417039
:10BA50004078012801D10AF0F1F8002C00D162B63B
:10BA600010BD70B5F24CA07848B90125A570FFF75C
:10BA7000E5FF0AF0F4F820B100200AF0BEF800203B
:10BA800070BD4FF08040E570C0F80453F7E770B523
:10BA9000EFF3108000F0010572B6E54C607800B954
:10BAA000FFDF6078401E6070607808B90AF0CAF85D
:10BAB000002D00D162B670BDDD4810B5817821B18E
:10BAC0000021C1708170FFF7E2FF002010BD10B5AA
:10BAD00004460AF0C4F8D6498978084000D001200D
:10BAE0002060002010BD10B5FFF7A8FF0AF0B7F8DE
:10BAF00002220123CE49540728B1CE4802602361B7
:10BB00000320087202E00A72C4F80433002088712E
:10BB100010BD2DE9F05FDFF818934278817889F83D
:10BB20000420002689F80510074689F80660007889
:10BB3000DFF804B3354620B1012811D0022811D016
:10BB4000FFDF0AF09EF84FF0804498B10AF0A0F8A9
:10BB5000B0420FD130460AF09FF80028FAD041E0F9
:10BB60000126EEE7FFF76AFF58460168C907FCD0D7
:10BB70000226E6E70120E060C4F80451AF490E60F8
:10BB80000107D1F84412AD4AC1F3423124321160A9
:10BB9000AA49343108604FF0020AC4F804A3A06037
:10BBA000A7480168C94341F3001101F10108016888
:10BBB00041F01001016000E020BFD4F8040100282A
:10BBC000FAD030460AF068F80028FAD0B8F1000F31
:10BBD00004D19B48016821F010010160C4F808A35A
:10BBE000C4F8045199F805004E4688B1387878B900
:10BBF0000AF035F880460AF0C9F901466FF00042B4
:10BC0000B8F1000F02D0C6E9032101E0C6E9031232
:10BC1000DBF80000C00701D00AF01DF8387810B139
:10BC20003572BDE8F09F4FF01808C4F80883C4F8D7
:10BC30002C510127C4F81870D4F82C010028FBD02F
:10BC4000C4F80C51C4F810517948C01D0AF036F8F8
:10BC50003570FFF748FF6761784930792031086017
:10BC6000C4F80483DDE770B5050000D1FFDF4FF0B5
:10BC700080424FF0FF30C2F808030021C2F80011E3
:10BC8000C2F80411C2F80C11C2F81011684C6170AE
:10BC900009F0F1FF10B10120A070607066480068E3
:10BCA000C00701D009F0D7FF2846BDE8704030E753
:10BCB0005F48007A002800D0012070472DE9FF5F1F
:10BCC0006048D0F800805F4A5F49083211608406FE
:10BCD000D4F8080100B10120D4F8241101B10121E8
:10BCE0008A46D4F81C1101B101218946D4F82011EB
:10BCF00009B1012700E00027D4F8001101B10121AA
:10BD00008B46D4F8041101B101210391D4F80C1130
:10BD100001B101210291D4F8101101B10121444D6A
:10BD2000019129780026009120B1C4F80861012012
:10BD300009F063FFBAF1000F04D0C4F824610920B0
:10BD400009F05BFFB9F1000F04D0C4F81C610A20B0
:10BD500009F053FF27B1C4F820610B2009F04DFF13
:10BD60003348C01D09F0B2FF00B1FFDFDFF8C49017
:10BD70000127BBF1000F10D0C4F80873E87818B1A0
:10BD8000EE70002009F039FF287A022805D103203F
:10BD900028720221C9F800102761039808B1C4F87D
:10BDA0000461029850B1C4F80C61287A032800D0CD
:10BDB000FFDFC9F800602F72FFF769FE019838B104
:10BDC000C4F81061287A012801D100F05DF867619C
:10BDD000009838B12E70287A012801D1FFF783FE30
:10BDE000FFF755FE1248C01D09F086FF1549091DD1
:10BDF000C1F80080BDE8FF9F0D4810B5C01D09F0D7
:10BE000065FF0B4940B1012008704FF0E021C1F8F7
:10BE10000002BDE8104011E6087A012801D1FFF7C1
:10BE200062FE0348BDE81040C01D09F065BF000078
:10BE30003C000020340C00400C0400401805004079
:10BE400010ED00E0100502400100000170B5224C29
:10BE5000A07808B909F0F6FE01208507A861207ACC
:10BE6000002603280AD100BFD5F80C0120B9002014
:10BE700009F012FF0028F7D1C5F80C6126724FF0C7
:10BE8000FF30C5F8080370BD70B5134C6079F0B190
:10BE9000012803D0A179401E814218DA09F0DFFEA3
:10BEA00005460AF073F86179012902D9A179491C84
:10BEB000A1710DB1216900E0E168411A022902DA9D
:10BEC00011F1020F06DC0DB1206100E0E060BDE879
:10BED000704008E670BD00003C00002010B5202036
:10BEE00000F07FF8202000F08DF84D49202081F8E7
:10BEF0000004F5F783FA4B4908604B48D0F8041367
:10BF000041F00101C0F80413D0F8041341F080712E
:10BF1000C0F80413424901201C39C1F8000110BDCA
:10BF200010B5202000F05DF83E480021C8380160BF
:10BF3000001D01603D4A481E10603B4AC2F80803DC
:10BF4000384B1960C2F80001C2F860013849086036
:10BF5000BDE81040202000F055B834493548091F8D
:10BF60000860704731493348086070472D48C83829
:10BF70000160001D521E026070472C4901200860BC
:10BF8000BFF34F8F70472DE9F0412849D0F8188052
:10BF900028480860244CD4F800010025244E6F1E68
:10BFA00028B14046F5F788F940B9002111E0D4F8EE
:10BFB000600198B14046F5F77FF948B1C4F80051E7
:10BFC000C4F860513760BDE8F041202000F01AB895
:10BFD00031684046BDE8F04119F0E8BBFFDFBDE83D
:10BFE000F08100280DDB00F01F0201219140400983
:10BFF000800000F1E020C0F88011BFF34F8FBFF345
:10C000006F8F7047002809DB00F01F02012191406B
:10C010004009800000F1E020C0F880127047000065
:10C0200020E000E0C806024000000240180502407F
:10C0300000040240010000010F4A12680D498A42C3
:10C040000CD118470C4A12680A4B9A4206D101B526
:10C0500009F06EFFFFF781FFBDE80140074909685D
:10C060000958084706480749054A064B704700002B
:10C0700000000000BEBAFECA5400002004000020E8
:10C080008013002080130020F8B51D46DDE9064727
:10C090000E000AD006F0BCFD2346FF1DBCB231469F
:10C0A0002A46009406F0C9F9F8BDD019224619466F
:10C0B00019F0B0FA2046F8BD70B50D4604461021BF
:10C0C00019F027FB258117206081A07B40F00A0032
:10C0D000A07370BD4FF6FF720A80014602200AF07D
:10C0E0006DB9704700897047827BD30701D19207F1
:10C0F00003D4808908800020704705207047827B28
:10C10000920700D58181704701460020098841F6D9
:10C11000FE52114200D00120704700B50346807BDB
:10C12000C00701D0052000BD59811846FFF7ECFF7C
:10C13000C00703D0987B40F004009873987B40F0D0
:10C1400001009873002000BD827B520700D509B121
:10C150004089704717207047827B61F3C302827366
:10C1600070472DE9FC5F0E46044601789646012093
:10C1700000FA01F14DF6FF5201EA020962684FF63A
:10C18000FF7B1188594502D10920BDE8FC9FB9F118
:10C19000000F05D041F6FE55294201D00120F4E7F9
:10C1A00041EA090111801D0014D000232B7094F87E
:10C1B00000C0052103221F464FF0020ABCF10E0FFA
:10C1C00076D2DFE80CF0F909252F47646B774791A9
:10C1D00093B4D1D80420D8E7616820898B7B9B0772
:10C1E00067D517284AD30B89834247D389891729F2
:10C1F00001D3814242D185F800A0A5F80100328028
:10C20000616888816068817B21F002018173C6E0EA
:10C21000042028702089A5F801006089A5F8030092
:10C220003180BCE0208A3188C01D1FFA80F841456A
:10C2300024D3062028702089A5F801006089A5F87C
:10C240000300A089A5F805000721208ACDE9000197
:10C25000636941E00CF0FF00082810D00820287026
:10C260002089A5F801006089A5F8030031806A1DC6
:10C27000694604F10C0008F033F910B15EE01020BB
:10C28000EDE730889DF800100844308087E00A20F0
:10C2900028702089A5F80100328044E00C20287025
:10C2A0002089A5F801006089A5F8030031803AE0F3
:10C2B00082E064E02189338800EB41021FFA82F8B2
:10C2C00043453BD3B8F1050F38D30E222A700BEA51
:10C2D0004101CDE90010E36860882A467146FFF706
:10C2E000D3FEA6F800805AE040202870608931888B
:10C2F000C01C1FFA80F8414520D32878714620F0F1
:10C300003F00123028702089A5F801006089CDE92E
:10C31000000260882A46E368FFF7B6FEA6F80080B0
:10C32000287840063BD461682089888037E0A0895E
:10C330003288401D1FFA80F8424501D204273DE0B3
:10C34000162028702089A5F801006089A5F803004F
:10C35000A089CDE9000160882A4671462369FFF76C
:10C3600093FEA6F80080DEE718202870207A687017
:10C37000A6F800A013E061680A88920401D405279A
:10C380001CE0C9882289914201D0062716E01E21AF
:10C39000297030806068018821F400510180B9F172
:10C3A000000F0BD0618878230022022009F05CFF87
:10C3B00061682078887006E0338003276068018810
:10C3C00021EA090101803846DFE62DE9FF4F85B0FB
:10C3D0001746129C0D001E461CD03078C10703D0B2
:10C3E00000F03F00192801D9012100E0002120467A
:10C3F000FFF7AAFEA8420DD32088A0F57F41FF39A0
:10C4000008D03078410601D4000605D5082009B0CF
:10C41000BDE8F08F0720FAE700208DF800008DF8C6
:10C42000010030786B1E00F03F0C0121A81E4FF078
:10C43000050A4FF002094FF0030B9AB2BCF1200F2E
:10C4400075D2DFE80CF08B10745E7468748C749C89
:10C4500074B674BB74C974D574E2747474F274F0F5
:10C4600074EF74EE748B052D78D18DF80090A07860
:10C470008DF804007088ADF8060030798DF8010061
:10C48000707800F03F000C2829D00ADCA0F10200EF
:10C49000092863D2DFE800F0126215621A621D6299
:10C4A0002000122824D004DC0E281BD01028DBD159
:10C4B0001BE016281FD01828D6D11FE0207880074F
:10C4C00001E020784007002848DAEFE020780007F4
:10C4D000F9E72078C006F6E720788006F3E72078B1
:10C4E0004006F0E720780006EDE72088C005EAE77F
:10C4F00020884005E7E720880005E4E72088C0049D
:10C50000E1E72078800729D5032D27D18DF800B0E9
:10C51000B6F8010082E0217849071FD5062D1DD30A
:10C5200081B27078012803D0022817D102E0CAE056
:10C53000022000E0102004228DF8002072788DF88F
:10C540000420801CB1FBF0F2ADF8062092B2424309
:10C550008A4203D10397ADF80890A7E07AE02078EB
:10C56000000777D598B282088DF800A0ADF80420B6
:10C57000B0EB820F6ED10297ADF8061096E02178ED
:10C58000C90667D5022D65D381B206208DF800005B
:10C59000707802285ED300BFB1FBF0F28DF8040082
:10C5A000ADF8062092B242438A4253D1ADF80890CA
:10C5B0007BE0207880064DD5072003E020784006F8
:10C5C0007FD508208DF80000A088ADF80400ADF8F4
:10C5D0000620ADF8081068E02078000671D5092023
:10C5E000ADF804208DF80000ADF8061002975DE06C
:10C5F0002188C90565D5022D63D381B20A208DF843
:10C600000000707804285CD3C6E72088400558D520
:10C61000012D56D10B208DF80000A088ADF8040044
:10C6200044E021E026E016E0FFE72088000548D539
:10C63000052D46D30C208DF80000A088ADF804002D
:10C64000B6F803006D1FADF80850ADF80600ADF860
:10C650000AA02AE035E02088C00432D5012D30D16F
:10C660000D208DF8000021E02088800429D4B6F840
:10C670000100E080A07B000723D5032D21D3307873
:10C6800000F03F001B2818D00F208DF800002088F4
:10C6900040F40050A4F80000B6F80100ADF8040022
:10C6A000ED1EADF80650ADF808B003976946059841
:10C6B000F5F730FC050008D016E00E208DF80000DC
:10C6C000EAE7072510E008250EE0307800F03F008B
:10C6D0001B2809D01D2807D00220059909F06EFEFD
:10C6E000208800F400502080A07B400708D5204619
:10C6F000FFF70AFDC00703D1A07B20F00400A07360
:10C70000284684E61FB5022806D101208DF80000D6
:10C7100088B26946F5F7FEFB1FBD0000F8B51D465F
:10C72000DDE906470E000AD006F072FA2346FF1D27
:10C73000BCB231462A46009405F07FFEF8BDD01900
:10C740002246194618F066FF2046F8BD2DE9FF4F36
:10C750008DB09B46DDE91B57DDF87CA00C46082B0D
:10C7600005D0E06901F002F950B11020D2E028882C
:10C77000092140F0100028808AF80010022617E0F6
:10C78000E16901208871E2694FF420519180E169EB
:10C790008872E06942F601010181E069002181733C
:10C7A0002888112140F0200028808AF800100426F3
:10C7B00038780A900A2038704FF0020904F1180006
:10C7C0004D460C9001F095FBB04681E0BBF1100F97
:10C7D0000ED1022D0CD0A9EB0800801C80B20221E2
:10C7E000CDE9001005AB52461E990D98FFF796FF54
:10C7F000BDF816101A98814203D9F74800790F90B6
:10C8000004E003D10A9808B138702FE04FF002011C
:10C81000CDE900190DF1160352461E990D98FFF748
:10C820007DFF1D980088401B801B83B2C6F1FF006E
:10C83000984200D203461E990BA8D9B15FF00002BE
:10C84000DDF878C0CDE9032009EB060189B2CDE916
:10C8500001C10F980090BDF8161000220D9801F04C
:10C86000CBFB387070B1C0B2832807D0BDF816007A
:10C8700020833AE00AEB09018A19E1E7022011B0AE
:10C88000BDE8F08FBDF82C00811901F0FF08022DE2
:10C890000DD09AF80120424506D1BDF82010814202
:10C8A00007D0B8F1FF0F04D09AF801801FE08AF892
:10C8B0000180C94800680178052902D1BDF8161029
:10C8C000818009EB08001FFA80F905EB080085B2AA
:10C8D000DDE90C1005AB0F9A01F00EFB28B91D988D
:10C8E0000088411B4145BFF671AF022D13D0BBF14B
:10C8F000100F0CD1A9EB0800801C81B20220CDE9F9
:10C90000000105AB52461E990D98FFF707FF1D98D1
:10C910000580002038700020B1E72DE9F8439C46DF
:10C92000089E13460027B26B9AB3491F8CB2F18F51
:10C93000A1F57F45FF3D05D05518AD882944891DD7
:10C940008DB200E000252919B6F83C800831414538
:10C9500020D82A44BCF8011022F8021BBCF80310AE
:10C9600022F8021B984622F8024B914606F03EF947
:10C970004FF00C0C41464A462346CDF800C005F066
:10C9800028FDF587B16B00202944A41D21440880AF
:10C9900003E001E0092700E083273846BDE8F8837B
:10C9A00010B50B88848F9C420CD9846BE0180488E6
:10C9B00044B1848824F40044A41D23440B801060F7
:10C9C000002010BD0A2010BD2DE9F0478AB00025D7
:10C9D000904689468246ADF8185007274BE00598E7
:10C9E00006888088000446D4A8F8006007A801954E
:10C9F00000970295CDE903504FF4007300223146B1
:10CA0000504601F0F9FA04003CD1BDF81800ADF829
:10CA10002000059804888188B44216D10A0414D4F1
:10CA200001950295039521F400410097049541F486
:10CA3000804342882146504601F0B4F804000BD1EF
:10CA40000598818841F40041818005AA08A94846DB
:10CA5000FFF7A6FF0400DCD000970598029501952A
:10CA6000039504950188BDF81C300022504601F062
:10CA700099F80A2C06D105AA06A94846FFF790FFA7
:10CA80000400ACD0ADF8185004E00598818821F47A
:10CA90000041818005AA06A94846FFF781FF0028CA
:10CAA000F3D00A2C03D020460AB0BDE8F08700205E
:10CAB000FAE710B50C46896B86B051B10C218DF8A0
:10CAC0000010A18FADF80810A16B01916946FAF72B
:10CAD00022FB00204FF6FF71A063E187A08706B01C
:10CAE00010BD2DE9F0410D460746896B0020069EDA
:10CAF0001446002911D0012B0FD132462946384661
:10CB0000FFF762FF002808D1002C06D032462946E4
:10CB10003846BDE8F04100F038BFBDE8F0812DE9AE
:10CB2000FC411446DDE9087C0E46DDE90A15521D7C
:10CB3000BCF800E092B2964502D20720BDE8FC8125
:10CB4000ACF8002017222A70A5F80160A5F8033080
:10CB50000522CDE900423B462A46FFF7DFFD0020D3
:10CB6000ECE770B50C4615464821204618F0F3FD59
:10CB700004F1080044F81C0F00204FF6FF71E0613B
:10CB800061842084A5841720E08494F82A0040F072
:10CB90000A0084F82A0070BD4FF6FF720A80014631
:10CBA000032009F00BBC30B585B00C460546FFF7F5
:10CBB00080FFA18E284629B101218DF80010694619
:10CBC000FAF7A9FA0020E0622063606305B030BD87
:10CBD000B0F84000704700005800002090F8462050
:10CBE000920703D4408808800020F3E70620F1E78D
:10CBF00090F846209207EDD5A0F84410EAE70146E8
:10CC0000002009880A0700D5012011F0F00F01D09B
:10CC100040F00200CA0501D540F004008A0501D5A4
:10CC200040F008004A0501D540F010000905D1D5B3
:10CC300040F02000CEE700B5034690F84600C0075C
:10CC400001D0062000BDA3F842101846FFF7D7FF19
:10CC500010F03E0F05D093F8460040F0040083F832
:10CC6000460013F8460F40F001001870002000BD88
:10CC700090F84620520700D511B1B0F84200A9E75C
:10CC80001720A7E710F8462F61F3C3020270A1E74F
:10CC90002DE9FF4F9BB00E00DDE92B34DDE929784B
:10CCA000289D24D02878C10703D000F03F00192820
:10CCB00001D9012100E000212046FFF7D9FFB04251
:10CCC00015D32878410600F03F010CD41E290CD062
:10CCD000218811F47F6F0AD13A8842B1A1F57F42D1
:10CCE000FF3A04D001E0122901D1000602D5042048
:10CCF0001FB0C5E5F9491D984FF0000A08718DF87D
:10CD000018A08DF83CA00FAA0A60ADF81CA0ADF8E1
:10CD100050A02978994601F03F02701F5B1C04F176
:10CD2000180C4FF0060E4FF0040BCDF858C01F2A18
:10CD30007ED2DFE802F07D7D107D267DAC7DF47D26
:10CD4000F37DF27DF17DF47DF07D7D7DEF7DEE7DE7
:10CD50007D7D7D7DED0094F84610B5F801008907D2
:10CD600001D5032E02D08DF818B022E34FF40061F4
:10CD7000ADF85010608003218DF83C10ADF84000F4
:10CD8000D8E2052EEFD1B5F801002083ADF81C00E4
:10CD9000B5F80310618308B1884201D901207FE111
:10CDA0000020A07220814FF6FF702084169801F0B9
:10CDB000A0F8052089F800000220029083460AAB03
:10CDC0001D9A16991B9801F097F890BB9DF82E00BC
:10CDD000012804D0022089F80100102003E001207E
:10CDE00089F8010002200590002203A90BA807F092
:10CDF00077FBE8BB9DF80C00059981423DD13A884C
:10CE0000801CA2EB0B01814237DB02990220CDE9A5
:10CE100000010DF12A034A4641461B98FFF77EFCAC
:10CE200002980BF1020B801C80B217AA03A901E043
:10CE3000A0E228E002900BA807F052FB02999DF8AF
:10CE40000C00CDE9000117AB4A4641461B98FFF79D
:10CE500065FC9DF80C100AAB0BEB01001FFA80FB80
:10CE600002981D9A084480B2029016991B9800E01F
:10CE700003E001F041F80028B6D0BBF1020F02D068
:10CE8000A7F800B053E20A208DF818004FE2002105
:10CE90000391072EFFF467AFB5F801002083ADF8CA
:10CEA0001C00B5F80320628300283FF477AF90425E
:10CEB0003FF674AF0120A072B5F805002081002074
:10CEC000A073E06900F052FD78B9E1690120887132
:10CED000E2694FF420519180E1698872E06942F67D
:10CEE00001010181E06900218173F01F20841E98F7
:10CEF000606207206084169800F0FBFF072089F825
:10CF000000000120049002900020ADF82A0028E0E3
:10CF10001DE2A3E13AE1EAE016E2AEE086E049E094
:10CF20000298012814D0E0698079012803D1BDF866
:10CF30002800ADF80E00049803ABCDE900B04A46D6
:10CF400041461B98FFF7EAFB0498001D80B204904D
:10CF5000BDF82A00ADF80C00ADF80E00059880B2BF
:10CF600002900AAB1D9A16991B9800F0C5FF28B9CC
:10CF700002983988001D05908142D1D2029801287B
:10CF800081D0E0698079012805D0BDF82810A1F58D
:10CF90007F40FF3803D1BDF82800ADF80E0004989B
:10CFA00003ABCDE900B04A4641461B98FFF7B6FBFC
:10CFB0000298BBE1072E02D0152E7FF4D4AEB5F84F
:10CFC00001102183ADF81C10B5F8032062830029FD
:10CFD0003FF4E4AE91423FF6E1AE0121A1724FF081
:10CFE000000BA4F808B084F80EB0052E07D0C0B22C
:10CFF000691DE26907F055FA00287FF444AF4FF647
:10D00000FF70208401A906AA14A8CDF800B081E819
:10D0100085032878214600F03F031D9A1B98FFF7EF
:10D0200095FB8246208BADF81C0080E10120032E89
:10D03000C3D14021ADF85010B5F801102183ADF8EF
:10D040001C100AAAB8F1000F00D00023CDE902039A
:10D0500004921D98CDF80480009038880022401E6C
:10D0600083B21B9800F0C8FF8DF8180090BB0B200E
:10D0700089F80000BDF8280037E04FF0010C052EBC
:10D080009BD18020ADF85000B5F801102183B5F890
:10D0900003002084ADF81C10B0F5007F03D90720F1
:10D0A0008DF8180085E140F47C4222840CA8B8F188
:10D0B000000F00D00023CDE90330CDE9018C1D988D
:10D0C00000903888401E83B21B9800F095FF8DF8C1
:10D0D000180028B18328A8D10220BDE05800002004
:10D0E0000D2189F80010BDF83000401C1EE1032E10
:10D0F00004D248067FF537AE002017E1B5F80110DD
:10D10000ADF81C102878400602D58DF83CE002E00E
:10D1100007208DF83C004FF000080320CDE90208FD
:10D120001E9BCDF810801D980193A6F1030B009073
:10D130001FFA8BF342461B9800F034FD8DF818005F
:10D140008DF83C80297849060DD52088C00506D584
:10D15000208BBDF81C10884201D1C4F824804046C1
:10D160008DF81880E2E0832801D14FF0020A4FF4D5
:10D170008070ADF85000BDF81C002083A4F820B0EA
:10D180001E986062032060841321CCE0052EFFF41A
:10D19000EAADB5F80110ADF81C10A28F62B3A2F58C
:10D1A0007F43FE3B28D008228DF83C204FF0000B37
:10D1B0000523CDE9023BDDF878C0CDF810B01D9A0B
:10D1C00080B2CDF804C040F400430092B5F80320CB
:10D1D0001B9800F0E7FC8DF83CB04FF400718DF81F
:10D1E0001800ADF85010832810D0F8B1A18FA1F528
:10D1F0007F40FE3807D0DCE00B228DF83C204FF654
:10D20000FE72A287D2E7A4F83CB0D2E000942B468D
:10D2100031461E9A1B98FFF780FB8DF8180008B165
:10D2200083284BD1BDF81C00208355E700942B4682
:10D2300031461E9A1B98FFF770FB8DF81800E8BB6B
:10D24000E18FA06B0844811D8DE8820343888288AA
:10D2500001881B98FFF763FC824668E095F801801F
:10D26000022E70D15FEA080002D0B8F1010F6AD136
:10D2700009208DF83C0007A800908DF840804346B7
:10D28000002221461B98FFF72CFC8DF842004FF03E
:10D29000000B8DF843B050B9B8F1010F12D0B8F1BE
:10D2A000000F04D1A18FA1F57F40FF380AD0A08FD5
:10D2B00040B18DF83CB04FF4806000E037E0ADF84D
:10D2C00050000DE00FA91B98F9F725FF82468DF855
:10D2D0003CB04FF48060ADF85000BAF1020F06D0B8
:10D2E000FC480068C07928B18DF8180027E0A4F840
:10D2F000188044E0BAF1000F03D081208DF81800A7
:10D300003DE007A800904346012221461B98FFF705
:10D31000E8FB8DF8180021461B98FFF7CAFB9DF823
:10D32000180020B9192189F80010012038809DF8D3
:10D330003C0020B10FA91B98F9F7EDFE8246BAF127
:10D34000000F33D01BE018E08DF818E031E02078B2
:10D35000000712D5012E10D10A208DF83C00E0887C
:10D36000ADF8400003201B9909F028F80820ADF81B
:10D370005000C1E648067FF5F6AC4FF0040A20885D
:10D38000BDF8501008432080BDF8500080050BD533
:10D39000A18FA1F57F40FE3806D11E98E062289843
:10D3A0002063A6864FF0030A5046A1E49DF81800BA
:10D3B00078B1012089F80000297889F80110BDF8BA
:10D3C0001C10A9F802109DF8181089F80410052007
:10D3D00038802088BDF8501088432080E4E72DE98C
:10D3E000FF4F8846087895B0012181404FF209002F
:10D3F000249C0140ADF820102088DDF88890A0F52D
:10D400007F424FF0000AFF3A06D039B1000705D538
:10D41000012019B0BDE8F08F0820FAE7239E4FF0F5
:10D42000000B0EA886F800B018995D460988ADF883
:10D430003410A8498DF81CB0179A0A718DF838B0CD
:10D44000086098F8000001283BD0022809D0032882
:10D450006FD1307820F03F001D303070B8F80400F4
:10D46000E08098F800100320022904D1317821F0DF
:10D470003F011B31317094F84610090759D505ABAF
:10D48000B9F1000F13D0002102AA82E80B00072097
:10D49000CDE90009BDF83400B8F80410C01E83B20D
:10D4A0000022159800F0A8FD0028D1D101E0F11C60
:10D4B000EAE7B8F80400A6F80100BDF81400C01CA3
:10D4C00004E198F805108DF81C1098F80400012864
:10D4D00006D04FF4007A02282CD00328B8D16CE192
:10D4E0002188B8F8080011F40061ADF8201020D0B0
:10D4F00017281CD3B4F84010814218D3B4F8441054
:10D50000172901D3814212D1317821F03F01C91C82
:10D510003170A6F801000321ADF83410A4F84400DE
:10D5200094F8460020F0020084F8460065E10525E5
:10D530007EE177E1208808F1080700F4FE60ADF88D
:10D54000200010F0F00F1BD010F0C00F03D038886F
:10D55000228B9042EBD199B9B878C00710D0B96846
:10D560000720CDE902B1CDF804B00090CDF810B09D
:10D57000FB88BA883988159800F014FB0028D6D1AA
:10D580002398BDF82010401C80294ED006DC1029BD
:10D590000DD020290BD0402987D124E0B1F5807F20
:10D5A0006ED051457ED0B1F5806F97D1DEE0C806D0
:10D5B00001D5082000E0102082460DA907AA052009
:10D5C000CDE902218DF83800ADF83CB0CDE90496E4
:10D5D00008A93888CDE9000153460722214615984D
:10D5E000FFF7B4F8A8E09DF81C2001214FF00A0ACB
:10D5F000002A9BD105ABB9F1000F00D00020CDE986
:10D6000002100720CDE90009BDF834000493401E44
:10D6100083B2218B0022159800F0EEFC8DF81C00DF
:10D620000B203070BDF8140020E09DF81C20012173
:10D630004FF00C0A002A22D113ABB9F1000F00D031
:10D640000020CDE902100720CDE900090493BDF8C0
:10D650003400228C401E83B2218B159800F0CCFC44
:10D660008DF81C000D203070BDF84C00401CADF84A
:10D67000340005208DF83800208BADF83C00BCE06C
:10D680003888218B88427FF452AF9DF81C004FF000
:10D69000120A00281CD1606AA8B1B878C0073FF40C
:10D6A00046AF00E018E0BA680720CDE902B2CDF835
:10D6B00004B00090CDF810B0FB88BA88159800F03F
:10D6C00071FA8DF81C00132030700120ADF8340081
:10D6D00093E00000580000203988208B8142D2D18D
:10D6E0009DF81C004FF0160A0028A06B08D0E0B38C
:10D6F0004FF6FF7000215F46ADF808B0019027E0BB
:10D7000068B1B978C907BED1E18F0DAB0844821D5D
:10D7100003968DE80C0243888288018809E0B87876
:10D72000C007BCD0BA680DAB03968DE80C02BB886D
:10D73000FA881598FFF7F3F905005ED0072D72D02F
:10D7400076E0019005AA02A92046FFF729F90146D3
:10D75000E28FBDF80800824201D00029F1D0E08FAD
:10D76000A16B084407800198E08746E09DF81C0003
:10D770004FF0180A40B1208BC8B138882083214669
:10D780001598FFF796F938E004F118000090237E11
:10D79000012221461598FFF7A4F98DF81C000028F6
:10D7A000EDD1192030700120ADF83400E7E70525F0
:10D7B00021461598FFF77DF93AE0208800F40070C3
:10D7C000ADF8200050452DD1A08FA0F57F41FE3946
:10D7D00001D006252CE0D8F808004FF0160A48B111
:10D7E000A063B8F80C10A1874FF6FF71E187A0F88D
:10D7F00000B002E04FF6FF70A087BDF8200030F4C3
:10D800007F611AD0782300220320159908F02CFD9F
:10D8100098F8000020712088BDF82010084320806F
:10D820000EE000E007252088BDF820108843208006
:10D83000208810F47F6F1CD03AE02188814321803A
:10D840009DF8380020B10EA91598F9F764FC05463B
:10D850009DF81C000028EBD086F801A00120307054
:10D86000208B70809DF81C0030710520ADF83400CD
:10D87000DEE7A18EE1B118980DAB0088ADF8340059
:10D880002398CDE90304CDE90139206B0090E36AC8
:10D89000179A1598FFF7FCF9054601208DF8380016
:10D8A0000EA91598F9F737FC00B10546A4F834B075
:10D8B00094F8460040070AD52046FFF7A0F910F07B
:10D8C0003E0F04D114F8460F20F004002070189881
:10D8D000BDF83410018028469BE500B585B00328CB
:10D8E00006D102208DF8000088B26946F9F713FCD2
:10D8F00005B000BD10B5384C0B782268012B02D062
:10D90000022B2AD111E013780BB1052B01D104238E
:10D91000137023688A889A802268CB88D380226813
:10D920000B891381498951810DE08B88938022688E
:10D93000CB88D38022680B8913814B8953818B89D3
:10D940009381096911612168F9F7E5FB22680021DB
:10D950000228117003D0002800D0812010BD832040
:10D9600010BD806B002800D001207047817801290C
:10D9700009D10088B0F5205F03D042F6010188424A
:10D9800001D10020704707207047F0B587B0002410
:10D9900015460E460746ADF8184011E00598008878
:10D9A000288005980194811DCDE902410721049446
:10D9B0000091838842880188384600F0F3F830B936
:10D9C00005AA06A93046FEF7EBFF0028E6D00A2894
:10D9D00000D1002007B0F0BD5800002010B58B78B2
:10D9E00083B102789A4205D10B885BB102E08B7952
:10D9F000091D4BB18B789A42F9D1B0F801300C88EF
:10DA0000A342F4D1002010BD812010BD072826D0EC
:10DA100012B1012A27D103E0497801F0070102E0A1
:10DA20004978C1F3C20105291DD2DFE801F00318CE
:10DA3000080C12000AB10320704702207047042826
:10DA40000DD250B10DE0052809D2801E022808D35E
:10DA500003E0062803D0032803D0052070470020E8
:10DA600070470F20704781207047C0B282060BD4E8
:10DA7000000607D5FE48807A4143C01D01EBD00067
:10DA800080B27047084670470020704770B5138811
:10DA90000B800B781C0625D5F54CA47A844204D85B
:10DAA00043F010000870002070BD956800F0070674
:10DAB00005EBD0052D78F54065F304130B70137852
:10DAC000D17803F0030341EA032140F20123B1FBC3
:10DAD000F3F503FB15119268E41D00FB012000EB38
:10DAE000D40070BD906870BD37B51446BDF8041001
:10DAF00011809DF804100A061ED5C1F30013DC49FD
:10DB0000A568897A814208D8FE2811D1C91DC908A3
:10DB10005A42284617F0F5FD0AE005EBD00100F067
:10DB20000702012508789540A843934018430870E0
:10DB3000207820F0100020703EBD2DE9F04107460E
:10DB4000C81C0E4620F00300B04202D08620BDE87B
:10DB5000F081C74D002034462E60AF802881AA7224
:10DB6000E8801AE0E988491CE980810614D4E1784C
:10DB700000F0030041EA002040F20121B0FBF1F285
:10DB800001FB12012068FFF770FF2989084480B269
:10DB90002881381A3044A0600C3420784107E1D441
:10DBA0000020D4E72DE9FF4F89B01646DDE9168A3B
:10DBB0000F46994623F44045084600F00DFB04004B
:10DBC0000FD0099804F0A6FE0290207800060AD52E
:10DBD000A748817A0298814205D887200DB0BDE818
:10DBE000F08F0120FAE7224601A90298FFF74EFFC5
:10DBF000834600208DF80C004046B8F1070F1AD07C
:10DC000001222146FFF702FF0028E7D120784006D5
:10DC100011D502208DF80C00ADF81070BDF804008D
:10DC2000ADF81200ADF814601898ADF81650CDF8A4
:10DC30001CA0ADF818005FEA094004D500252E4667
:10DC4000A84601270CE02178E07801F0030140EAC2
:10DC5000012040F20121B0FBF1F2804601FB128766
:10DC60005FEA494009D5B84507D1A178207901F08C
:10DC7000030140EA0120B04201D3BE4201D907208E
:10DC8000ACE7A8191FFA80F9B94501D90D20A5E71D
:10DC90009DF80C0028B103A90998F9F73AFA002871
:10DCA0009CD1B84507D1A0784FEA192161F3010052
:10DCB000A07084F804901A9800B10580199850EA71
:10DCC0000A0027D0199830B10BEB06002A461999A3
:10DCD00017F0A0FC0EE00BEB06085746189E0998BB
:10DCE00004F084FF2B46F61DB5B239464246009536
:10DCF00004F06FFB224601A90298FFF7C7FE9DF8CA
:10DD00000400224620F010008DF80400DDE9011027
:10DD1000FFF7EAFE002061E72DE9FF4FDFF85091A1
:10DD200082461746B9F80610D9F8000001EB410108
:10DD300000EB810440F20120B2FBF0F185B000FB62
:10DD400011764D46DDF84C8031460698FFF78DFE82
:10DD500029682A898B46611A0C3101441144AB8829
:10DD600089B28B4202D8842009B038E70699CDB237
:10DD7000290603D5A90601D50620F5E7B9F806C09E
:10DD80000CF1010C1FFA8CFCA9F806C0149909B11A
:10DD9000A1F800C0A90602D5C4F8088007E0104425
:10DDA00080B2A9F80800191A01EB0B00A060224606
:10DDB000FE200699FFF798FEE77026712078390A51
:10DDC00061F30100320AA17840F0040062F301011E
:10DDD000A17020709AF802006071BAF80000E0802B
:10DDE00000262673280602D599F80A7000E001275C
:10DDF000A80601D54FF000084D4600244FF0070952
:10DE00000FE0CDE902680196CDF800900496E9880C
:10DE10002046129B089AFFF7C5FE0028A4D1641C77
:10DE2000E4B2BC42EDD300209EE72DE9F0478046E6
:10DE300000F0D2F9070005D0002644460C4D40F210
:10DE4000012919E00120BDE8F087204600F0C4F95F
:10DE50000278C17802F0030241EA0222B2FBF9F330
:10DE600009FB13210068FFF700FE304486B201E091
:10DE7000F4050020641CA4B2E988601E8142E4DC41
:10DE8000A8F10100E8802889801B288100203870D3
:10DE9000D9E710B5144631B1491E218004F03AFD8E
:10DEA000A070002010BD012010BD10B5D24904465D
:10DEB0000088CA88904201D30A2010BD096800EB8F
:10DEC000400001EB80025079A072D08820819178C7
:10DED000107901F0030140EA0120A081A078E11C43
:10DEE000FFF7D4FD20612088401C2080E0800020C6
:10DEF00010BD0121018270472DE9FF4F85B04FF61B
:10DF0000FF788246A3F8008048681F460D46807857
:10DF10008DF8060048680088ADF8040000208DF8F0
:10DF20000A00088A0C88A04200D304462C8241E0F3
:10DF3000288A401C2882701D6968FFF74FFDB8BB16
:10DF40003988414501D1601E38806888A04236D3A7
:10DF5000B178307901F0030140EA012901A9701D6F
:10DF6000FFF73CFD20BB298941452CD000223146DA
:10DF70000798FFF74BFDD8B92989494518D1E968B9
:10DF80000391B5F80AC0D6F808B05046CDF800C0E5
:10DF900004F02CFEDDF800C05A460CF1070C1FFA05
:10DFA0008CFC4B460399CDF800C004F0DCF950B16D
:10DFB000641CA4B2204600F00FF90600B8D1641E1C
:10DFC0002C820A20D0E67C807079B871F088B88005
:10DFD0003178F07801F0030140EA01207881A7F858
:10DFE0000C90504604F096FC324607F10801FFF70A
:10DFF0004DFD38610020B7E62DE9FF4F87B081461F
:10E000001C469246DDF860B0DDF85480089800F0B8
:10E01000E3F805000CD0484604F07CFC297809069A
:10E0200008D57549897A814204D887200BB0D6E596
:10E030000120FBE7CAF309062A4601A9FFF726FDDE
:10E040000746149807281CD000222946FFF7DEFC5B
:10E050000028EBD12878400613D501208DF8080060
:10E060000898ADF80C00BDF80400ADF80E00ADF84E
:10E070001060ADF8124002A94846F9F74AF80028A6
:10E08000D4D12978E87801F0030140EA0121AA7887
:10E09000287902F0030240EA0220564507D0B1F584
:10E0A000007F04D9611E814201DD0B20BEE786425C
:10E0B00001D90720BAE7801B85B2A54200D92546C1
:10E0C000BBF1000F01D0ABF80050179818B1B91987
:10E0D0002A4617F09FFAB8F1000F0DD03E4448468B
:10E0E0004446169F04F094FD2146FF1DBCB2324603
:10E0F0002B46009404F0A1F9002097E72DE9F041A8
:10E1000007461D461646084600F066F804000BD088
:10E11000384604F0FFFB2178090607D53649897A8D
:10E12000814203D8872012E5012010E522463146BE
:10E13000FFF7ACFC65B12178E07801F0030140EA1B
:10E140000120B0F5007F01D8012000E000202870F8
:10E150000020FCE42DE9F04107461D46164608461E
:10E1600000F03AF804000BD0384604F0D3FB2178D5
:10E17000090607D52049897A814203D88720E6E439
:10E180000120E4E422463146FFF7AEFCFF2D14D017
:10E190002178E07801F0030240EA022040F20122F7
:10E1A000B0FBF2F302FB130015B900F2012080B2BC
:10E1B000E070000A60F3010121700020C7E410B58F
:10E1C0000C4600F009F828B1C18821804079A07080
:10E1D000002010BD012010BD0749CA88824209D322
:10E1E00040B1096800EB40006FF00B0202EB8000C9
:10E1F0000844704700207047F405002010B508F06F
:10E20000C3FAF4F753FB08F025F9BDE8104008F015
:10E21000EDB9302834BF012000207047202834BFDA
:10E220004FF0A0420C4A012300F01F0003FA00F057
:10E23000002914BFC2F80C05C2F808057047202851
:10E2400034BF4FF0A041044900F01F00012202FA40
:10E2500000F0C1F8180570470003005070B5034680
:10E26000002002466FF02F050EE09C5CA4F1300602
:10E270000A2E02D34FF0FF3070BD00EB800005EB9B
:10E280004000521C2044D2B28A42EED370BD30B559
:10E290000A230BE0B0FBF3F403FB1404B0FBF3F030
:10E2A0008D183034521E05F8014CD2B2002AF1D13B
:10E2B00030BD30B500234FF6FF7510E0040A44EA84
:10E2C000002084B2C85C6040C0F30314604005EADB
:10E2D00000344440E0B25B1C84EA40109BB293429D
:10E2E000ECD330BD2DE9F041FA4B0026012793F81D
:10E2F00060501C7893F864C0B8B183F88D40A3F8DF
:10E300008E1083F88C2083F88A70BCF1000F0CBF4C
:10E3100083F8906083F89050EF488068008804F09C
:10E3200065FCBDE8F04104F0FBB84FF6FF7083F8E0
:10E330008D40A3F88E0083F88C2083F88A70BCF19E
:10E34000000F14BF83F8905083F89060BDE8F0810F
:10E3500070B5E14E0446306890F898100025012908
:10E3600019D090F89210012924D090F86810012952
:10E370002AD090F88A1001291CBF002070BD65705A
:10E3800017212170D0F88C106160B0F890102181B5
:10E3900080F88A5016E065701C212170D0F8991021
:10E3A0006160D0F89D10A16090F8A110217380F8F1
:10E3B000985007E0657007212170D0F894106160D3
:10E3C00080F89250012070BD65701421217000F119
:10E3D0006A012022201D17F01DF9012121723068E9
:10E3E00080F86850BB48B0F86C20A0F89420B26860
:10E3F000537B80F8963080F89210108804F0F6FB7A
:10E4000004F09DF8DEE7B448006890F86810002931
:10E4100014BFB0F86C004FF6FF70704770B5AE4C8B
:10E4200006462068002808BFFFDF002520684570E9
:10E430006660002808BFFFDF2068417800291CBF04
:10E44000FFDF70BDA42117F086F92068FF2101705D
:10E450007F2180F8361013214184282180F865102F
:10E46000012180F8581080F85D5008F0C3FDBDE828
:10E47000704008F01CB898490968097881420CBFBF
:10E480000120002070479448006890F82200C0F3F3
:10E49000400070479048006890F8220000F00100AA
:10E4A00070478D48006890F82200C0F30010704754
:10E4B0002DE9F04388480024036893F82400B3F85A
:10E4C00022C0C0F38001C0F34002114400F00100FB
:10E4D0000144CCF3001060B3BCF1130F21D00BDC6E
:10E4E000BCF1100F02BF7D4830F81100BDE8F08389
:10E4F000BCF1120F15D008E0BCF1150F09D0BCF12A
:10E500001D0F04BF7648BDE8F083FFDF2046BDE85D
:10E51000F083744A002032F8112011FB0020BDE87E
:10E52000F083714A002032F8112011FB0020BDE871
:10E53000F08393F85A2093F85B002E264FF47A77F5
:10E540004FF014084FF04009022A04BF4AF2D745A1
:10E55000B5FBF7F510D0012A04BF4AF22F75B5FBC1
:10E56000F7F510D04AF62315B5FBF7F5082A08BFD2
:10E570004E4613D0042A18D02646082A0ED0042A64
:10E5800013D0022A49D004F12806042A0FD0082A01
:10E590001CBF4FF01908082204D00AE04FF01408FD
:10E5A00006F5A8764FF0400203E006F5A8764FF096
:10E5B000100218FB026212FB0152C1EB01114B4D1C
:10E5C00001EB810105EB810111441CF0010F4FF4B7
:10E5D000C8724FF4BF7504BFCCF34006002E77D04D
:10E5E000CCF3400601F5A571EEB1082804BF16462C
:10E5F00040270CD0042804BF2E46102707D002283D
:10E6000007BF04F11806042704F12806082707EBC2
:10E61000870706EB870631441CE004F118064FF02B
:10E6200019080422C5E7082804BF164640270CD065
:10E63000042804BF2E46102707D0022807BF04F184
:10E640001806042704F12806082707EB871706EBAE
:10E650008706314401F19C0693F8651010F00C0F09
:10E6600008BF00213144082804BF164640270CD0BB
:10E67000042804BF2E46102707D0022807BF04F144
:10E680001806042704F128060827C7EBC70707EB7D
:10E69000470706EB4706314498311CF0010F27D09D
:10E6A000082808BF40200CD0042804BF2A461020A8
:10E6B00007D0022807BF04F11802042004F1280241
:10E6C000082000EB400303EB0010104401444AE033
:10E6D0004DE000000006002060000020BC5B02004E
:10E6E0008E891300C45B0200B45B0200D4FEFFFFFE
:10E6F000082804BF944640260CD0042804BFAC462A
:10E70000102607D0022807BF04F1180C042604F1D4
:10E71000280C082606EB86169B8F0CEB860C6144B2
:10E72000EB2B20D944F2552C0B3303FB0CF39B0D40
:10E73000082807D0042802D0022805D008E02A467D
:10E74000102008E0402006E004F11802042002E056
:10E7500004F12802082000EB801002EB800000F595
:10E76000A57003FB001101F26510BDE8F08301F50F
:10E77000A571082804BF944640260CD0042804BF85
:10E78000AC46102607D0022807BF04F1180C042657
:10E7900004F1280C082606EB8616B3F844300CEB7F
:10E7A000860C6144EB2BDED944F2552C0B3303FB72
:10E7B0000CF39B0D0828C5D00428C0D00228C7D16F
:10E7C000C2E7FE4840F271210068806A4843704702
:10E7D000FA48006890F83500002818BF01207047FB
:10E7E00010B5F74C207B022818BF032808D1207DE4
:10E7F00004F115010DF023FC08281CBF012010BDF9
:10E80000207B002816BF022800200120BDE8104010
:10E8100009F054B9EA4908737047E849096881F872
:10E82000300070472DE9F047E44C2168087B002850
:10E8300016BF022800200120487301F10E0109F0E3
:10E8400027F92168087B022816BF0328012200222D
:10E8500081F82F204FF0080081F82D00487B01F14E
:10E860000E034FF001064FF00007012804BF5B794B
:10E8700013F0C00F0AD001F10E03012804D158791A
:10E8800000F0C000402801D0002000E0012081F805
:10E890002E00002A04BF91F8220010F0040F07D0C8
:10E8A000087D01F115010DF0CAFB216881F82D00EA
:10E8B0002068476006F0AAF92168C14D4FF00009B1
:10E8C000886095F82D000DF0D6FB804695F82F0056
:10E8D000002818BFB8F1000F04D095F82D000DF0F6
:10E8E00091F968B195F8300000281CBF95F82E000A
:10E8F00000281DD0697B05F10E0001290ED012E021
:10E900006E734A4605F10E01404609F016F995F876
:10E910002D1005F10E000DF0A5FC09E0407900F086
:10E92000C000402831D0394605F10E0009F03CF90D
:10E930002068C77690F8220010F0040F08BFBDE8E9
:10E94000F087002795F82D000DF010FA050008BF9C
:10E95000BDE8F08710210EF0C8F9002818BFBDE807
:10E96000F08720683A4600F11C01C676284609F077
:10E97000E4F8206800F11C0160680EF0DBFD6068BF
:10E98000BDE8F04701210EF0F0BD0DF0A8FC4A46AD
:10E9900005F10E0109F0D1F8CAE7884A1268137B25
:10E9A0000370D2F80E000860508A8880704778B5EE
:10E9B00083490446814D407B08732A682078107093
:10E9C0006088ADF8000080B200F00101C0F34003A0
:10E9D00041EA4301C0F3800341EA8301C0F3C0036D
:10E9E00041EAC301C0F3001341EA0311C0F340132D
:10E9F00041EA4311C0F3801041EA80105084E07D69
:10EA0000012808BF012607D0022808BF022603D02C
:10EA1000032814BFFFDF0826286880F85A60607E4C
:10EA2000012808BF012607D0022808BF022603D00C
:10EA3000032814BFFFDF0826286880F85B60217B6D
:10EA400080F82410418C1D290CBF0021616881626F
:10EA5000617D80F83510A17B002916BF02290021B5
:10EA600001210175D4F80F10C0F81510B4F8131077
:10EA7000A0F81910A17EB0F8662061F30302A0F897
:10EA80006620E17E012918BF002180F834100020A3
:10EA900078BD4A480068408CC0F3001131B1C0F322
:10EAA0008000002804BF1F20704702E0C0F340012F
:10EAB00009B10020704710F0010F14BFEE20FF20B5
:10EAC00070473E480068408CC0F3001119B1C0F394
:10EAD000800028B102E0C0F3400008B10020704778
:10EAE000012070473549002209680A664B8C1D2BAE
:10EAF0000CBF81F8642081F86400704700232F4A1E
:10EB0000126882F859309164A2F84C00012082F812
:10EB100059007047294A0023126882F85830A2F839
:10EB200054000120116582F8580070472349096894
:10EB300081F85D0070472148006890F95D007047DA
:10EB40001E48006890F82200C0F3401070471B4830
:10EB5000006890F82200C0F3C000704701207047A1
:10EB60001648006890F85B00704770B508F02CFA02
:10EB700008F00BFA08F00EF908F08CF90F4C206839
:10EB8000016E491C016690F83300002530B108F091
:10EB900031FA07F08CFC206880F83350206845700B
:10EBA00090F8371021B1BDE87040042009F06BBC2B
:10EBB00090F8641001B3006E814203E06000002011
:10EBC0000006002018D8042009F05DFC206890F8A9
:10EBD000220010F0010F07D0A06843220188BDE891
:10EBE00070400120FFF77EBBBDE8704043224FF626
:10EBF000FF710020FFF776BBBDE87040002009F0F0
:10EC000042BC2DE9F04782B00F468146FE4E4FF0E0
:10EC100000083068458C15F0030F10D015F0010F77
:10EC200005F0020005D0002808BF4FF0010806D00B
:10EC300004E0002818BF4FF0020800D1FFDF4FF0BA
:10EC4000000A544615F0010F05F002000DD080B9FE
:10EC500015F0040F0DD04AF00800002F1CBF40F043
:10EC6000010040F0020440D08FE010B115F0040F15
:10EC70000DD015F0070F10D015F0010F05F00200B0
:10EC800036D0002808BF15F0040F27D03DE0002F34
:10EC900018BF4AF0090478D134E02FB14AF00804D3
:10ECA00015F0200F14D070E0316805F02002B1F8A3
:10ECB0004400104308BF4AF0010466D04AF018042B
:10ECC00015F0200F61D191F85A10082959D155E05B
:10ECD000316891F85A10082950D152E04AF00800E2
:10ECE000002F18BF40F001044FD140F010044CE059
:10ECF000002818BF15F0040F07D0002F18BF4AF0E6
:10ED00000B0442D14AF018043FE015F0030F3BD149
:10ED100015F0040F38D077B131684AF0080091F847
:10ED20005A1008290CBF40F0020420F0020415F02C
:10ED3000200F21D029E0316805F02002B1F844000D
:10ED4000104308BF4AF003041FD04AF0180015F022
:10ED5000200F08D091F85A10082914BF40F002047F
:10ED600020F0020411E091F85A20082A14BF40F064
:10ED7000010020F00100EDE7082902D024F0010491
:10ED800003E044F0010400E0FFDF15F0400F1BD06A
:10ED9000C7B93168B1F84400002804BF488C10F0AE
:10EDA000010F0BD110F0020F08BF10F0200F05D19A
:10EDB00015F0010F08BF15F0020F03D091F85A00AB
:10EDC000082801D044F040047068A0F800A0017841
:10EDD00021F02001017007210EF078FB4146706898
:10EDE0000EF06BFD214670680EF073FD14F0010FFC
:10EDF0000AD006230022854970680EF044FD306871
:10EE0000417B70680EF0A4FB14F0020F18D0D6E915
:10EE10000010B9F1000F4FF006034FF0010207D0C8
:10EE20001C310EF030FD012170680EF09EFB07E0F2
:10EE300015310EF028FD3068017D70680EF095FBED
:10EE400014F0040F18BFFFDF14F0080F17D0CDF82F
:10EE500000A03068BDF800100223B0F86600020977
:10EE600062F30B01ADF800109DF80110032260F36E
:10EE700007118DF80110694670680EF004FD012F2E
:10EE800061D13068B0F84410E9B390F82200C0F3C3
:10EE90004000C0BB70680EF00CFD401CC7B230686B
:10EEA000B0F84420B0F85610551AC7F1FF018D4252
:10EEB000A8BF0D46AA423AD990F8220010F0010FDF
:10EEC00035D144F01004214670680EF002FDF81CA4
:10EED000C0B2ED1E284482B23068B0F86610036EEE
:10EEE000090951FA83F190F85C30494F1944BC4646
:10EEF0000023E1FB07C31B096FF0240C03FB0C117B
:10EF000080F85C1000E01EE090F85B00012101F049
:10EF100037F80090BDF800009DF80210032340EA86
:10EF200001400190042201A970680EF0ACFC306829
:10EF3000AAB2016C70680EF0FAFC3068B0F8561096
:10EF40002944A0F8561014F0400F06D0D6E900105E
:10EF5000012306225D310EF096FC14F0200F18BF3D
:10EF6000FFDF0020002818BFFFDF02B0BDE8F087F8
:10EF70002DE9F843244C2068002808BFFFDF2068F3
:10EF8000417839BB0178FF2924D0002680F8316010
:10EF9000A0F85660867080F83760304607F08EFF24
:10EFA00007F0B3FC206890F95D0007F048FD1948B0
:10EFB00007F04BFD184807F067FF606807F081FF16
:10EFC000206890F8240010F0010F06D0252007F0EB
:10EFD00044FD09E00C20BDE8F88310F0020F18BFD3
:10EFE000262075D007F039FD206890F85A102520AA
:10EFF00007F049FC206880F82C6007F059FF206872
:10F0000090F85A10002009E0600000200E06002051
:10F0100053E4B36EB05B0200AD5B020007F07BFD12
:10F020000F21052007F0DFFC206890F82E10002942
:10F0300001BF90F82F10002990F8220010F0040F63
:10F0400075D005F0E3FD054620682946806806F086
:10F05000F9FADFF83084074690FBF8F008FB1070EF
:10F060004142284605F0D3FA2168886097FBF8F002
:10F070004A68104448600CF0DFFF0146206842688F
:10F0800091426FD8C0E90165FF4D4FF0010895F836
:10F090002D000CF0F0FF814695F82F000127002885
:10F0A00018BFB9F1000F04D095F82D000CF0AAFD9F
:10F0B000A8B195F8300000281CBF95F82E00002854
:10F0C00025D0697B05F10E00012916D01AE0FFE773
:10F0D00010F0040F14BF2720FFDF83D184E73A46E6
:10F0E0006F7305F10E01484608F027FD95F82D10C5
:10F0F00005F10E000DF0B6F809E0407900F0C0000F
:10F10000402815D0414605F10E0008F04DFD20685D
:10F1100090F8220010F0040F24D095F82D000CF088
:10F1200025FE05001ED010210DF0DFFD40B119E0D5
:10F130000DF0D5F83A4605F10E0108F0FEFCE6E7C1
:10F1400020683A4600F11C01C776284608F0F5FC15
:10F15000206800F11C0160680EF0ECF90121606884
:10F160000EF003FA2068417B0E3007F020FC206887
:10F1700090F8581059B3B0F85410A0F84410016D2D
:10F18000016490F82210C1F30011E9B9B0F86600EB
:10F1900002210509ADF80050684606F011FE28B1BD
:10F1A000BDF80000C0F30B00A84204D1BDF8000078
:10F1B000401CADF800002168BDF80000B1F86620E1
:10F1C00060F30F12A1F86620206880F8586020686C
:10F1D00090F8591031B1B0F84C108187816C81637F
:10F1E00080F85960B0F86610026E090951FA82F190
:10F1F00090F85C20DFF894C2114463460022E1FBE2
:10F200000C3212096FF0240302FB031180F85C102A
:10F210000CF095FF032160680DF014F8216881F867
:10F2200033000020BDE8F8839949886070472DE9D4
:10F23000F043974C83B0226892F831303BB1508C48
:10F240001D2808BFFFDF03B0BDE8F0438DE40126B1
:10F250000027F1B1054692F85C0007F0FEFB20683C
:10F2600090F85B10FF2007F00EFB20684FF4A571AB
:10F2700090F85B20002007F050FD206890F82210E5
:10F2800011F0030F00F02E81002D00F0258100F019
:10F2900029B992F822108046D07EC1F300110029CE
:10F2A00056D0054660680780017821F02001017082
:10F2B000518C132937D01FDC102908BF022144D0FC
:10F2C000122908BF062140D0FFDF6F4D606805F1AD
:10F2D0000E010EF021F9697B60680EF039F92068A3
:10F2E000418C1D2918BF152965D0B0F84420016C48
:10F2F00060680EF046F95EE0152918BF1D29E3D1BC
:10F300004FF001010EF0E2F86068017841F0200151
:10F310000170216885B11C310EF00CF90121606883
:10F320000EF023F9D1E700210EF0D0F860680178E3
:10F3300041F020010170C8E715310EF0FBF820689C
:10F34000017D60680EF011F9BFE70EF0BFF8BCE771
:10F350000021FFF756FC6068C17811F03F0F2AD0FA
:10F36000017911F0100F26D00EF0AEF82368024696
:10F3700093F82410C1F38000C1F3400C604401F005
:10F38000010100EB010C93F82C10C1F38000C1F3D4
:10F390004005284401F001010844ACEB0000C1B273
:10F3A00093F85A0000F0ECFD009003230422694614
:10F3B00060680EF068FA2068002590F8241090F834
:10F3C0002C0021EA000212F0010F18BF01250ED116
:10F3D00011F0020F04D010F0020F08BF022506D072
:10F3E00011F0040F03D010F0040F08BF0425B8F18A
:10F3F000000F2BD0012D1BD0022D08BF26201BD0C3
:10F40000042D14BFFFDF272016D0206890F85A1073
:10F41000252007F038FA206890F82210C1F3001177
:10F4200069B101224FF49671002007F076FC0DE0DF
:10F43000252007F012FBE8E707F00FFBE5E790F85F
:10F440005A204FF49671002007F067FC206890F86E
:10F450002C10294380F82C1090F8242032EA010166
:10F460001DD04670418C13292CD027DC102904BFF5
:10F4700003B0BDE8F083122924D000BFC1F300100F
:10F48000002807E040420F000006002053E4B36E5E
:10F490006000002018BFFFDF03B0BDE8F083418C9F
:10F4A0001D2908BF80F82C70DBD0C1F300110029A2
:10F4B00014BF80F8316080F83170D2E7152918BF89
:10F4C0001D29DBD190F85A2003B04FF00101BDE8AF
:10F4D000F043084607F002BE90F85B200121084681
:10F4E00007F0FCFD2168002DC87E7CD04A8C3D468B
:10F4F000C2F34000002808BF47F0080512F0400F93
:10F5000018BF45F04005002819BFD1F83890B1F870
:10F510003C80D1F84090B1F84480606807210780B2
:10F520000DF0D4FF002160680EF0C7F9294660682D
:10F530000EF0CFF915F0080F15D02068BDF80010B7
:10F540000223B0F86600020962F30B01ADF8001067
:10F550009DF80110032260F307118DF80110694630
:10F5600060680EF090F960680EF06CF82168C0F1E8
:10F57000FE00B1F85620A8EB02018142A8BF014667
:10F58000CFB2D019404542D245F0100160680EF06C
:10F59000A0F960680EF056F82168C0F1FE00B1F8DD
:10F5A0005610A8EB01018142A8BF0146CFB26068A6
:10F5B0000EF07FF93844421C2068B0F86610036EE4
:10F5C000090951FA83F190F85C30FF4D1944AC46BB
:10F5D0000023E1FB05C31B096FF0240C03FB0C1196
:10F5E00080F85C1000E038E090F85B00012100F04A
:10F5F000C7FC0090BDF800009DF80210032340EA0C
:10F6000001400190042201A960680EF03CF92168D4
:10F6100091F8220010F0400F05D0012306225D3141
:10F6200060680EF030F920683A46B0F8560000EBFA
:10F63000090160680EF07BF92068B0F85610394473
:10F64000A0F8561008F0D0F8002818BFFFDF206897
:10F650004670867003B0BDE8F0830121FFF7D1FA50
:10F66000F0E7DA4810B50068417841B90078FF2822
:10F6700005D000210846FFF7DAFD002010BD07F095
:10F68000A3FC07F082FC07F085FB07F003FC0C20CD
:10F6900010BD10B5CD4C206890F8220010F0010F7D
:10F6A0001CBFA06801884FF03C0212BF01204FF63A
:10F6B000FF710020FEF716FE2168012081F8370057
:10F6C00010BDC249096881F8320070472DE9F04148
:10F6D000002508F0A4FE002800F00581BB4C20683E
:10F6E000417801270026012906D0022901D00329EB
:10F6F0007ED0FFDFBDE8F081817802260029418CB1
:10F7000046D0C1F34002002A08BF11F0010F70D0AB
:10F7100090F85B204FF001014FF0000007F0DEFC95
:10F72000216891F82200C0F34000002814BF0C208B
:10F73000222091F85B1007F0A6F82068467090F838
:10F74000330058B106F09FFE206890F85B0010F07F
:10F750000C0F0CBF4020452007F042FC206890F8B9
:10F760003400002818BF07F089FC216891F85B007D
:10F7700091F8651010F00C0F08BF0021962007F0DB
:10F78000C1FB08F028F8002818BFFFDFBDE8F081B2
:10F79000C1F3001282B110293FD090F8330020B19C
:10F7A00006F071FE402007F01BFC206890F8221044
:10F7B00011F0040F36D043E090F8242090F82C305C
:10F7C0009A422AD1B0F84400002808BF11F0010F76
:10F7D00005D111F0020F08BF11F0200F7ED04FF0BD
:10F7E00001014FF00000FFF722FD2068418C01E08D
:10F7F00040E034E011F0010F04BFC1F340010029E3
:10F8000007D1B0F85610B0F84420914218BFBDE8B7
:10F81000F08180F83170BDE8F081BDE8F041002151
:10F82000012004E590F83510012914BF03291025A3
:10F8300045F00E0190F85A204FF0000007F04EFC02
:10F84000206890F83400002818BF07F017FC00214A
:10F85000962007F057FB20684670BDE8F081B0F8AD
:10F860005610B0F8440081423DD0BDE8F04101217E
:10F870000846DCE48178D9B1418C11F0010F1CD02D
:10F8800080F8687090F86A20B0F86C100120FEF7DC
:10F8900029FD2068467007F097FB07F076FB07F01C
:10F8A00079FA07F0F7FABDE8F041032008F0EBBD64
:10F8B0008178BDE8F0410120B9E411F0020F04BFE6
:10F8C000FFDFBDE8F081B0F85610808F81420AD08A
:10F8D00001210846FFF7ABFC032000E003E02168AC
:10F8E0004870BDE8F081BDE8F041FFF73EB9FFF791
:10F8F0003CB910B5354C206890F8341049B1363019
:10F9000007F0CBFB18B921687F2081F8360007F09B
:10F91000ABFB206890F8330018B107F06BFB06F0E2
:10F92000C6FD08F07CFDA8B1206890F82210C1F354
:10F93000001179B14078022818BFFFDF00210120B3
:10F94000FFF775FC2068417800291EBF4078012828
:10F95000FFDF10BDBDE81040FFF707B92DE9F04704
:10F960001A4C0F4680462168B8F1030F488C08BF37
:10F97000C0F3400508D000F0010591F832000028DE
:10F9800018BF4FF0010901D14FF0000907F059F8F5
:10F990000646B8F1030F0CBF4FF002084FF0010804
:10F9A00035EA090008BFBDE8F087206890F8330009
:10F9B00090B10CF0A7FB38700146FF280CD06068AE
:10F9C000C01C0CF078FB03E053E4B36E6000002031
:10F9D00038780CF0A4FB064360680178C1F380120C
:10F9E00021680B7D9A4208D10622C01C153115F002
:10F9F000E5FD002808BF012000D000203978FF294C
:10FA000006D0C8B9206890F82D00884216D113E0BE
:10FA1000A0B1616811F8030BC0F380100CF00FFB6C
:10FA200005460CF06FFC38B128460CF09FF918B170
:10FA300010210DF05AF908B1012000E000202168E2
:10FA400091F8221011F0040F01D0F0B11AE0CEB9F4
:10FA5000FE4890F83500002818BF404515D1616870
:10FA600011F8030BC0F380100CF0E9FA04460CF017
:10FA700049FC38B120460CF079F918B110210DF08D
:10FA800034F910B10120BDE8F0870020BDE8F0870F
:10FA90002DE9F04FEE4D074683B0286800264078E8
:10FAA000022818BFFFDF28684FF07F0990F8341054
:10FAB00049B1363007F0F1FA002804BF286880F811
:10FAC000369007F0D1FA68680DF022FD0446002F49
:10FAD00000F0048268680DF0A6FE002800F0FE81A8
:10FAE00006F07DFF002800F0F981FF20DFF864B305
:10FAF000DFF8588300274FF0010A062C80F00082BF
:10FB0000DFE804F0EFEFEF03EFF78DF80000694650
:10FB10000320FFF723FF002800F0E480296891F814
:10FB2000340010B191F89800D0B12868817801298B
:10FB30004CD06868042107800DF0C8FC08F10E0164
:10FB400068680DF0E9FC98F80D1068680DF000FD8C
:10FB50002868828F816B68680DF037FD00F04DB921
:10FB60009DF8000081F898A00A7881F89920FF2874
:10FB70000FD001F19B029A310CF086FA002808BFE1
:10FB8000FFDF286890F89A1041F0020180F89A107F
:10FB90000DE068680278C2F3801281F89A20D0F8EC
:10FBA0000320C1F89B20B0F80700A1F89F00286847
:10FBB00000F1A10490F836007F2808BFFFDF286815
:10FBC00090F83610217080F83690AEE790F8220059
:10FBD0009BF80490C0F38014686864F386190721C9
:10FBE00007800DF073FC002168680DF066FE494641
:10FBF00068680DF06EFE0623002208F10E016868A9
:10FC00000DF041FE2868417B68680DF0A1FC686832
:10FC10000DF018FD29688A8FC0F1FE018A42B8BF35
:10FC20001146CFB2BA423DD9F81EC7B249F0100A08
:10FC3000514668680DF04DFE68680DF03AFE384494
:10FC4000431C2868B0F86610026E090951FA82F167
:10FC500090F85C20DFF800920A44C8464FF0000C90
:10FC6000E2FB098C4FEA1C116FF0240C01FB0C2104
:10FC700080F85C1090F85B001A46012100F080F9D2
:10FC80000190BDF804009DF80610032340EA0140EE
:10FC90000290042202A968680DF0F5FD51466868DB
:10FCA0000DF017FE34B1D5E90010012306225D31B5
:10FCB0000DF0E9FD28683A46816B68680DF037FE63
:10FCC0002868A0F85670818F8F420CBF0121002157
:10FCD00080F8311007F088FD002818BFFFDF8CE0A6
:10FCE00007E00DE128688078002840F0F98000F0F6
:10FCF000F5B88DF8000068680178C1F38019D0F874
:10FD000003100191B0F80700ADF80800694605201E
:10FD1000FFF724FE0028286873D08178002972D06C
:10FD200090F85BA0D5E90104D0F80F10C4F80E10CC
:10FD3000B0F813106182417D2175817D6175B0F845
:10FD40001710E182B0F819106180B0F81B10A18083
:10FD5000B0F81D10E18000F11F0104F1080015F05A
:10FD60000EFE686890F8241001F01F01217690F8CB
:10FD70002400400984F86C0184F854A084F855A04C
:10FD8000286890F8651084F8561090F85D0084F8A3
:10FD900057009DF80010A86800F05BF9022008F0F9
:10FDA00072FB6868DBF800400DF1040A0780082147
:10FDB0000DF08CFB002168680DF07FFD214668681E
:10FDC0000DF087FD0623002208F10E0168680DF092
:10FDD0005AFD2868417B68680DF0BAFB494668689F
:10FDE0000DF0C3FB06230122514668680DF04BFD60
:10FDF00007F0FAFC002818BFFFDF032029684870CD
:10FE000070E066E0FFE76868AC684FF001080278D0
:10FE1000617BC2F3401211406173D0F80F10C4F837
:10FE20000E10B0F813106182417D2175817D6175DE
:10FE3000B0F81710E182B0F819106180B0F81B100B
:10FE4000A180B0F81D10E18008E00000000600204D
:10FE500060000020A85B020053E4B36E00F11F01B4
:10FE600004F1080015F08BFD686890F8241001F08B
:10FE70001F01217690F82400400984F86C0184F871
:10FE8000548084F85580286890F8651084F85610DE
:10FE900090F85D0084F857009DF80010A86800F005
:10FEA000D8F8286880F868A090F86A20B0F86C103C
:10FEB0000120FEF717FA2868477007F085F807F069
:10FEC00064F806F067FF06F0E5FF012008F0DBFAB2
:10FED00008E090F82200C0F3001008B1012601E00C
:10FEE000FEF743FE286890F8330018B107F082F857
:10FEF00006F0DDFA66B100210120FFF798F910E065
:10FF0000286890F82200C0F300100028E8D0E5E748
:10FF100028688178012904D190F85B10FF2006F051
:10FF2000B2FC28684178002919BF4178012903B043
:10FF3000BDE8F08F4078032818BFFFDF03B0BDE8AD
:10FF4000F08F70B57E4C06460D462068807858B11B
:10FF500006F04FFC21680346304691F85B202946A5
:10FF6000BDE8704009F042B806F043FC2168034642
:10FF7000304691F85A202946BDE8704009F036B85D
:10FF800078B50C4600210091082804BF4FF4C870D2
:10FF900040210DD0042804BF4FF4BF70102107D0BA
:10FFA000022807BF01F11800042101F128000821EF
:10FFB000521D02FB010562489DF80010006890F890
:10FFC0005C2062F3050141F040068DF8006090F876
:10FFD0005B00012828D002282DD0082818BFFFDF99
:10FFE0002FD000BF26F080008DF80000C4EB041075
:10FFF00000EB80001E2101EB800005FB040451484A
:020000040001F9
:10000000844228BFFFDF5048A0FB0410BDF8011058
:10001000000960F30C01ADF80110BDF800009DF877
:10002000021040EA014078BD9DF8020020F0E00097
:100030008DF80200D6E79DF8020020F0E0002030A5
:1000400004E09DF8020020F0E00040308DF802004E
:10005000C8E72DE9F0413A4D04460E46286890F86D
:100060006800002818BFFFDF0027286880F86A7042
:100070002188A0F86C106188A0F88210A188A0F8EF
:100080008410E188A0F8861094F86C1180F888102C
:1000900090F82F1049B1427B00F10E01012A04D1E2
:1000A000497901F0C001402934D090F8301041B1B5
:1000B000427B00F10E01012A04BF497911F0C00F03
:1000C00028D000F1760015F051FC6868FF2E017809
:1000D000C1F380116176D0F80310C4F81A10B0F89B
:1000E0000700E08328681DD0C167E18BA0F880106D
:1000F00000F17002511E30460BF0C6FF002808BF09
:10010000FFDF286890F86F1041F0020180F86F104F
:10011000BDE8F081D0F80E10C0F87610418AA0F842
:100120007A10D2E7C767A0F88070617E80F86F1000
:10013000D4F81A100167E18BA0F87410BDE8F081C3
:1001400060000020C4BF0300898888880178406867
:1001500029B190F80C1190F8730038B901E001F062
:10016000A9BD19B1042901D00120704700207047B2
:1001700070B50C460546062102F006FC606008B129
:10018000002006E00721284602F0FEFB606018B15F
:1001900001202070002070BD022070BD2DE9FC47B9
:1001A0000C4606466946FFF7E3FF00287DD19DF81F
:1001B000000050B1FEF727F9B0427CD0214630460E
:1001C0000AF000F9002873D12DE00DF02FFEB042A7
:1001D00071D02146304612F093FF002868D1019D6E
:1001E00095F8D00022E0012000E00020804695F83C
:1001F00037004FF0010A4FF00009F0B195F83800D0
:1002000080071AD584F8019084F800A084F804903F
:10021000E68095F839102172698F6181A98FA181DB
:1002200085F8379044E0019D95F80C015835002879
:10023000DBD1E87E0028D8D0D5E7304602F0E8FCD4
:10024000070000D1FFDF384601F0F8FE40B184F826
:1002500001900F212170E680208184F804A027E01E
:10026000304602F0C3FC070000D1FFDFB8F1000FF9
:1002700021D0384601F039FFB8B19DF8000038B9F7
:100280000198D0F8F8004188B14201D180F800907F
:10029000304607F07CFB84F801900C21217084F833
:1002A0000490E680297F217200E004E085F81B902D
:1002B0000120BDE8FC870020FBE71CB56946FFF77D
:1002C00057FF00B1FFDF684601F000FDFB49002049
:1002D0008968A1F8D2001CBD2DE9FC4104460E46F8
:1002E000062002F0F9FA0546072002F0F5FA284444
:1002F000C7B20025A8463E4417E02088401C80B2C3
:100300002080B04202D34046A4F8008080B2B842B8
:1003100004D3B04202D20020BDE8FC816946FFF759
:1003200027FF0028F8D06D1CEDB2AE42E5D84FF69D
:10033000FF7020801220EFE738B54FF6FF70ADF860
:1003400000000DE00621BDF8000002F02FFB04467E
:100350000721BDF8000002F029FB0CB100B1FFDF5E
:1003600000216846FFF7B8FF0028EBD038BD70B514
:1003700007F07AFB0BF04FFCD14C4FF6FF760025CF
:100380006683A683CFA0257001680079A4F140029E
:10039000657042F8421FA11C1071601C13F07DF8BB
:1003A00025721B2060814FF4A471A181E08121821C
:1003B0000321A1740422E274A082E082A4F13E0031
:1003C000218305704680BD480C300570A4F11000F3
:1003D0000570468070BD70B5B84C16460D4660601D
:1003E000217007F0BBFAFFF7A7FFFFF7C0FF2078E7
:1003F00010F09BFEB5480EF0C4F92178606812F049
:100400005EFF20780AF056FE284608F097FBAF48BA
:10041000FEF704F8217860680AF0BAF831462078CF
:1004200013F038FEBDE870400BF0F5BB10B50124A9
:100430000AB1002010BD21B1012903D000242046BB
:1004400010BD02210DF0B0FAF9E72DE9F0470400E4
:1004500000D1FFDF9A4802211C308146FFF73CFFA4
:1004600000B1FFDF964D0620B5F81C8002F034FA8B
:100470000646072002F030FA3044C6B2701CC7B2FC
:10048000A88BB04228D120460DF046FCB0B12078B0
:1004900018283FD1207901283CD1E088062102F0BC
:1004A00073FA040000D1FFDF208807F070FA20887B
:1004B000062102F07BFA40B3FFDF2BE0287860B31F
:1004C00000266670142020702021201D15F043F9AD
:1004D000022020712E701DE0B84217D12046FDF792
:1004E00037FFD0B12078172814D1207968B1E0887F
:1004F000072102F049FA40B1008807F048FAE08885
:10050000072102F053FA00B1FFDF03E02146FFF7B5
:1005100045FE10B10120BDE8F08702214846FFF7F3
:10052000DBFE10B9A98B4145AAD12046BDE8F047B2
:1005300013F0F6BD10B501F064FB08B10C2010BD3E
:100540000BF0BCFB002010BD10B50446007818B1BC
:10055000012801D0122010BD01F064FB20B10BF086
:100560005DFD08B10C2010BD207801F011FBE21DEB
:1005700004F11703611CBDE810400BF044BC10B53A
:10058000044601F03EFB08B10C2010BD207828B1D4
:10059000012803D0FF280BD0122010BD01F0F8FA7B
:1005A000611C0BF04BFB08B1002010BD072010BDF3
:1005B00001200BF07DFBF7E710B50BF032FD08B121
:1005C000002010BD302010BD10B5044601F02AFBFC
:1005D00008B10C2010BD20460BF01DFD002010BD01
:1005E00010B501F01FFB20B10BF018FD08B10C2075
:1005F00010BD0BF06DFC002010BDFF2181704FF687
:10060000FF7181802D4949680A7882718A88028148
:100610004988418101214170002070477CB5002547
:10062000022A19D015DC12F10C0F15D009DC12F1D9
:10063000280F11D012F1140F0ED012F1100F11D19A
:100640000AE012F1080F07D012F1040F04D04AB9E2
:1006500002E0D31E052B05D8012806D0022808D0B9
:1006600003280AD0122528467CBD1046FEF75EFA04
:10067000F9E710460EF030F8F5E7084614466946EB
:10068000FFF776FD08B10225EDE79DF8000001981F
:10069000002580F85740E6E710B5134601220CF01C
:1006A00061FB002010BD10B5044611F03AFB05288F
:1006B0000ED0204610F028FD002010BD6C00002058
:1006C000E4070020FFFFFFFF1F000000A40600203A
:1006D0000C20F2E710B5044601F0A4FA08B10C2092
:1006E000EBE72146002007F0C0F90020E5E710B550
:1006F000044610F097FD50B108F0A6FC38B1207800
:1007000008F041FA20780EF0F5FA0020D5E70C2029
:10071000D3E710B5044601F085FA08B10C20CCE708
:100720002146012007F0A1F90020C6E738B50446AC
:100730004FF6FF70ADF80000A079E179884216D03D
:100740002079FDF766FD90B16079FDF762FD70B12B
:100750000022A079114614F011F940B90022E07985
:10076000114614F00BF910B9207A072801D912208C
:1007700038BD08F076FC60B911F0D3FA48B9002111
:100780006846FFF7A9FD20B1204606F057F8002083
:1007900038BD0C2038BD2DE9FC41817805461A2969
:1007A00025D00EDC16292DD2DFE801F02C2C2C2CC4
:1007B0002C212C2C2C2C2C2C2C2C2C2C2C2C2C218F
:1007C00021212A291ED00BDCA1F11E010C2919D2EE
:1007D000DFE801F018181818181818181818180D4C
:1007E0003A3904290ED2DFE801F00D020D02288803
:1007F000B0F5706F06D201276946FFF7B9FC18B152
:10080000022089E5122087E59DF8000001F0C7F974
:10081000019C08B1F43401E004F5B8749DF80000BF
:1008200001F0BDF9019E08B1F53601E006F271163E
:100830006846FFF78BFC08B1207808B10C206BE507
:100840002770A8783070684601F040FA002063E510
:100850007CB50D466946FFF78BFC002618B12E606B
:100860002E7102207CBD9DF8000001F098F9019CDA
:100870009DF80000583401F092F9019884F8406026
:1008800081682960017B297194F840100029F5D115
:1008900000207CBD70B5044691F8550091F85630A3
:1008A0000D4610F00C0F00D100232189A0880CF018
:1008B000E8FB696A81421DD2401A401CA1884008A9
:1008C000091A8AB2A2802189081A2081668895F8BF
:1008D000541010460CF07CFB864200D230466080FB
:1008E000E68895F8551020890CF072FB864200D2FC
:1008F0003046E08070BDF0B585B00D46064603A9D0
:10090000FFF736FC00282DD19DF80C0060B30022C3
:100910000499FB20B1F84A30FB2B00D30346B1F811
:100920004C40FB20FB2C00D30446DFF80CCC9CE8A9
:10093000811000900197CDF808C0ADF80230ADF8F5
:1009400006406846FFF7A6FF6E80BDF80400E88009
:10095000BDF808006881BDF80200A880BDF8060057
:100960002881002005B0F0BD0122D1E72DE9F0413A
:1009700086B0044600886946FFF7FAFB002868D174
:100980002189E08801F0B1F9002862D1A18860884E
:1009900001F0ABF900285CD12189E08801F0B3F9BE
:1009A000002856D1A188608801F0ADF9070050D128
:1009B000208802A9FFF79FFF00B1FFDFBDF81010EC
:1009C00062880920914244D3BDF80C10E28891421C
:1009D0003FD3BDF81210BDF80E2023891144A28820
:1009E0001A44914235D39DF80000019D4FF0000854
:1009F000012640B185F89B61019890F8DE0105F56C
:100A0000CD7540B914E085F80561019890F828018A
:100A100005F5827508B13A2718E0E088688060889B
:100A2000E8802089A880A08828810122019909E016
:100A3000E08868806088E8802089A880A088288174
:100A4000019900222846FFF725FF2E7085F80180C6
:100A5000384606B0BDE8F08188E710B5044601F0DD
:100A6000E1F820B10BF0DAFA08B10C2025E6207885
:100A700001F08EF8E279611C0BF051FC08B1002006
:100A80001BE6022019E610B503780446002B4068E7
:100A900013460A46014609D05FF001000CF0FAFA4D
:100AA0006168496A884203D9012006E60020F5E71B
:100AB000002002E62DE9F04117468A781E4680465E
:100AC00042B11546C87838B10446690706D52AB13F
:100AD000012104E00725F5E70724F6E70021620776
:100AE00002D508B1012000E00020014206D0012219
:100AF00011464046FFF7C7FF98B93BE051B10022CD
:100B000001214046FFF7BFFF58B9600732D50122E7
:100B100011461FE058B1012200214046FFF7B3FF04
:100B200008B1092096E7680724D5012206E0680786
:100B30004FEA44700AD5002813DB00220121404609
:100B4000FFF7A1FFB0B125F0040513E0002811DA8A
:100B5000012200214046FFF796FF58B124F004041B
:100B600008E0012211464046FFF78DFF10B125F045
:100B70000405F3E73D70347000206BE710B586B0D4
:100B80000446008803A9FFF7F3FA002806D1A088DD
:100B900030B1012804D0022802D0122006B08CE522
:100BA0006B4602AA214603A8FFF784FF0028F5D16F
:100BB0009DF80C3000220121002B049B06D083F805
:100BC000A511049B93F8F2316BBB24E083F80F115D
:100BD000049B93F834313BB9049B93F80E311BB955
:100BE000049B93F87D300BB13A2010E0049B83F80E
:100BF0000E11049B9DF8081083F81011049B9DF8BA
:100C0000001083F81111049BA188A3F81211049914
:100C100081F80F21C2E7049B93F8A4311BB9049B10
:100C200093F87D300BB13A2010E0049B83F8A411B7
:100C3000049B9DF8081083F8A611049B9DF80010F2
:100C400083F8A711049BA188A3F8A811049981F83F
:100C5000A521A3E710B504460020A17801B9012021
:100C6000E2780AB940F0020001F056F8002803D1FA
:100C70002046BDE8104081E71FE570B51C460D46D3
:100C800018B1012801D0122070BD1946104601F09C
:100C900053F830B12146284601F058F808B1002039
:100CA00070BD302070BD70B5044600780E46012836
:100CB00004D018B1022801D0032841D1607828B1AE
:100CC000012803D0022801D0032839D1E07B10B9D4
:100CD000A078012834D1A07830F0050130D110F08F
:100CE000050F2DD06289E188E0783346FFF7C5FF14
:100CF000002826D1A07805281ED16589A2892189DE
:100D000020793346FFF7B9FF00281AD15FF00100C0
:100D100004EB40014A8915442218D3789278934213
:100D20000ED1CA8889888A420AD1401CC0B20228E2
:100D3000EED3E088A84203D3A07B08B1072801D9ED
:100D4000122070BD002070BD10B586B0044600F0C2
:100D50004BFF08B10C2021E7022104F10A0001F049
:100D600008F8A0788DF80800A0788DF80000607869
:100D70008DF8040020788DF80300A07B8DF8050025
:100D8000E07B00B101208DF80600A078C10717D0E4
:100D9000E07800F0E5FF8DF80100E088ADF80A008A
:100DA0006089ADF80C00A078400716D5207900F0D6
:100DB000D7FF8DF802002089ADF80E00A0890AE067
:100DC00040070AD5E07800F0CBFF8DF80200E088FC
:100DD000ADF80E006089ADF8100002A810F02EFAF0
:100DE0000028B8D168460DF08AFFD7E610B5044652
:100DF0000121FFF758FF002803D12046BDE810402D
:100E0000A2E75AE40278012A01D0BAB118E0427888
:100E10003AB1012A05D0022A12D189B1818879B16B
:100E200000E059B1418849B1808838B101EB8101B6
:100E3000490000EB8000B1EB002F01D20020704789
:100E40001220704770B5044600780D46012809D07D
:100E500010F067FF052803D010F001F9002800D03A
:100E60000C2070BD0DF00DFE88B10DF01FFE0DF0D1
:100E700023FF0028F5D125B160780DF0B4FE0028DD
:100E8000EFD1A1886088BDE8704010F0FDB9122054
:100E900070BD10B504460121FFF7B4FF002804D14E
:100EA0002046BDE810400121CCE706E42DE9F047DB
:100EB0000746B0F84C50FB2092460E46FB2D00D35F
:100EC0000546DFF87886B8F80A00A84200D2054641
:100ED00097F85510284600F076FEB8F80C108142BD
:100EE00000D208468146B7F84A40FB20FB2C00D3CD
:100EF0000446B8F80E00A04200D2044697F85410F9
:100F0000204600F060FEB8F81010814200D208467A
:100F10004FF4A4721B2C01D0904203D11B2D25D07D
:100F2000914523D0F580A6F808907480B080524691
:100F300039463046FFF7AEFC01203070F0881B3890
:100F4000E02800D9FFDF70881B38E02800D9FFDFD8
:100F5000308940F64814A0F5A470A04200D9FFDF04
:100F6000B088A0F5A470A04200D9FFDFBDE8F087EB
:100F7000F0B5871FDDE9056540F67B44A74213D233
:100F80008F1FA74210D288420ED8B2F5FA7F0BD23B
:100F9000A3F10A00241FA04206D2521C4A43B2EB1E
:100FA000830F01DAAE4201D90020F0BD0120F0BD6F
:100FB0002DE9FC47477A0446884678077ED0F80832
:100FC0007CD194F83A0008B9012F77D100252E463C
:100FD000F90788F0010919D0208A494600F0ACFED3
:100FE000F0B36089494600F0B1FEC8B3208A618938
:100FF000884263D8A18EE08DCDE90001238D628CFB
:10100000A18BE08AFFF7B4FF50B30125B8070ED5D6
:1010100004EB4500828EC18DCDE90012038D428C18
:10102000818BC08AFFF7A4FFD0B16D1C2E467807D4
:101030001DD504EB45074946388A00F07DFE78B19E
:101040007889494600F082FE50B1388A7989884211
:1010500057D8B98EF88DCDE900013B8D7A8C00E030
:1010600009E0B98BF88AFFF783FF20B16D1CB8F156
:10107000000F03D02AE03020BDE8FC87228A01213E
:101080001FE0B14203D004EB4100008A024404EBAC
:101090004100C38A878ABB4233D1838B478BBB42D3
:1010A0002FD1438C078CBB422BD1038DC78CBB4205
:1010B00027D143890089834223D100E021E0491CE4
:1010C000C9B2A942DDD3608990421AD3207810B109
:1010D000012816D10DE0A078B8F1000F07D040B17B
:1010E000012806D0022804D003280AD101E00028F4
:1010F000EED1607838B1012805D0022803D003284A
:1011000001D01220B8E70020B6E7002150E70178AF
:10111000C90702D0406812F0D6BF12F0A3BF2DE974
:10112000F04788B00D46AFF66422D2E9009201463E
:1011300090462846FFF73CFF06000CD100F054FD16
:1011400040B9FE4F387828B90CF070FEA0F57F4109
:10115000FF3902D00C2008B008E7032105F1100088
:1011600000F007FEF54801AA3E380190F4480290CD
:10117000F24806211038039007A801F0D3FB0400C1
:1011800035D003210BF04EFBB98AA4F84A10FA8A35
:10119000A4F84C20FB7C0093BA46BB7C208801F06D
:1011A000AEFC00B1FFDF208806F0F0FB218804F1DF
:1011B0000E0000F041FDE3A004F11207006800906A
:1011C0000321684604F0F2FD002069460A5C3A54A7
:1011D000401CC0B20328F9D3A88B6080688CA08023
:1011E000288DE080687A410703D508270AE00920A6
:1011F000B1E7C10701D0012704E0800701D502272C
:1012000000E000273A46BAF81800114610F0D0F86E
:101210000146A062204610F0D9F817F00C0F09D053
:1012200001231A46214600200BF034FF616A8842F0
:1012300000D90926002784F85E7084F85F70A878CA
:1012400000F0A6FC6076D5F80300C4F81A00B5F8E3
:101250000700E083C4F8089084F80C80012084F82B
:101260000001024604F582712046FFF71FFE8DF84B
:1012700000700121684604F099FD9DF8000000F01F
:101280000701C0F3C1021144C0F3401008448DF8B7
:101290000000401D2076092801D208302076002168
:1012A00020460BF0BFFA68780DF0F6FBF6BBA97884
:1012B0002878EA1C0DF0C3FB48B10DF0F7FBA978C4
:1012C0002878EA1C0DF069FC060002D052E01226D4
:1012D00050E0687A00F005010020CA0700D0012024
:1012E0008A0701D540F00200490701D540F0080007
:1012F0000DF08EFB06003DD1214603200DF077FC5A
:10130000060037D10DF07DFC060033D1697A01F07B
:1013100005018DF81010697AC90706D06889ADF803
:101320001200288AADF81400012000E022E0697A5A
:101330008A0700D5401C490707D505EB40004189C5
:10134000ADF81610008AADF8180004A80FF076FF6B
:10135000064695F83A0000B101200DF06BFB4EB93E
:101360000DF0AAFC060005D1A98F20460FF008FF5A
:10137000060008D0208806F00AFB2088062101F02C
:1013800015FB00B1FFDF3046E5E601460020C6E66A
:1013900038B56A48007878B910F0C3FC052805D044
:1013A0000CF044FDA0F57F41FF3905D068460FF0F1
:1013B000AEFF040002D00CE00C2038BD009800887D
:1013C00006F0E5FA00980621008801F0EFFA00B176
:1013D000FFDF204638BD1CB582894189CDE9001266
:1013E0000389C28881884088FFF7C2FD08B10020C8
:1013F0001CBD30201CBD70B50546FFF7ECFF002872
:101400000ED12888062101F0BFFA040007D000F0B1
:1014100051FC20B1D4F8F800017831B901E0022084
:1014200070BDD4F84411097809B13A2070BD052186
:101430008171D4F8F81000200881D4F8F810A88839
:101440004881D4F8F810E8888881D4F8F810288901
:10145000C881D4F8F800028941898A4204D8827987
:10146000082A01D88A4201D3122070BD2988418000
:10147000D4F8F81002200870002070BD3EB5044674
:101480000BF002FCB0B12D480125A0F140024570DF
:10149000236842F8423F2379002113714170694665
:1014A000062001F0FAF900B1FFDF684601F0D3F938
:1014B00010B10EE012203EBDBDF80440029880F845
:1014C0000051684601F0C7F918B9BDF80400A04200
:1014D000F4D100203EBD70B505460088062101F01C
:1014E00053FA040007D000F0E5FB20B1D4F8F8105F
:1014F000087830B901E0022070BDD4F844010078CA
:1015000008B13A2070BD9620005D10F0010F21D087
:10151000D5F802004860D5F80600886054F8F80F46
:10152000698910228181206805F10C010E3014F0C8
:1015300071F80320216807E0CC5B0200E40700207B
:101540007800002011223300087021682888488024
:10155000002070BD0C2070BD38B504460078EF281F
:101560004DD86088ADF80000009800F013FC88B3F7
:101570006188080708D4D4E9012082423FD8202A94
:101580003DD3B0F5804F3AD8207B18B3072836D822
:10159000607B28B1012803D0022801D003282ED176
:1015A0004A0703D4022801D0032805D1A07B08B143
:1015B000012824D1480707D4607D28B1012803D031
:1015C000022801D003281AD1C806E07D03D50128DE
:1015D00015D110E013E0012801D003280FD1C8066F
:1015E00009D4607E012803D0022801D0032806D147
:1015F000A07E0F2803D8E07E18B1012801D0122068
:1016000038BD002038BDF8B514460D46064607F033
:1016100028FD08B10C20F8BD3046FFF79DFF0028DB
:10162000F9D1FDF788FA2870B07554B9FF208DF80C
:10163000000069460020FDF76DFA69460020FDF7BD
:101640005DFA3046BDE8F840FDF7B1B90022DAE7AF
:1016500070B50C46054612B11F2907D80CE0FF2CC7
:1016600004D8FCF71EFF18B11F2C01D9122070BD41
:101670002846FCF700FF08B1002070BD422070BD75
:1016800010B50446408810B1FDF71BFA78B12078F8
:10169000618800F001026078FFF7DAFF002805D1C9
:1016A000FDF7F7F96288824203D9072010BD1220A6
:1016B00010BD10466168FDF72DFA002010BD10B571
:1016C0000446408810B1FCF7DEFE70B120786188D6
:1016D00000F001026078FFF7BBFF002804D16088AA
:1016E0006168FDF70BFA002010BD122010BD7CB51B
:1016F000044640784225012808D8A078FCF7BBFEB4
:1017000020B120781225012802D090B128467CBD56
:10171000FDF71DFA20B1A0880028F7D08028F5D861
:10172000FDF71CFA60B160780028EFD0207801281E
:1017300008D006F04BFA044607F05DF900287DD08A
:101740000C207CBDFDF74CF810B9FDF7F9F990B30A
:1017500007F087FC0028F3D1FCF755FEA0F57F4188
:10176000FF39EDD1FDF75EF8A68842F210704643CE
:10177000A079FDF7B7F9FCF78DFEF8B1002207213B
:1017800001A801F0CFF8040043D0F748032184609A
:1017900020460AF052FF2046FDF746FDF34DA88A89
:1017A000A4F84A00E88AA4F84C00FCF77AFE60B17D
:1017B000288B01210DE0FFE712207CBD314600207F
:1017C00007F0E4F9D8B3FFDF4CE0FDF7C9F90146B3
:1017D000288B07F086FA0146A0620022204606F018
:1017E000F8F9FCF75EFEB0B9FDF7BAF910F00C0F8E
:1017F00011D001231A46214618460BF04BFC616AB2
:10180000884208D90721BDF8040001F0CFF800B1E3
:10181000FFDF09207CBDE87C0090AB7CEA8AA98AC6
:10182000208801F06CF900B1FFDF208806F0AEF8E7
:101830003146204607F0AAF918B101E008E011E0AE
:10184000FFDF002204F5CD712046FFF72FFB09E0F2
:1018500044B1208806F09BF82088072101F0A6F803
:1018600000B1FFDF00207CBD002140E770B50D46D0
:10187000072101F089F8040003D094F8730110B136
:101880000AE0022070BD94F86500142801D01528E4
:1018900002D194F8C00108B10C2070BD1022294675
:1018A00004F5BA7013F0B6FE012084F8730100202D
:1018B00070BD10B5072101F067F818B190F87311E9
:1018C00011B107E0022010BD90F86510142903D073
:1018D000152901D00C2010BD022180F873110020C1
:1018E00010BD2DE9FC410C464BF68032122194428A
:1018F0001DD8E4B16946FEF73BFC002815D19DF8E0
:10190000000000F04CF9019E9DF80000583600F0F0
:1019100046F9019DAD1C2F882246394630460AF013
:1019200082FE2888B842F6D10020BDE8FC81084636
:10193000FBE77CB5044600886946FEF719FC0028E1
:1019400010D19DF8000000F02AF9019D9DF80000DB
:10195000583500F024F90198A27890F82C109142A3
:1019600001D10C207CBD7F212972A9720021E9726E
:10197000E17880F82D10217980F82E10A17880F878
:101980002C1000207CBD1CB50C466946FEF7F0FB10
:1019900000280AD19DF8000000F001F9019890F8A4
:1019A000730000B10120207000201CBD7CB50D46E5
:1019B00014466946FEF7DCFB002809D19DF80000BB
:1019C00000F0EDF8019890F82C00012801D00C20CF
:1019D0007CBD9DF8000000F0E2F8019890F86010DE
:1019E000297090F86100207000207CBD70B50D4614
:1019F0001646072100F0C8FF18B381880124C38868
:101A0000428804EB4104AC4217D842F2107463439D
:101A1000A4106243B3FBF2F2521E94B24FF4FA7276
:101A2000944200D91446A54200D22C46491C641C9D
:101A3000B4FBF1F24A43521E91B290F8AC211AB9AC
:101A400001E0022070BD01843180002070BD10B51E
:101A50000C46072100F098FF48B180F8DF4024B120
:101A600090F8DD1009B107F052F9002010BD0220F6
:101A700010BD017899B1417889B141881B290ED3F5
:101A800081881B290BD3C188022908D337490268F2
:101A9000403941F8522F40684860002070471220BA
:101AA000704710B504460FF07FFC204607F0E8F8B9
:101AB000002010BD10B507F0E6F8002010BD2DE99C
:101AC000F04115460F4606460122114638460FF0F2
:101AD0006FFC04460121384607F003F9844200D226
:101AE000044601213046653C00F05EF806460121BF
:101AF000002000F059F8304401219630844206D984
:101B000000F19601201AB0FBF1F0401C81B229804F
:101B10000020BDE8F08110B5044600F083F808B15C
:101B20000C2010BD601C0AF0D5FB207800F00100ED
:101B3000FCF773FE207800F001000CF0B2FF0020EB
:101B400010BD10B50446072000F0B8FE08B10C2007
:101B500010BD2078C00715D000226078114612F021
:101B60000DFF28B1122010BD6C000020E4070020FA
:101B7000A06809F06AF86078D4F8041009F06EF8EB
:101B80000020F0E7002009F060F800210846F5E7A2
:101B900018B1022801D0012070470020704708B119
:101BA000002070470120704710B5012904D0022998
:101BB00005D0FFDF2046D6E7C000503001E08000AE
:101BC0002C3084B2F6E711F00C0F04D04FF474718E
:101BD00001EB801006E0022902D0C000703001E065
:101BE00080003C3080B2704710B510F09AF804289D
:101BF00005D010F096F8052801D00020B3E70120A9
:101C0000B1E710B5FFF7F0FF10B10DF019F828B9E2
:101C100007F027FA20B1FCF7DBFD08B10120A2E7AD
:101C20000020A0E710B5FFF7DFFF18B907F019FA99
:101C3000002898D0012096E72DE9FE4300250F46A5
:101C400080460A260421404604F0D9F840460AF0AE
:101C5000BCFF062000F040FE044616E06946062060
:101C600000F01BFE0BE000BFBDF80400B84206D038
:101C70000298042241460E3013F0A0FC50B1684691
:101C800000F0E9FD0500EFD0641E002C06DD002DFC
:101C9000E4D005E040460AF0A1FFF5E705B9FFDF13
:101CA000D8F800000AF0B5FF761E01D00028C9D090
:101CB000BDE8FE8390F8D01090F8730020B919B1F8
:101CC000042901D0012070470020704701780029C5
:101CD0000AD0416891F8DD20002A05D0002281F861
:101CE000DD20406807F013B870471B38E12806D2A2
:101CF000B1F5A47F03D344F29020814201D9122090
:101D0000704700207047FB2802D8B1F5296F01D930
:101D1000112070470020704770B514460546012217
:101D200000F05CF8002806D121462846BDE8704046
:101D3000002200F053B870BD042803D321B9B0F5D8
:101D4000804F01D90020704701207047042803D339
:101D500021B9B0F5804F01D90020704701207047AC
:101D6000012802D018B100207047022070470120DE
:101D7000704710B500224FF4C84408E030F8123024
:101D8000A34200D9234620F81230521CD2B28A4214
:101D9000F4D3E8E680B2C1060BD401071CD4810657
:101DA0004FEAC07101D5B9B900E099B1800713D4E9
:101DB00010E0410610D481060ED4C1074FEA8071AD
:101DC00004D0002902DB400704D405E0010703D456
:101DD000400701D401207047002070470AB101225A
:101DE00000E00222024202D1C80802D109B100205B
:101DF000704711207047000030B5058825F4004475
:101E000021448CB24FF4004194420AD2121B92B288
:101E10001B339A4201D2A94307E005F40041214354
:101E200003E0A21A92B2A9431143018030BD0844D5
:101E3000083050434A31084480B2704770B51D469F
:101E400016460B46044629463046049AFFF7EFFF34
:101E50000646B34200D2FFDF2821204613F07BFC68
:101E60004FF6FF70A082283EB0B265776080B0F573
:101E7000004F00D9FFDF618805F13C00814200D2AC
:101E8000FFDF60880835401B343880B220801B2873
:101E900000D21B2020800020A07770BD8161886166
:101EA00070472DE9F05F0D46C188044600F128090E
:101EB000008921F4004620F4004800F062FB10B1D4
:101EC0000020BDE8F09F4FF0000A4FF0010BB04535
:101ED0000CD9617FA8EB0600401A0838854219DC4E
:101EE00009EB06000021058041801AE06088617FCF
:101EF000801B471A083F0DD41B2F00DAFFDFBD42BD
:101F000001DC294600E0B9B2681A0204120C04D0C0
:101F1000424502DD84F817A0D2E709EB06000180F4
:101F2000428084F817B0CCE770B5044600F128026F
:101F3000C088E37D20F400402BB110440288438820
:101F400013448B4201D2002070BD00258A4202D387
:101F50000180458008E0891A0904090C418003D0FA
:101F6000A01D00F01EFB08E0637F008808331844C2
:101F700081B26288A01DFFF73FFFE575012070BDAB
:101F800070B5034600F12804C588808820F4004617
:101F90002644A84202D10020188270BD9889358855
:101FA000A84206D3401B75882D1A2044ADB2C01E2E
:101FB00005E02C1AA5B25C7F20443044401D0C88FB
:101FC000AC4200D90D809C8924B10024147009888A
:101FD000198270BD0124F9E770B5044600F12801AB
:101FE000808820F400404518208A002825D0A18947
:101FF000084480B2A08129886A881144814200D2B5
:10200000FFDF2888698800260844A189884212D108
:10201000A069807F2871698819B1201D00F0C1FA7C
:1020200008E0637F28880833184481B26288201D45
:10203000FFF7E2FEA6812682012070BD2DE9F04166
:10204000418987880026044600F12805B94218D046
:1020500004F10A0821F400402844418819B140469F
:1020600000F09FFA08E0637F00880833184481B2CB
:1020700062884046FFF7C0FE761C6189B6B2B9425D
:10208000E8D13046BDE8F0812DE9F04104460B4629
:1020900027892830A68827F40041B4F80A80014433
:1020A0000D46B74201D10020ECE70AB1481D10608F
:1020B00023B1627F691D184613F0ACFA2E88698837
:1020C00004F1080021B18A1996B200F06AFA06E01C
:1020D000637F62880833991989B2FFF78DFE4745FF
:1020E00001D1208960813046CCE78188C088814257
:1020F00001D101207047002070470189808881420A
:1021000001D1012070470020704770B58588C388D1
:1021100000F1280425F4004223F4004114449D42B8
:102120001AD08389058A5E1925886388EC18A6422F
:1021300014D313B18B4211D30EE0437F08325C19E4
:102140002244408892B2801A80B22333984201D24E
:1021500011B103E08A4201D1002070BD012070BDA1
:102160002DE9F0478846C1880446008921F40046DD
:1021700004F1280720F4004507EB060900F001FAF6
:10218000002178BBB54204D9627FA81B801A0025C4
:1021900003E06088627F801B801A083823D4E289BC
:1021A00062B1B9F80020B9F802303BB1E81A2177E2
:1021B000404518DBE0893844801A09E0801A21770D
:1021C00040450ADB607FE1890830304439440844E7
:1021D000C01EA4F81280BDE8F087454503DB01204E
:1021E0002077E7E7FFE761820020F4E72DE9F74F6A
